:100000000C9416240C94F4260C941F270C944A2765
:100010000C9475270C94A0270C94CB270C94F627EE
:100020000C9421280C9447240C9447240C944724C6
:100030000C9447240C9447240C9447240C94472494
:100040000C9447240D94C3420C9447240C944724E9
:100050000C9447240C9447240D94DC570C944924A9
:100060000C9447240D94681C0C9447240C9447244A
:100070000C9447240C9447240C9447240C94472454
:100080000C9447240C9447240C9447240C94472444
:100090000C9447240C9447240C9447240C9430323D
:1000A0000C9447240C9447240C9447240C94472424
:1000B0000C9447240C9447240C9447240C94472414
:1000C0000C9447240C9447240C9447240C94472404
:1000D0000C9447240C9447240C9447240C944724F4
:1000E0000C944724922597259C25A625B0252926E2
:1000F000BA25C225CA25D425DE25E825F7250126FF
:1001000029260B2615261F264D2650263F26432638
:1001100049268726542658265E26622666266C26A1
:100120007026742687267A267E268226422A422A2E
:100130004A2A522A622A6A2A722A7A2A822A5A2A3F
:100140005A017C014E014A015C01520156016C01C9
:1001500054016401560144013401300178017201F7
:100160005001560166013E013A0156016E015E01E1
:10017000620140012E014201700138014C0146012B
:1001800076013C016801600174016A014801560171
:1001900056015601560156015601560156015601A7
:1001A0005601560156015601560156015601560197
:1001B0005601560156015601560156015601560187
:1001C0005601560156015601560156015601560177
:1001D0005601560156015601560156015601560167
:1001E0005601560156015601560156015601560157
:1001F0005601560156015601560156015601560147
:10020000560156015601560136017A01084AD73B7C
:100210003BCE016E84BCBFFDC12F3D6C74319ABDD5
:1002200056833DDA3D00C77F11BED9E4BB4C3E91F9
:100230006BAAAABE000000803F05A84CCDB2D44EE8
:10024000B93836A9020C50B9918688083CA6AAAAEA
:100250002ABE000000803F000D942C1C0D944D6BB5
:100260000D94E36B0D94341C0D94246C0D947D6BF4
:100270000D94576B0D94016C0D94676B0D94066C87
:100280000D944B6B0D944F6B0D94206C0D945B6B28
:100290000D94766B0D94126C0D94596B0D94106C3B
:1002A0000D942A6C0D94166C0D941A6C0D94CA6BF7
:1002B0000D94502A0D94236B0D94146C0D943B6B8C
:1002C0000D946C6B0D943D6B0D941D6C0D94F06B47
:1002D0000D94696B0D94746B0D94186C0D940B6CEC
:1002E0000D94516B0D94286C0D946E6B0D945D6B99
:1002F0000D94266C0D94986B0D94266B00000A0BE0
:1003000002090C0D0E0807030401000000000000A4
:1003100000000000000000000000000000000000DD
:10032000000000000000000012111000000000009A
:1003300000000000000000000000000000000000BD
:1003400000000102102020080810204010204080EA
:100350000201020108040201010204081020408089
:100360008040201008040201800402018040201017
:100370000804020108040201010204081020408060
:10038000010204081020408005050505070508083E
:100390000808020202020A0A08080404040401010F
:1003A0000101010101010303030303030303040724
:1003B00007070C0C0C0C0C0C0C0C020202020606BB
:1003C0000606060606060B0B0B0B0B0B0B0B0000B1
:1003D0002200250028002B002E00310034000201ED
:1003E0000000050108010B01000021002400270086
:1003F0002A002D0030003300010100000401070134
:100400000A01476F20746F3A00737570706F7274D1
:1004100000455230370058206F7220592073776999
:1004200074636820737475636B00455230370058ED
:10043000206F722059207377697463682062726F2D
:100440006B656E0045523036005A207377697463CD
:100450006820737475636B0045523035005A207301
:1004600077697463682062726F6B656E0045523005
:1004700034005361666574792063697263756974C9
:1004800000455230330048656174657220657272B0
:100490006F7200455230320054656D702073656E86
:1004A000736F722042454400455230310054656DEF
:1004B000702073656E736F72004552524F52202D3B
:1004C0002053544F5050454400756C74696D616BF6
:1004D00065722E636F6D2F0054696E6B65725F31AC
:1004E000392E30332E3100202000000000000000A3
:1004F000000080C07098ECE6F6F6E6EC9870C0005C
:10050000000000000000000000000000000080E08B
:1005100038CEF7F9FEFFFF03010103FFFFFEFDF3F5
:10052000CE38E0C0000000000080E0709CE7F9FEDB
:10053000FFFFFFFFFFFFFF3C18183CFFFFFFFFFF1F
:10054000FFFFFCFBE79C30E080071F30276F6F6FD9
:100550006F6F6F6F6F6F6F6F6E6E6F6F6F6F6F6FAD
:100560006F6F6F6F6F27301F070908E38191B1FF2D
:10057000B09080E007081C22414141221C07081C62
:100580003E7F7F7F3E1C07087F6E6C787267420754
:10059000081C224A524C201F07087F7F415F5F7F63
:1005A0007F07087F7F5155457F7F08080982F884BF
:1005B00084F8820907086070381E09080405082AB3
:1005C0002A2A2A2A070810387C1010101E07081C37
:1005D00022404F40221C05083E3E003E3E05087F5B
:1005E0007F3E1C080708492A1C7F1C2A490B080863
:1005F000080808080808083E1C080B08081C3E08E4
:10060000080808080808080708087C466F467C08A0
:1006100006082214082214080608081422081422C6
:100620000608221408221408050826340816320782
:10063000087F5D4941495D7F07081C3E7F71773E19
:100640001C07081C22414F49221C07080708137F7A
:100650001308070708404A55404A55400508609E60
:10066000819E60801506060606FEFEFEFEFC00006A
:100670000000000000FCFEFEFEFC0000000EFEFE7E
:10068000FEFE0000E0FCFEFEFCE0E0000000CECE3E
:10069000CE000000C0C0C0C0C0C08000000000008C
:1006A0000080C0C0800000000000008080C0C0C08A
:1006B000C0C0C0C080800000000006FEFEFEFE003C
:1006C00000000080C0C0C00000000000008080C0AA
:1006D000C0C080808000000000C0C0C0C00080C0DA
:1006E000C0C0C08000000000007FFFFFFFFF80004F
:1006F0000000000080FFFFFFFFFF00000000FFFF81
:10070000FFFF000000FFFFFFFF0000000000FFFFF1
:10071000FF00000081F1FFFF3F0F3FFFFCF0F0FC06
:10072000FF3F0F3FFFFEF880000000C1E1F1F171D3
:1007300031010183FFFFFFFC000000FFFFFFFF000E
:100740000C3EFFFFF7C301000000FCFEFF87031112
:100750003131333F3F3F1E000001FFFFFFFF070322
:1007600001010101000000000000010307070F0F55
:100770000F0F0F0F0F0707070F0F06000000070FDF
:100780000F07000000070F0F0700000000000F0F09
:100790000F0000060F0F070100000001070F0F07F1
:1007A0000100000001070F0F06000003070F0F0EE6
:1007B0000E060703070F0F07000000070F0F0700C3
:1007C000000000030F0F0F060000000307070F0EC5
:1007D0000E0E0E0E0E06000000000F0F0F0F000091
:1007E00000000000004300432F0048656174696EFB
:1007F00067207072696E7468656164005072657616
:100800003A200043414E43454C002073656300206D
:100810006D696E0020686F75720020686F75727365
:100820000011150A0000191512000006090906003A
:10083000000000000000005F000000070007001437
:100840007F147F14242A7F2A1223130864623649F6
:100850005522500005030000001C224100004122E7
:100860001C00082A1C2A0808083E0808005030000E
:100870000008080808080060600000201008040252
:100880003E5149453E00427F400042615149462168
:1008900041454B311814127F1027454545393C4AD4
:1008A0004949300171090503364949493606494924
:1008B000291E0036360000005636000000081422BB
:1008C00041141414141441221408000201510906A1
:1008D000324979413E7E1111117E7F494949363EA8
:1008E000414141227F4141221C7F494949417F09C1
:1008F0000901013E414151327F0808087F00417FD4
:1009000041002040413F017F081422417F40404088
:10091000407F0204027F7F0408107F3E4141413E38
:100920007F090909063E4151215E7F091929464682
:100930004949493101017F01013F4040403F1F20AB
:1009400040201F7F2018207F63140814630304785D
:100950000403615149454300007F414102040810EE
:100960002041417F00000402010204404040404019
:10097000000102040020545454787F48444438381D
:1009800044444420384444487F3854545418087E22
:10099000090102081454543C7F0804047800447D83
:1009A00040002040443D00007F10284400417F402B
:1009B000007C041804787C080404783844444438E3
:1009C0007C14141408081414187C7C0804040848C7
:1009D00054545420043F4440203C4040207C1C2080
:1009E00040201C3C4030403C44281028440C5050CF
:1009F000503C4464544C44000836410000007F00E1
:100A000000004136080008082A1C08081C2A0808AB
:100A1000473120462569205A2569205825692059E3
:100A2000256900473238205A30205830205930008C
:100A30006275696C64706C6174652E006F6620610C
:100A4000646A757374696E6720796F757200746873
:100A5000726F756768207468652070726F63657364
:100A60007300492077696C6C20677569646520792B
:100A70006F7500434F4E54494E55450043414E4318
:100A8000454C00746F207072696E74206974210087
:100A9000616E64207072657373207468652062757E
:100AA00074746F6E006F6E207468652053442D63FC
:100AB0006172640053656C656374206120707269B3
:100AC0006E742066696C650032312F3231004C45FE
:100AD000542753205052494E540052656164696E48
:100AE0006720636172642E2E2E0032312F32310066
:100AF000796F757220556C74696D616B6572322EF9
:100B00002E2E00746861742063616D6520776974AE
:100B10006800506C6561736520696E73657274203E
:100B200053442D636172640032312F3231006D61A4
:100B30006B652061203344205072696E7421004936
:100B4000276D207265616479206C657427730032AB
:100B5000302F32310041524520594F5520524541E6
:100B600044593F0066726F6D206E6F7A7A6C652E05
:100B70002E2E006D6174657269616C2065786974F0
:100B800073005075736820627574746F6E20776897
:100B9000656E0031392F323100434F4E54494E5566
:100BA00045004C6F6164696E67206D6174657269A0
:100BB000616C2E2E2E0031382F32310061626F763B
:100BC0006520746865206172726F772E00796F7589
:100BD0007220556C74696D616B6572322C0066729F
:100BE0006F6D207468652072656172206F660049C0
:100BF0006E73657274206E6577206D6174657269BD
:100C0000616C0031372F323100434F4E54494E55FD
:100C100045006D6174657269616C206C6F61646917
:100C20006E67007072696E746865616420686561E2
:100C300074696E6720666F7200506C656173652021
:100C4000776169742C0031362F32310053656C6541
:100C5000637420746865206D6174657269616C00ED
:100C60006974206973207573696E672E006F662042
:100C70006D6174657269616C006B6E6F777320775C
:100C8000686174206B696E64004E6F7720796F75B0
:100C90007220556C74696D616B6572320031352F4D
:100CA000323100434F4E54494E554500697320740C
:100CB0006869732072696768743F00596F752068AE
:100CC0006176652063686F73656E0031342F323151
:100CD00000594553004E4F00206173206D617465CB
:100CE0007269616C2C0031332F3231004D41544513
:100CF0005249414C00556C74696D616B6572322EBE
:100D000000696E7365727420696E2074686973007F
:100D10006D6174657269616C20796F752077696C9B
:100D20006C004E6578742C2073656C656374207458
:100D300068650031322F3231005245414459004D2F
:100D40003834004731204625692058256920592527
:100D50006900746F20696E73657274206D617465CB
:100D60007269616C2E00746865206E6578742073FA
:100D700074657020697300746865206275696C64BD
:100D8000706C617465004E6F7720746861742077B1
:100D900065206C6576656C65640031312F323100F9
:100DA000434F4E54494E554500746865207269673B
:100DB000687420636F726E65722E2E2E00526570FD
:100DC000656174207468697320666F720031302F1A
:100DD000323100434F4E54494E554500444F4E4525
:100DE00000746865206C65667420636F726E65724E
:100DF0002E2E2E0052657065617420746869732010
:100E0000666F7200392F323100434F4E54494E55B0
:100E1000450062697420726573697374616E6365FD
:100E20002E00756E74696C20796F75206665656C2F
:100E30002061006275696C64706C61746520616E1C
:100E400064206E6F7A7A6C6500536C69646520610A
:100E5000207061706572206265747765656E003818
:100E60002F323100434F4E54494E554500434F4EAB
:100E700054494E554500473120462569205A3000D7
:100E800047312046256920582569205925690047A2
:100E90003120462569205A350074686520627569DD
:100EA0006C64706C617465206C6576656C2E007086
:100EB0006170657220746F2066696E652D74756E41
:100EC00065006E6F772075736520612073686565B6
:100ED00074206F6600526570656174207468697370
:100EE00020737465702C2062757400372F323100C6
:100EF000434F4E54494E55450066726F6D207468DD
:100F000065206275696C64706C6174652E0069732C
:100F10002061206D696C6C696D6574657220617704
:100F200061790073637265772074696C6C207468F2
:100F300065206E6F7A7A6C65005475726E207269E6
:100F4000676874206275696C64706C6174650036E2
:100F50002F323100434F4E54494E55450047312002
:100F6000462569205A3000473120462569205825FA
:100F7000692059256900473120462569205A3500E6
:100F800066726F6D20746865206275696C64706C40
:100F90006174652E0069732061206D696C6C696DE8
:100FA000657465722061776179007363726577207B
:100FB00074696C6C20746865206E6F7A7A6C650059
:100FC0005475726E206C656674206275696C64700D
:100FD0006C61746500352F323100434F4E54494ED9
:100FE000554500473120462569205A3000473120B9
:100FF0004625692058256920592569004731204632
:101000002569205A350066726F6D2074686520620C
:1010100075696C64706C6174652E0061206D696C1B
:101020006C696D65746572206177617900756E74A5
:10103000696C20746865206E6F7A7A6C65206973BC
:1010400000526F74617465207468652062757474F1
:101050006F6E00342F323100434F4E54494E554588
:1010600000434F4E54494E554500473120462569AF
:10107000205A2569205825692059256900676F691C
:101080006E6720746F20646F2074686174206E6FC7
:10109000772E0061646A7573746D656E74732C20AD
:1010A000776520617265007765206E6565642074E0
:1010B0006F20646F20736F6D6500416674657220E8
:1010C0007472616E73706F72746174696F6E0033E5
:1010D0002F323100434F4E54494E55450047312081
:1010E000462569205A25690061206669727374205B
:1010F00072756E2077697A6172642E0077616C6B0D
:1011000020796F75207468726F7567680066697200
:101110007374207374617274757020492077696CE0
:101120006C0042656361757365207468697320693A
:10113000732074686500322F323100434F4E54499A
:101140004E554500627574746F6E20746F20636F26
:101150006E74696E756500556C74696D616B65724E
:101160002120507265737320746865007374617216
:10117000747570206F6620796F75720057656C63A7
:101180006F6D6520746F2074686520666972737472
:1011900000312F323100434F4E54494E55450043E4
:1011A00000432F00436C69636B20746F2072657479
:1011B00075726E004275696C64706C617465207440
:1011C000656D702E3A004300432F00436C69636BDA
:1011D00020746F2072657475726E004E6F7A7A6C2F
:1011E000652074656D70657261747572653A003F53
:1011F0003F3F004578706572742066756E63746950
:101200006F6E730041646A757374206275696C64F3
:10121000706C617465005365742066616E20737034
:10122000656564004D6F7665206D617465726961F6
:101230006C00496E73657274206D617465726961CA
:101240006C005261697365206275696C64706C61D1
:101250007465004C6F776572206275696C64706CA0
:1012600061746500486F6D6520686561640048655C
:1012700061747570206275696C64706C617465006E
:10128000486561747570206E6F7A7A6C6500507273
:1012900065666572656E636573003C205245545502
:1012A000524E002500432F004300432F0043003FD0
:1012B0003F3F00466163746F727920726573657495
:1012C0000052756E74696D65207374617473005695
:1012D000657273696F6E00506F7765722062756416
:1012E000676574005072696E742061726561004DAB
:1012F0006F74696F6E2073657474696E67730052E2
:10130000657472616374696F6E2073657474696E5D
:1013100067730054656D70657261747572652063E2
:101320006F6E74726F6C00486561746572207469C9
:101330006D656F75740053637265656E20636F6EC3
:10134000747261737400536C6565702074696D65A7
:1013500072005363726F6C6C2066696C656E616DB0
:10136000657300436C69636B20736F756E64004C2A
:1013700045442073657474696E67730055736572B4
:1013800020696E74657266616365003C2052455445
:1013900055524E0054696E6B65725F31392E303391
:1013A0002E31006F66660073006F6666202F200086
:1013B0006D696E202F2000250044697361626C65A1
:1013C0006400456E61626C6564005374616E6461B3
:1013D00072640053686F7274207469636B004F66A7
:1013E000660025005374616E64617264204D6F6401
:1013F00065004765656B204D6F6465003F3F3F00AA
:101400004765656B204D6F6465003E005374616EE7
:1014100064617264204D6F6465003E003C2052455B
:101420005455524E005573657220696E746572662C
:10143000616365003F3F3F0020476C6F772077680E
:10144000656E20646F6E6500204F6E207768696C52
:1014500065207072696E74696E670020416C7761F7
:101460007973204F66660020416C77617973204F55
:101470006E004272696768746E657373003C205237
:10148000455455524E002500250042726967687424
:101490006E657373004C454400203F3F3F004F662C
:1014A00066003E0053686F7274207469636B003E7F
:1014B000005374616E646172642062656570003E01
:1014C000003C2052455455524E00436C69636B20DA
:1014D000736F756E64005363726F6C6C2066696C19
:1014E000656E616D6573003E004E6F207363726FB1
:1014F0006C6C696E67003E003C2052455455524E5C
:10150000005363726F6C6C2066696C656E616D650B
:1015100073002500436C69636B20746F20726574DF
:1015200075726E0053637265656E20636F6E7472C0
:10153000617374003F3F3F00496E766572742061AD
:1015400078697300417869732073746570732F6DC7
:101550006D004D6F746F722043757272656E74000A
:101560004D61782E20617869732073706565640021
:10157000416363656C65726174696F6E003C2052F3
:10158000455455524E004D4F54494F4E0054696ECC
:101590006B65725F31392E30332E31004D61722010
:1015A000203820323031392031383A33343A353826
:1015B0000052657475726E006D00204D61743A00C2
:1015C0003A005072696E74696E673A003A004D6174
:1015D0006368696E65206F6E20666F723A005265AF
:1015E0007475726E00746F2064656661756C743F0B
:1015F0000052657365742065766572797468696EEA
:101600006700594553004E4F0050524546455245DC
:101610004E43455300250046616E20737065656436
:10162000004731205A343000414456414E4345442E
:1016300000432F004300436C69636B20746F20727A
:10164000657475726E00526F7461746520746F20DA
:1016500065787472756465004E6F7A7A6C65207473
:10166000656D70657261747572653A004732380055
:10167000473238205A30004732382058302059300D
:10168000004255494C442D7C504C41544500414446
:1016900056414E4345440052455455524E00545015
:1016A0004C410050500054505520393541004350B2
:1016B000452B004E796C6F6E00504300435045003F
:1016C00041425300504C41006C63645F6D6174652E
:1016D0007269616C5F72657365745F64656661757C
:1016E0006C747300496D706F72742066726F6D2038
:1016F0005344004578706F727420746F2053440017
:10170000437573746F6D697A65003C20524554557A
:10171000524E004C6F61647320616C6C206D61747B
:10172000657269616C7300536176657320616C6CDE
:10173000206D6174657269616C73004D6F646966D8
:1017400079207468652073657474696E6773002509
:101750000046616E3A2000430043002500466C6F4E
:10176000773A006D6D003F3F3F0053746F72652004
:1017700061732070726573657400466C6F77202505
:101780000046616E004469616D657465720048656C
:1017900061746564206275696C64706C6174650065
:1017A00054656D7065726174757265003C205245B8
:1017B0005455524E00250025006D6D004300432016
:1017C0000043200054656D70657261747572653AEE
:1017D00020003C2052455455524E004300430054D3
:1017E000656D7065726174757265004D4154455246
:1017F00049414C004E657720707265736574003CFA
:101800002052455455524E005052455345545300B2
:1018100025004D6174657269616C20666C6F77009C
:10182000250046616E207370656564006D6D004D26
:101830006174657269616C204469616D657465727B
:101840000043004275696C64706C61746520546576
:101850006D702E004D4154455249414C00696E2037
:101860004D4154455249414C2E54585400746F20F8
:101870007468652053442063617264005361766527
:1018800064206D6174657269616C73004F4B000A6E
:10189000006469616D657465723D000A00666C6F75
:1018A000773D000A0066616E5F73706565643D0098
:1018B0000A006265645F74656D706572617475724B
:1018C000653D000A003D0072657472616374696F62
:1018D0006E5F73706565645F000A003D0072657439
:1018E00072616374696F6E5F6C656E6774685F00C8
:1018F0000A003D0074656D70657261747572655F94
:10190000000A0074656D70657261747572653D00E2
:101910000A006E616D653D005B6D617465726961A1
:101920006C5D0A0052656164696E67206361726470
:101930002E2E2E00506C6561736520696E73657282
:10194000742063617264004E6F2053442D434152F2
:10195000442100696E76616C6964200066726F6D67
:10196000207468652053442063617264004C6F6189
:10197000646564206D6174657269616C73004F4BBE
:101980000072657472616374696F6E5F7370656510
:10199000645F0072657472616374696F6E5F6C6519
:1019A0006E6774685F0074656D70657261747572DE
:1019B000655F006469616D6574657200666C6F7760
:1019C0000066616E5F7370656564006265645F7474
:1019D000656D70657261747572650074656D7065B2
:1019E00072617475726500416464696E67206D612F
:1019F00074657269616C20006E616D65005B6D617C
:101A000074657269616C5D005374617274207265F3
:101A10006164206D6174657269616C7300666F75D5
:101A20006E64206F6E20636172642E004E6F206DB5
:101A30006174657269616C2066696C6500526561EC
:101A400064696E6720636172642E2E2E00506C658F
:101A500061736520696E73657274206361726400DE
:101A60004E6F2053442D43415244210053656C6511
:101A700063746564206D6174657269616C3A004FCE
:101A80004B004D4154455249414C00636F6D6573A5
:101A9000206F757420746865206E6F7A7A6C6500AB
:101AA000576169742074696C6C206D61746572692A
:101AB000616C0052454144590043414E43454C003E
:101AC000466F7277617264696E67206D61746572CA
:101AD00069616C0061626F7665207468652061726F
:101AE000726F772E00796F7572206D616368696E11
:101AF000652C0066726F6D20746865206261636B8F
:101B000073696465206F6600496E73657274206E38
:101B10006577206D6174657269616C00524541445E
:101B2000590043414E43454C006D617465726961D3
:101B30006C20696E73657274696F6E00436F6F6CB1
:101B4000696E67206E6F7A7A6C6520666F720048E6
:101B5000656174696E67206E6F7A7A6C6520666F56
:101B60007200250046616E3A2000430043002500C4
:101B7000466C6F773A006D6D004D415445524941B6
:101B80004C0052656D6F7665206D61746572696198
:101B90006C0052454144590043414E43454C00526C
:101BA0006576657273696E67206D617465726961CF
:101BB0006C00666F72206D6174657269616C207271
:101BC000656D6F76616C00436F6F6C696E67206E38
:101BD0006F7A7A6C650048656174696E67206E6F14
:101BE0007A7A6C65004348414E474500534554544A
:101BF000494E47530052455455524E004D383420FB
:101C0000582059204500473120462569205825692C
:101C100020592569006563686F3A004572726F72DA
:101C20003A0041424F52540041424F5254005455E1
:101C30004E450054554E45004D4154455249414C86
:101C4000004348414E4745004D4154455249414C9F
:101C5000004348414E474500524553554D457C0091
:101C600050415553494E477C004241434B0042414D
:101C7000434B0054554E450054554E450041424F8C
:101C800052547C0050415553457C004D3630312034
:101C900058257520592575205A2575204C25750025
:101CA0003F3F3F00536C6565702074696D6572003D
:101CB0004D6F7665206D6174657269616C004C458D
:101CC00044204272696768746E657373005265746C
:101CD00072616374696F6E004D6174657269616CE5
:101CE00020666C6F770046616E20737065656400D6
:101CF0004275696C64706C6174652074656D702EDA
:101D00000054656D7065726174757265005370651D
:101D10006564003C2052455455524E002500250074
:101D20002500432F004300432F00430025003F3F81
:101D30003F00456E64206F66207072696E74206C7F
:101D4000656E6774680052657472616374207370A5
:101D50006565640052657472616374206C656E67BA
:101D60007468003C2052455455524E006D6D006D14
:101D70006D2F736563006D6D006D6D00456E6420A1
:101D80006F66207072696E7420726574726163741C
:101D9000006D6D2F7365630052657472616374200A
:101DA0007370656564006D6D005265747261637473
:101DB000206C656E67746800524554524143544923
:101DC0004F4E0025004272696768746E6573730038
:101DD00025004D6174657269616C20666C6F7700D7
:101DE000250046616E2073706565640025005072A1
:101DF000696E742073706565640054554E450043E8
:101E000000432F00436C69636B20746F207265740C
:101E100075726E004E6F7A7A6C652074656D7065B0
:101E2000726174757265005072696E742066696EB5
:101E30006973686564005072696E74657220636FBF
:101E40006F6C696E6720646F776E004300432000FB
:101E500068006D696E0054696D6520004241434B16
:101E600020544F204D454E550041626F7274696E8B
:101E7000672E2E2E0041626F727420746865207088
:101E800072696E743F00594553004E4F00507265A1
:101E9000706172696E6720746F207072696E743A37
:101EA0000048656174696E672075702E2E2E00548F
:101EB000554E450041424F52540025732076732001
:101EC0002573006D6174657269616C2E00666F72B6
:101ED000206120646966666572656E740054686985
:101EE000732066696C65206973206372656174652F
:101EF0006400434F4E54494E55450043414E4345BF
:101F00004C0054696D65206C6566740054696D659C
:101F1000206C65667420756E6B6E6F776E00432F54
:101F200000430048656174696E67206275696C647E
:101F3000706C61746500432F0043004865617469EB
:101F40006E67005072696E74696E673A0054554E40
:101F5000450050415553450066726F6D20746865A9
:101F600020736C696365722E0073657474696E67A3
:101F700020776974682073657474696E67006F7682
:101F8000657272696465206D616368696E6500548D
:101F90006869732066696C652077696C6C00434FD3
:101FA0004E54494E55450043414E43454C003C205C
:101FB0004241434B003C2052455455524E0053443D
:101FC00020434152440047312046313230303020E6
:101FD00058256920592569003B464C41564F523AD5
:101FE000556C746947436F6465003B464C41564FDE
:101FF000523A556C746947436F6465004E6F2066B2
:10200000696C657320666F756E6421004F4B004FDD
:102010004B0052656164696E6720636172642E2EA5
:102020002E00506C6561736520696E736572742053
:1020300063617264004E6F2053442D43415244212A
:10204000004E6F20696E666F20617661696C616217
:102050006C65004E6F7A7A6C6520006D006D004DE6
:102060006174657269616C200068006D696E00546E
:10207000696D6520003B4D545950453A003B4E4F29
:102080005A5A4C455F4449414D455445523A003BEC
:102090004D4154455249414C3A003B54494D453A13
:1020A00000466F6C646572006F66207072696E74B2
:1020B000696E6720617265610054726965642070A1
:1020C00072696E74696E67206F7574004552524F65
:1020D000523A0052455455524E20544F204D4149DA
:1020E0004E00756C74696D616B65722E636F6D2F38
:1020F0004552303800476F20746F3A007265616452
:10210000696E672053442D636172642100457272C9
:102110006F72207768696C650052455455524E20A5
:10212000544F204D41494E001F001F2F001F0042F9
:1021300075696C64706C61746520001F001F2F004E
:102140001F004E6F7A7A6C6520006F6666006F6EB6
:10215000004275696C64706C6174653A20006F664A
:1021600066006F6E004E6F7A7A6C653A20004241CD
:10217000434B004241434B0052657475726E2074AC
:102180006F206D61696E206D656E7500434F4F4C19
:1021900000434F4F4C00436F6F6C20646F776E208D
:1021A000616C6C005052494E54005052494E5400DC
:1021B0005374617274207072696E74005072656835
:1021C000656174001F002F001F002F004D41544512
:1021D0005249414C005354415254004348414E47E8
:1021E00045004D4F56450053455454494E47530002
:1021F000414456414E434544005052494E540050CC
:10220000524548454154004D41494E54454E414E7A
:102210004345004D4154455249414C005052494EAE
:102220005400570045787472756465720057617484
:102230007461676520457874727564657200570033
:102240004275696C64706C61746500576174746187
:102250006765204275696C64706C61746500570035
:10226000546F74616C00546F74616C20506F7765AB
:102270007220427564676574004241434B004241DD
:10228000434B00436C69636B20746F2072657475F7
:10229000726E0053544F52450053746F7265206F35
:1022A0007074696F6E7300506F7765722042756449
:1022B000676574004B640044657269766174697681
:1022C0006520636F6566662E004B6900496E746514
:1022D0006772616C20636F656666696369656E74B9
:1022E000004B700050726F706F7274696F6E616C2A
:1022F00020636F6566662E004241434B00424143B6
:102300004B00436C69636B20746F20726574757247
:102310006E004155544F005374617274205049440B
:10232000206175746F74756E650053544F5245008B
:1023300053746F7265205049442073657474696EDC
:102340006773005049442073657474696E67730045
:1023500045787472756465720043414E43454C0084
:1023600054696D656F7574006661696C6564210000
:10237000504944204175746F74756E650054656DE5
:10238000706572617475726520746F6F206869671B
:1023900068006661696C656421005049442041759C
:1023A000746F74756E650074686520736574746904
:1023B0006E67732E00596F752063616E2073746FA2
:1023C00072650066696E69736865642100504944EE
:1023D000204175746F74756E6500434F4E54494EBD
:1023E0005545001F2F001F004275696C64706C61B9
:1023F0007465004578747275646572001F2F001F44
:10240000002F002E005049442074756E696E6700DD
:102410004379636C65730074756E696E67206379C8
:10242000636C6573001F0054656D7065726174752F
:1024300072650074756E696E672074656D70657283
:102440006174757265004241434B004241434B0049
:10245000436C69636B20746F2072657475726E00D3
:1024600053544152540053746172742050494420B3
:102470006175746F74756E65005049442074756E93
:1024800065206F7074696F6E73004578747275643F
:102490006572004275696C64706C617465004B64B0
:1024A000004465726976617469766520636F65665C
:1024B000662E004B6900496E74656772616C20631B
:1024C0006F656666696369656E74004B7000507273
:1024D0006F706F7274696F6E616C20636F65666692
:1024E0002E004275696C642D7C706C6174650050BF
:1024F0004944206D6F6465004241434B00424143B3
:102500004B00436C69636B20746F20726574757245
:102510006E004155544F0053746172742050494409
:10252000206175746F74756E650053544F52450089
:1025300053746F7265205049442073657474696EDA
:102540006773005049442073657474696E67730043
:10255000504944206F6666004558545255444552D0
:10256000004255494C442D7C504C41544500524545
:102570005455524E006F66660020736563004D61CE
:10258000782E20706F77657200506572696F6420D5
:102590006F66206D61782E20706F776572006F66B0
:1025A0006600206D696E0054696D656F7574004931
:1025B000646C652074696D656F7574004241434BAE
:1025C000004241434B00436C69636B20746F20727F
:1025D000657475726E0053544F52450053746F7298
:1025E00065206F7074696F6E730048656174657201
:1025F00020636865636B006D6D2F7300582F592041
:102600004A65726B004D61782E20582F59204A651B
:10261000726B006D6D2F731E00416363656C00412A
:102620006363656C65726174696F6E004241434B10
:10263000004241434B00436C69636B20746F20720E
:10264000657475726E0053544F52450053746F7227
:10265000652073657474696E677300416363656CAC
:1026600065726174696F6E006D6D2F730045004D6A
:1026700061782E2073706565642045006D6D2F7341
:10268000005A004D61782E207370656564205A00F1
:102690006D6D2F730059004D61782E207370656544
:1026A000642059006D6D2F730058004D61782E2005
:1026B00073706565642058004241434B00424143BA
:1026C0004B00436C69636B20746F20726574757284
:1026D0006E0053544F52450053746F7265207365FA
:1026E0007474696E6773004D61782E205370656550
:1026F00064004500457874727564657220286D41E8
:1027000029005A005A206178697320286D412900F8
:10271000582F5900582F59206178697320286D412E
:1027200029004241434B004241434B00436C6963E3
:102730006B20746F2072657475726E0053544F5223
:10274000450053746F72652073657474696E6773A6
:10275000004D6F746F722043757272656E74006DF8
:102760006D00456E64206C656E67746800456E642C
:10277000206F66207072696E74206C656E67746875
:10278000006D6D2F730052657472616374207370F5
:10279000656564006D6D005265747261637400520A
:1027A000657472616374206C656E67746800424181
:1027B000434B004241434B00436C69636B20746F91
:1027C0002072657475726E0053544F5245005374F5
:1027D0006F72652073657474696E677300526574F7
:1027E00072616374696F6E2073657474696E677368
:1027F000006E6F00796573003A00496E76657274F9
:102800000045004578747275646572005A005A007C
:1028100059005900580058004241434B004241437F
:102820004B00436C69636B20746F20726574757222
:102830006E0053544F52450053746F726520696E99
:102840007665727420666C61677300496E76657296
:102850007420617869730045004520737465707356
:102860002F6D6D005A005A2073746570732F6D6D53
:10287000005900592073746570732F6D6D005800F6
:10288000582073746570732F6D6D004241434B0087
:102890004241434B00436C69636B20746F20726547
:1028A0007475726E0053544F52450053746F7265C5
:1028B0002073746570732F6D6D0041786973207398
:1028C000746570732F6D6D006D6D005A004D6178E9
:1028D000696D756D205A20636F6F7264696E6174E3
:1028E00065006D6D002D004D6178696D756D205925
:1028F00020636F6F7264696E617465006D6D00595D
:10290000004D696E696D756D205920636F6F72643B
:10291000696E617465006D6D002D004D6178696DA3
:10292000756D205820636F6F7264696E6174650005
:102930006D6D0058004D696E696D756D205820638E
:102940006F6F7264696E617465004241434B00426F
:1029500041434B00436C69636B20746F2072657454
:1029600075726E0053544F52450053746F72652058
:1029700061786973206C696D697473005072696E57
:10298000742061726561002500476C6F77004C45CB
:102990004420736C65657020676C6F77006F6666A6
:1029A0000025004C434420736C65657020636F6E96
:1029B00074726173740053637265656E006F66664E
:1029C000006D696E0053637265656E2074696D6594
:1029D0006F75740025004C454420736C656570204C
:1029E0006272696768746E657373004C69676874B6
:1029F000006F6666006D696E004C45442074696D19
:102A0000656F7574004241434B004241434B0043A4
:102A10006C69636B20746F2072657475726E0053FD
:102A2000544F52450053746F7265206F7074696F14
:102A30006E7300536C6565702074696D6572004734
:102A400031204631323030302058256920592569EF
:102A5000006D6D00526F7461746520746F2065782D
:102A6000747275646500526573657420706F736964
:102A700074696F6E00436C69636B202620686F6C0D
:102A80006420746F206C6F616400436C69636B2019
:102A90002620686F6C6420746F2070756C6C001F4A
:102AA000001F2F001F2F001F004E6F7A7A6C6520C9
:102AB00000546F67676C65206865617465720042D9
:102AC00041434B004241434B00436C69636B2074AC
:102AD0006F2072657475726E0054554E45005455E2
:102AE0004E45004D6F7265206F7074696F6E730094
:102AF0004D6F7665206D6174657269616C004D384B
:102B000034205830205930004D3834205830205966
:102B1000300047312046313230303020582569208E
:102B2000592569004D383420583020593000446907
:102B30007361626C652058592D737465707065728D
:102B4000730044697361626C652058592D73746514
:102B50007070657273004D6F7665206865616420E2
:102B6000746F2066726F6E74004D6F7665206865B5
:102B7000616420746F2066726F6E7400486F6D65BB
:102B8000206865616400486F6D6520686561640058
:102B90004241434B004241434B00436C69636B200D
:102BA000746F2072657475726E0053656C65637422
:102BB000206F7074696F6E004D38342045300047C7
:102BC000323820583000473238205930006D6D00BF
:102BD0006D6D2F7300486F6D65205A2061786973A1
:102BE000005A206178697320706F736974696F6E21
:102BF000005A004D6F7665205A206178697300484D
:102C00006F6D65205920617869730059206178697A
:102C10007320706F736974696F6E0059004D6F7621
:102C2000652059206178697300486F6D65205820D0
:102C3000617869730058206178697320706F7369D7
:102C400074696F6E0058004D6F766520582061786A
:102C50006973004241434B004241434B00436C695E
:102C6000636B20746F2072657475726E0020414C26
:102C70004C00486F6D6520616C6C20617865730055
:102C80004D6F76652061786973003F3F3F0044696E
:102C90007361626C65207374657070657273005245
:102CA00065636F766572207072696E740041646A44
:102CB000757374205A20706F736974696F6E004D5C
:102CC0006F76652061786973003C205245545552F7
:102CD0004E004D3834004578706572742066756E0C
:102CE0006374696F6E73006D6D005A005265636F97
:102CF000766572207072696E742066726F6D005214
:102D000065636F7665722068656967687400434122
:102D10004E43454C00436C69636B20746F207265B1
:102D20007475726E005052494E540053746172743F
:102D3000207072696E74005265636F7665722070E0
:102D400072696E740041424F52540041424F5254D6
:102D50000041626F7274207072696E740054554E37
:102D6000450054554E450054756E65206D656E7571
:102D700000202F20005A0052656164696E6720664A
:102D8000696C652E2E2E006D6D005A0074686520EA
:102D90006275696C64706C617465006E6F7A7A6CD0
:102DA0006520746F7563686573004D6F7665205A92
:102DB00020756E74696C20746865004D3834205835
:102DC0003020593000473120462569205A25692096
:102DD0005825692059256900473238205A30205833
:102DE00030205930006D6D005A0043414E43454C30
:102DF0000053544F524500746865206275696C64D5
:102E0000706C617465006E6F7A7A6C6520746F7592
:102E100063686573004D6F7665205A20756E74691E
:102E20006C20746865004D383420583020593000CB
:102E300053746F7265205A206F6666736574006DF7
:102E40006D005A004261627973746570205A206186
:102E5000786973006D6D0059004261627973746521
:102E60007020592061786973006D6D0058004261CF
:102E700062797374657020582061786973004241EB
:102E8000434B004241434B00436C69636B20746FBA
:102E90002072657475726E00426162797374657038
:102EA00070696E67001F001F2F001F004275696C5C
:102EB00064706C6174652000250046616E001F001F
:102EC0001F2F001F004E6F7A7A6C65200025006D61
:102ED0006D2F73005370656564200025006D6D1DB6
:102EE0002F7300466C6F7720005A0042616279733D
:102EF00074657070696E6700476F746F20706167EA
:102F000065203200436F6E74726F6C206F7074694D
:102F10006F6E7300546F67676C65204C4544006D9D
:102F20006D2F7300582F59204A65726B004D6178E0
:102F30002E20582F59204A65726B006D6D2F731E1D
:102F400000416363656C00416363656C6572617425
:102F5000696F6E006D6D2F730052657472616374DA
:102F6000207370656564006D6D00526574726163F5
:102F7000740052657472616374206C656E67746866
:102F800000546F67676C65204C454400436F6E7456
:102F9000726F6C206F7074696F6E7300476F746F1F
:102FA000207061676520310055534220636F6D6D5D
:102FB000756E69636174696F6E2E2E2E00486561AF
:102FC00074696E67206275696C64706C6174650009
:102FD00048656174696E67206E6F7A7A6C6500501F
:102FE000617573696E672E2E2E00436C69636B20CA
:102FF000746F20636F6E74696E75652E2E2E00508F
:1030000061757365642E2E2E0025005061757369FD
:103010006E672E2E2E005061757365642E2E2E0065
:103020001F001F2F001F004275696C64706C617473
:103030006520001F001F2F001F004E6F7A7A6C65FD
:10304000200041424F52540041424F5254004162CD
:103050006F7274207072696E740054554E4500543E
:10306000554E450054756E65206D656E75001F00E8
:103070002F001F002F00250048656174696E6720CE
:1030800075702E2E2E2000436865636B2066656583
:103090006465722E005072696E742070617573657C
:1030A000642E006973737565206465746563746567
:1030B000642E004D6174657269616C207472616E7A
:1030C00073706F727400434F4E54494E5545005013
:1030D00072696E74207061757365642E2043686533
:1030E000636B206665656465722E004D6174657260
:1030F00069616C207472616E73706F727420697391
:103100007375652064657465637465642E0065631A
:10311000686F3A004572726F723A005072696E744D
:1031200065722073746F70706564206475652074B7
:103130006F206572726F72732E20466978207468F2
:1031400065206572726F7220616E642075736520F0
:103150004D39393920746F20726573746172742E21
:10316000202854656D70657261747572652069738D
:103170002072657365742E20536574206974206114
:10318000667465722072657374617274696E672902
:10319000005072696E7465722068616C7465642E8B
:1031A000206B696C6C28292063616C6C656421005C
:1031B0004D32313820496E76616C696420657874CF
:1031C000727564657220004D31303920496E766128
:1031D0006C696420657874727564657220004D3185
:1031E000303520496E76616C69642065787472753B
:1031F00064657220004D31303420496E76616C690F
:1032000064206578747275646572200020403A000D
:103210002042403A00202F0020423A00202F002078
:10322000543A006F6B00456E6473746F7020737452
:10323000696C6C2070726573736564206166746577
:1032400072206261636B696E67206F66662E20452F
:103250006E6473746F7020737475636B3F00456E9A
:103260006473746F70206E6F742070726573736511
:103270006420616674657220686F6D696E67206492
:103280006F776E2E20456E6473746F702062726F5C
:103290006B656E3F00456E6473746F70206E6F7463
:1032A000207072657373656420616674657220684E
:1032B0006F6D696E6720646F776E2E20456E647344
:1032C000746F702062726F6B656E3F002200556EE6
:1032D0006B6E6F776E20636F6D6D616E643A202246
:1032E00000456C656374726F6E6963735F746573B8
:1032F00074004163746976652045787472756465FD
:10330000723A2000496E76616C6964206578747247
:103310007564657200540020423A300020423A3110
:10332000006F6B20523A00726573756D6500206402
:103330003A0020693A0020703A006F6B0020643A2E
:103340000020693A0020703A006F6B002200556E31
:103350006B6E6F776E20636F6D6D616E643A2022C5
:10336000006F70656E00545249474745524544000E
:103370007A5F6D61783A20006F70656E0054524933
:1033800047474552454400795F6D61783A20006FA8
:1033900070656E0054524947474552454400785F76
:1033A0006D696E3A20005265706F7274696E6720A5
:1033B000656E6473746F7020737461747573004606
:1033C00049524D574152455F4E414D453A4D61720C
:1033D0006C696E20556C74696D616B6572323B204F
:1033E000537072696E7465722F6772626C206D61C2
:1033F0007368757020666F722067656E3620464967
:10340000524D574152455F55524C3A687474703A68
:103410002F2F6769746875622E636F6D2F556C74FA
:10342000696D616B65722050524F544F434F4C5F32
:1034300056455253494F4E3A312E30204D41434864
:10344000494E455F545950453A556C74696D616BEE
:1034500065722045585452554445525F434F554E6E
:10346000543A310A00453A005A3A00593A0020438A
:103470006F756E7420583A2000453A005A3A005948
:103480003A00583A003F0020573A002569206D69FC
:103490006E2C2025692073656300456E6420666983
:1034A0006C65206C69737400426567696E2066699B
:1034B0006C65206C69737400726573756D6500705E
:1034C0006175736500256920686F757273202569C1
:1034D000206D696E7574657300446F6E652070723F
:1034E000696E74696E672066696C65006F6B005267
:1034F0006573656E643A20005072696E746572205F
:1035000073746F707065642064756520746F2065D6
:1035100072726F72732E2046697820746865206518
:1035200072726F7220616E6420757365204D393937
:103530003920746F20726573746172742E20285460
:10354000656D70657261747572652069732072654E
:103550007365742E205365742069742061667465E8
:10356000722072657374617274696E6729004E6FA0
:10357000204C696E65204E756D62657220776974A6
:103580006820636865636B73756D2C204C61737480
:10359000204C696E653A20004E6F20436865636B6E
:1035A00073756D2077697468206C696E65206E751F
:1035B0006D6265722C204C617374204C696E653AA3
:1035C0002000636865636B73756D206D69736D6151
:1035D0007463682C204C617374204C696E653A20CA
:1035E000004C696E65204E756D62657220697320AE
:1035F0006E6F74204C617374204C696E65204E753B
:103600006D6265722B312C204C617374204C696E95
:10361000653A20004D313130002020506C616E6ED3
:10362000657242756666657242797465733A200008
:103630002046726565204D656D6F72793A20004DA8
:103640006172202038203230313900436F6D70694B
:103650006C65643A200054696E6B65725F31392E77
:1036600030332E3100207C20417574686F723A200F
:10367000004D617220203820323031392031383A03
:1036800033353A303000204C6173742055706461DA
:103690007465643A2000312E302E30004D61726C1A
:1036A000696E200020536F667477617265205265E1
:1036B00073657400205761746368646F6720526596
:1036C000736574002042726F776E206F757420529C
:1036D00065736574002045787465726E616C205264
:1036E0006573657400506F7765725570007374610F
:1036F0007274002200656E717565696E6720220024
:10370000446F6E6520736176696E672066696C65CB
:103710002E006F6B004D3239002F2F616374696F7B
:103720006E3A00FF01010000E0400000E0400000B0
:10373000E0406563686F3A004572726F723A00004C
:10374000002110422063308440A550C660E7700815
:103750008129914AA16BB18CC1ADD1CEE1EFF1319C
:1037600012100273325222B5529442F772D6623965
:103770009318837BB35AA3BDD39CC3FFF3DEE362EC
:1037800024433420040114E664C774A44485546AB5
:10379000A54BB528850995EEE5CFF5ACC58DD5537C
:1037A00036722611163006D776F6669556B4465B05
:1037B000B77AA719973887DFF7FEE79DD7BCC7C44C
:1037C00048E5588668A7784008611802282338CC55
:1037D000C9EDD98EE9AFF9488969990AA92BB9F5DC
:1037E0005AD44AB77A966A711A500A333A122AFDA5
:1037F000DBDCCBBFFB9EEB799B588B3BBB1AABA6AC
:103800006C877CE44CC55C222C033C600C411CAEF4
:10381000ED8FFDECCDCDDD2AAD0BBD688D499D97BB
:103820007EB66ED55EF44E133E322E511E700E9F44
:10383000FFBEEFDDDFFCCF1BBF3AAF599F788F880B
:1038400091A981CAB1EBA10CD12DC14EF16FE180DC
:1038500010A100C230E3200450254046706760B9D3
:10386000839893FBA3DAB33DC31CD37FE35EF3B12C
:10387000029012F322D2323542145277625672EA23
:10388000B5CBA5A89589856EF54FE52CD50DC5E27C
:1038900034C324A01481046674476424540544DBB3
:1038A000A7FAB79987B8975FE77EF71DC73CD7D3CC
:1038B00026F2369106B01657667676154634564C83
:1038C000D96DC90EF92FE9C899E9898AB9ABA9441C
:1038D00058654806782768C018E1088238A3287D13
:1038E000CB5CDB3FEB1EFBF98BD89BBBAB9ABB756C
:1038F0004A545A376A167AF10AD01AB32A923A2EE3
:10390000FD0FED6CDD4DCDAABD8BADE89DC98D26BB
:103910007C076C645C454CA23C832CE01CC10C1FF2
:10392000EF3EFF5DCF7CDF9BAFBABFD98FF89F170B
:103930006E367E554E745E932EB23ED10EF01E7CD6
:103940003C3E5E2B3D3F2F5B5D3B2C2A225C0020E2
:10395000746F6F206C6F6E67206578747275736911
:103960006F6E2070726576656E7465640020636F9B
:103970006C6420657874727573696F6E20707265FF
:1039800076656E746564006563686F3A00205A3A24
:103990000020593A0020583A00656E6473746F70C5
:1039A00073206869743A200024F4D43050C38E2008
:1039B000C2A24017828B7011127A910D816CD90AC4
:1039C000A861E108C7586607615143061E4B5D05B3
:1039D000C145A7041A411104093D98037139310307
:1039E0004036DB0265339102D4305402802E1D0232
:1039F000632CEE01752AC501B028A00110278101B2
:103A00008F2564012B244B01E0223401AC211F01DE
:103A10008D200D01801FFC00841EED00971DDF002E
:103A2000B81CD200E61BC600201BBC00641AB20002
:103A3000B219A8000A19A0006A189900D1179100BC
:103A400040178B00B516840031167E00B31579003F
:103A50003A157300C7146F0058146A00EE1366001D
:103A60008813630025135E00C7125B006C125700B9
:103A700015125400C111510070114F0021114B005B
:103A8000D61049008D104700461044000210420035
:103A9000C00F4000800F3E00420F3C00060F3B006D
:103AA000CB0E3800930E37005C0E3500270E340025
:103AB000F30D3200C10D3100900D3000600D2E006D
:103AC000320D2D00050D2C00D90C2B00AE0C290059
:103AD000850C29005C0C2700350C27000E0C2600F5
:103AE000E80B2400C40B2400A00B23007D0B230053
:103AF0005A0B2100390B2100180B2000F80A1F0077
:103B0000D90A1E00BB0A1E009D0A1D00800A1D0066
:103B1000630A1C00470A1B002C0A1B00110A1A002A
:103B2000F7091A00DD091900C4091900AB091900C9
:103B3000920917007B091800630917004C09160049
:103B400036091600200916000A091500F5081500A7
:103B5000E0081400CC081400B8081400A4081400ED
:103B6000900813007D0812006B081300580812001B
:103B70004608120034081100230811001208110031
:103B800001081100F0071000E0071000D007100036
:103B9000C0071000B0070F00A107100091070E002A
:103BA00083070F0074070F0065070E0057070E000C
:103BB00049070E003B070D002E070E0020070D00E1
:103BC00013070D0006070D00F9060C00ED060D00A9
:103BD000E0060C00D4060C00C8060C00BC060C0065
:103BE000B0060C00A4060B0099060C008D060B0015
:103BF00082060B0077060B006C060B0061060A00BC
:103C000057060B004C060A0042060A0038060A0056
:103C10002E060A0024060A001A060A0010060900E9
:103C200007060A00FD050900F4050900EB05090077
:103C3000E2050900D9050900D0050900C7050900FA
:103C4000BE050900B5050800AD050800A505090079
:103C50009C050800940508008C05080084050800F0
:103C60007C050800740508006C0507006505080060
:103C70005D050700560508004E05070047050700CB
:103C80004005080038050700310507002A05070030
:103C9000230507001C050600160507000F05070091
:103CA0000805060002050700FB040600F5040700EE
:103CB000EE040600E8040600E2040700DB04060048
:103CC000D5040600CF040600C9040600C30406009C
:103CD000BD040600B7040600B1040500AC040600EC
:103CE000A6040600A00405009B0406009504050038
:103CF000900406008A04050085040500800406007F
:103D00007A04050075040500700405006B040500C5
:103D100066040500610405005C0405005704050005
:103D2000520405004D040500480405004304050045
:103D30003E0404003A040500350405003004040084
:103D40002C04050027040400230405001E040400BD
:103D50001A04040016040500110404000D040400F4
:103D6000090405000404040000040400FC0304002A
:103D7000F8030400F4030400F0030400EC0304005F
:103D8000E8030400E4030400E0030400DC0304008F
:103D9000D8030400D4030400D0030400CC030400BF
:103DA000C8030300C503030024F404D9201BC40C7A
:103DB0005C0E9804C4095F0265077101F405F900FF
:103DC000FB04B30048048700C10369005803550091
:103DD00003034500BE023A008402310053022A0068
:103DE0002902250004022000E4011C00C80119007A
:103DF000AF01170098011400840113007101100035
:103E00006101100051010E0043010D0036010B004D
:103E10002B010B0020010B00150109000C0109000A
:103E200003010800FB000800F3000800EB00070096
:103E3000E4000600DE000600D8000600D2000600FE
:103E4000CC000500C7000500C2000500BD0004004D
:103E5000B9000400B5000400B1000400AD00040086
:103E6000A9000400A5000300A20003009F000400B5
:103E70009B000300980003009500020093000300DC
:103E8000900003008D0002008B00030088000200F8
:103E90008600020084000300810002007F0002000F
:103EA0007D0002007B000200790002007700010023
:103EB000760002007400020072000100710002002E
:103EC0006F0002006D0001006C0002006A0001003A
:103ED0006900020067000100660001006500010042
:103EE0006400020062000100610001006000010046
:103EF0005F0002005D0001005C0001005B0001004A
:103F00005A0001005900010058000100570001004B
:103F1000560001005500010054000100530000004C
:103F20005300010052000100510001005000010047
:103F30004F0001004E0000004E0001004D00010046
:103F40004C0001004B0000004B0001004A00010042
:103F5000490001004800000048000100470001003E
:103F60004600000046000100450000004500010039
:103F70004400010043000000430001004200000033
:103F8000420001004100000041000100400001002A
:103F90003F0000003F0001003E0000003E00010025
:103FA0003D0000003D0001003C0000003C0000001E
:103FB0003C0001003B0000003B0001003A00000013
:103FC0003A0001003900000039000100380000000B
:103FD0003800000038000100370000003700010001
:103FE00036000000360000003600010035000000F9
:103FF00035000000350001003400000034000000EE
:1040000034000100330000003300000033000100E1
:1040100032000000320000003200010031000000D8
:1040200031000000310001003000000030000000CD
:10403000300001002F0000002F0000002F000000C2
:104040002F0001002E0000002E0000002E000100B5
:104050002D0000002D0000002D0000002D000100AB
:104060002C0000002C0000002C0000002C0001009F
:104070002B0000002B0000002B0000002B00010093
:104080002A0000002A0000002A0000002A00010087
:10409000290000002900000029000000290000007C
:1040A000290001002800000028000000280000006E
:1040B0002800000028000100270000002700000061
:1040C0002700000027000000270001002600000054
:1040D0002600000026000000260000002600010047
:1040E000250000002500000025000000250000003C
:1040F000250000002500010024000000240000002D
:10410000240000002400000024000100230000001F
:104110002300000023000000230000002300000013
:104120002300000023000100220000002200000004
:1041300022000000220000002200000022000100F6
:1041400021000000210000002100000021000000EB
:1041500021000000210000002100010020000000DB
:1041600020000000200000002000000020000000CF
:104170002000000020000000200001001F000000BF
:104180001F0000001F0000001F0000001F000000B3
:104190001F0000001F0001001E0000001E000000A4
:1041A0001E0000001E0000006563686F3A003A20A0
:1041B0004578747275646572207377697463686595
:1041C00064206F66662E204D494E54454D50207434
:1041D00072696767657265642021003A20457874CA
:1041E0007275646572207377697463686564206FA3
:1041F00066662E204D415854454D502074726967B3
:10420000676572656420210054656D706572617424
:1042100075726520686561746564206265642073E9
:1042200077697463686564206F66662E204D415817
:1042300054454D502074726967676572656420212A
:104240002100202D20496E76616C696420657874A8
:104250007275646572206E756D6265722021005002
:104260004944204175746F74756E652061626F7288
:104270007465642E00504944204175746F74756EE6
:10428000652066696E6973686564212050757420C5
:10429000746865204B702C204B6920616E64204B44
:1042A0006420636F6E7374616E747320696E746FD3
:1042B00020436F6E66696775726174696F6E2E68F0
:1042C00000504944204175746F74756E65206661B5
:1042D000696C6564212074696D656F757400204098
:1042E0003A006F6B20543A006F6B20423A005049FD
:1042F00044204175746F74756E65206661696C65E4
:1043000064212054656D70657261747572652074E6
:104310006F6F206869676800204B643A2000204B6B
:10432000693A2000204B703A200020436C6173737F
:1043300069632050494420002054753A2000204BE6
:10434000753A2000206D61783A2000206D696E3A40
:10435000200020643A200020626961733A200050F6
:104360004944204175746F74756E65207374617271
:104370007400504944204175746F74756E652066F1
:1043800061696C65642E2042616420657874727581
:10439000646572206E756D6265722E004572726F73
:1043A000723A000000000018070100A8071400304E
:1043B000082800B8083C0038095000C009640048CB
:1043C0000A7800C80A8C00480BA000C80BB400484B
:1043D0000CC800C80CDC00400DF000C00D04013812
:1043E0000E1801B00E2C01280F4001A00F54011827
:1043F00010680188107C01001190013013F401480D
:104400001558024017BC0228192003F01A8403A88B
:104410001CE803401E4C0443616E6E6F7420656E91
:10442000746572207375626469723A20004D32348B
:10443000004D3233202573006175746F25692E6736
:10444000006572726F722077726974696E6720748A
:104450006F2066696C650043617264206572726FDB
:10446000723A004E6F74205344207072696E746902
:104470006E67002F005344207072696E74696E6716
:10448000206279746520002E0044656C6574696F44
:104490006E206661696C65642C2046696C653A2003
:1044A0000046696C652064656C657465643A002E2D
:1044B000006F70656E206661696C65642C204669CA
:1044C0006C653A200057726974696E6720746F20BA
:1044D00066696C653A20002E006F70656E2066611B
:1044E000696C65642C2046696C653A20002E006F6B
:1044F00070656E206661696C65642C2046696C6528
:104500003A200046696C652073656C656374656468
:10451000002053697A653A200046696C65206F7007
:10452000656E65643A20002E006F70656E206661CE
:10453000696C65642C2046696C653A200053442000
:1045400063617264206F6B006F70656E526F6F7481
:10455000206661696C656400766F6C756D652E69A7
:104560006E6974206661696C656400534420696EED
:104570006974206661696C002F002F0043616E6EC4
:104580006F74206F70656E20737562646972006568
:1045900063686F3A004572726F723A0048617264E4
:1045A000636F6465642044656661756C742053654F
:1045B0007474696E6773204C6F6164656400563073
:1045C00031300053746F7265642073657474696E62
:1045D00067732072657472696576656400204400B3
:1045E0002049002020204D333031205000504944D4
:1045F0002073657474696E67733A00205A002059FD
:104600000020204D323036205800486F6D65206FF5
:10461000666673657420286D6D293A002045002078
:104620005A0020580020420020540020204D3230F3
:1046300035205300416476616E6365642076617253
:104640006961626C65733A20533D4D696E20666501
:1046500065647261746520286D6D2F73292C205458
:104660003D4D696E2074726176656C206665656487
:104670007261746520286D6D2F73292C20423D6D69
:10468000696E696D756D207365676D656E742074F4
:10469000696D6520286D73292C20583D6D617869FE
:1046A0006D756D205859206A65726B20286D6D2FCD
:1046B00073292C20205A3D6D6178696D756D205AE3
:1046C000206A65726B20286D6D2F73292C20204580
:1046D0003D6D6178696D756D2045206A65726B204E
:1046E000286D6D2F73290020540020204D32303466
:1046F000205300416363656C65726174696F6E3A43
:1047000020533D616363656C65726174696F6E2CE3
:1047100020543D7265747261637420616363656CDB
:1047200065726174696F6E00204500205A0020593F
:104730000020204D3230312058004D6178696D7570
:104740006D20416363656C65726174696F6E2028CA
:104750006D6D2F7332293A00204500205A002059F0
:104760000020204D3230332058004D6178696D753E
:104770006D2066656564726174657320286D6D2FA8
:1047800073293A00204500205A0020590020204D6E
:10479000393220580053746570732070657220752B
:1047A0006E69743A0053657474696E67732053744C
:1047B0006F726564006563686F3A00544553540D29
:1047C0000A000D0A00556E6B6E6F776E20636F6D79
:1047D0006D616E643A20000D0A003F0054696E6BF3
:1047E00065725F31392E30332E31004E414E494EC5
:1047F000495459494E46CDCCCC3D0AD7233C17B736
:10480000D13877CC2B329595E6241FB14F0A0000A2
:1048100020410000C84200401C4620BCBE4CCA1BC0
:104820000E5AAEC59D74CBAA2C01320111241FBEB5
:10483000CFEFD1E2DEBFCDBF00E00CBF13E0A0E0C0
:10484000B2E0E8E2F3EF02E00BBF02C007900D9286
:10485000AE34B107D9F727E1AEE4B3E001C01D9251
:10486000AA3FB207E1F714E2C5E1D4E200E006C0D6
:1048700021970109802FFE010F946E71C331D1077A
:1048800080E00807A9F70F94676C0D9482790C9467
:1048900000001F920F920FB60F9211242F933F9397
:1048A0008F939F93AF93BF9380914F039091500349
:1048B000A0915103B091520330914E0323E0230F96
:1048C0002D3720F40196A11DB11D05C026E8230F48
:1048D0000296A11DB11D20934E0380934F03909328
:1048E0005003A0935103B0935203809153039091CE
:1048F0005403A0915503B09156030196A11DB11D1B
:104900008093530390935403A0935503B09356039D
:10491000BF91AF919F918F913F912F910F900FBEBB
:104920000F901F9018952FB7F89460914F037091D6
:10493000500380915103909152032FBF08953FB7C8
:10494000F8948091530390915403A0915503B09132
:10495000560326B5A89B05C02F3F19F00196A11D4F
:10496000B11D3FBFBA2FA92F982F8827820F911D05
:10497000A11DB11DBC01CD0142E0660F771F881F4C
:10498000991F4A95D1F708958F929F92AF92BF9247
:10499000CF92DF92EF92FF926B017C01D0DF4B014F
:1049A0005C01C114D104E104F104F1F093D0C7DF3C
:1049B000DC01CB0188199909AA09BB09883E9340FB
:1049C000A105B10570F321E0C21AD108E108F10890
:1049D00088EE880E83E0981EA11CB11CC114D1047E
:1049E000E104F10421F7DDCFFF90EF90DF90CF904D
:1049F000BF90AF909F908F9008958230910538F0CE
:104A0000880F991F880F991F05970197F1F708954F
:104A1000789484B5826084BD84B5816084BD85B599
:104A2000826085BD85B5816085BDEEE6F0E0808160
:104A300081608083E1E8F0E0108280818260808381
:104A4000808181608083E0E8F0E080818160808304
:104A5000E1EBF0E0808184608083E0EBF0E0808136
:104A600081608083E1E9F0E08081826080838081E1
:104A700081608083E0E9F0E0808181608083E1EA09
:104A8000F0E0808182608083808181608083E0EAC1
:104A9000F0E0808181608083E1E2F1E080818260EA
:104AA0008083808181608083E0E2F1E080818160A9
:104AB0008083EAE7F0E08081846080838081826087
:104AC0008083808181608083808180688083109270
:104AD000C100089508951F93CF93DF93182FEB0122
:104AE00061E016D1209711F460E004C0CF3FD105FA
:104AF00031F461E0812FDF91CF911F9145C1E12F0A
:104B0000F0E0E450FD4FE4914E2F50E0FA01319770
:104B1000E231F10508F09DC08827EE58FF4F8F4F16
:104B20000D946E7184B5806884BDC7BD97C084B58F
:104B3000806284BDC8BD92C08091800080688093EF
:104B40008000D0938900C093880088C08091800045
:104B5000806280938000D0938B00C0938A007EC0D7
:104B600080918000886080938000D0938D00C093F6
:104B70008C0074C08091B00080688093B000C093B6
:104B8000B3006CC08091B00080628093B000C0938D
:104B9000B40064C080919000806880939000D093AE
:104BA0009900C09398005AC08091900080628093D1
:104BB0009000D0939B00C0939A0050C080919000C9
:104BC000886080939000D0939D00C0939C0046C065
:104BD0008091A00080688093A0008091A0008F7BCE
:104BE0008093A000D093A900C093A80037C0809103
:104BF000A00080628093A000D093AB00C093AA0075
:104C00002DC08091A00088608093A000D093AD005B
:104C1000C093AC0023C08091200180688093200164
:104C2000D0932901C093280119C08091200180628E
:104C300080932001D0932B01C0932A010FC0809153
:104C40002001886080932001D0932D01C0932C0116
:104C500005C0C038D1050CF04CCF46CFDF91CF91C5
:104C60001F91089590E0FC013197E231F10508F0C1
:104C70004EC08827EC57FF4F8F4F0D946E71809177
:104C800080008F7703C0809180008F7D80938000AB
:104C9000089580918000877FF9CF84B58F7702C017
:104CA00084B58F7D84BD08958091B0008F7703C057
:104CB0008091B0008F7D8093B00008958091900026
:104CC0008F7707C0809190008F7D03C08091900006
:104CD000877F8093900008958091A0008F7707C010
:104CE0008091A0008F7D03C08091A000877F80937A
:104CF000A0000895809120018F7707C08091200146
:104D00008F7D03C080912001877F809320010895CB
:104D1000CF93DF9390E0FC01EE5BFC4F2491FC010C
:104D2000E857FC4F8491882361F190E0880F991F28
:104D3000FC01E851FC4FC591D491FC01E253FC4FBA
:104D4000A591B491611109C09FB7F894888120950D
:104D500082238883EC912E230BC0623061F49FB7CD
:104D6000F8943881822F809583238883EC912E2BB1
:104D70002C939FBF06C08FB7F894E8812E2B288311
:104D80008FBFDF91CF9108951F93CF93DF93282F8B
:104D900030E0F901E450FD4F8491F901EE5BFC4FE6
:104DA000D491F901E857FC4FC491CC23C1F0162FE0
:104DB000811158DFEC2FF0E0EE0FFF1FE253FC4FA4
:104DC000A591B4918FB7F894111105C09C91ED2F66
:104DD000E095E92302C0EC91ED2BEC938FBFDF91BE
:104DE000CF911F91089508951F920F920FB60F92C1
:104DF00011240BB60F922F933F934F935F936F93B2
:104E00007F938F939F93AF93BF93EF93FF93E09123
:104E10000E02F0910F021995FF91EF91BF91AF91A2
:104E20009F918F917F916F915F914F913F912F91C2
:104E30000F900BBE0F900FBE0F901F9018951F92F2
:104E40000F920FB60F9211240BB60F922F933F9330
:104E50004F935F936F937F938F939F93AF93BF9382
:104E6000EF93FF93E0911002F09111021995FF91D9
:104E7000EF91BF91AF919F918F917F916F915F91D2
:104E80004F913F912F910F900BBE0F900FBE0F903F
:104E90001F9018951F920F920FB60F9211240BB608
:104EA0000F922F933F934F935F936F937F938F93C3
:104EB0009F93AF93BF93EF93FF93E0911202F09112
:104EC00013021995FF91EF91BF91AF919F918F912F
:104ED0007F916F915F914F913F912F910F900BBEFA
:104EE0000F900FBE0F901F9018951F920F920FB644
:104EF0000F9211240BB60F922F933F934F935F9312
:104F00006F937F938F939F93AF93BF93EF93FF9391
:104F1000E0911402F09115021995FF91EF91BF9164
:104F2000AF919F918F917F916F915F914F913F9141
:104F30002F910F900BBE0F900FBE0F901F901895E2
:104F40001F920F920FB60F9211240BB60F922F9350
:104F50003F934F935F936F937F938F939F93AF9301
:104F6000BF93EF93FF93E0910A02F0910B02199522
:104F7000FF91EF91BF91AF919F918F917F916F9131
:104F80005F914F913F912F910F900BBE0F900FBEED
:104F90000F901F9018951F920F920FB60F92112429
:104FA0000BB60F922F933F934F935F936F937F9323
:104FB0008F939F93AF93BF93EF93FF93E0910C0276
:104FC000F0910D021995FF91EF91BF91AF919F91D3
:104FD0008F917F916F915F914F913F912F910F90A2
:104FE0000BBE0F900FBE0F901F9018951F920F923F
:104FF0000FB60F9211240BB60F922F933F934F933E
:105000005F936F937F938F939F93AF93BF93EF9330
:10501000FF93E0911602F09117021995FF91EF911D
:10502000BF91AF919F918F917F916F915F914F91C0
:105030003F912F910F900BBE0F900FBE0F901F90BE
:1050400018951F920F920FB60F9211240BB60F9264
:105050002F933F934F935F936F937F938F939F9380
:10506000AF93BF93EF93FF93E0911802F091190271
:105070001995FF91EF91BF91AF919F918F917F9182
:105080006F915F914F913F912F910F900BBE0F90B9
:105090000FBE0F901F901895CF92DF92EF92FF9264
:1050A0000F931F93CF93DF93CDB7DEB72A970FB639
:1050B000F894DEBF0FBECDBF88E89FEF90938C03BE
:1050C00080938B030E945633811102C0109291038A
:1050D0004091910388E0840F405E682F0E945B330B
:1050E0000E9473320E948A3943E656E066E180E00E
:1050F0000E94CF3A68ED74E086E30E946C3780919D
:10510000910381508335C8F00E94793280917003F9
:10511000811149C02091910330E0220F331F40914B
:105120002202429FC001439F900D112464E670E06B
:105130000F941D7188E0CFDC36C007E116E1E12C49
:10514000F12CDE2C40919103842F90E0880F991F61
:1051500097012D5E3F4F2817390744F4440F4451FF
:105160004E19202F612F80E00E9495398091910384
:10517000282F30E0220F331F2E153F0534F0880F03
:10518000202F4FE7612F8D1904C0202F4FE7612F8B
:1051900080E00E9495392FEFE21AF20A1E5F0E5F3F
:1051A0001A3279F6B1CF80919003811105C08091B8
:1051B0008A03882309F455C08091700381110CC0C3
:1051C000809122022FEF829FC001112464E670E0DB
:1051D0000F941D7188E07FDC109290031092910370
:1051E00080914B0981FF04C040E060E080E003C093
:1051F00046E368E288E20E945B330E94733280E0FB
:1052000094E00F945179853599F460E088ED98E049
:105210002A960FB6F894DEBF0FBECDBFDF91CF91B7
:105220001F910F91FF90EF90DF90CF900C94D2A13F
:10523000C0908A031A8219821C821B8285E09BE43B
:10524000282F9E838D8388E8482FE12CFA8000E088
:105250001C813E815FEF60E070E088ED98E00E9485
:10526000F1A02A960FB6F894DEBF0FBECDBFDF9136
:10527000CF911F910F91FF90EF90DF90CF90089505
:10528000CF92EF92FF920F931F93CF93DF93CDB7FF
:10529000DEB72A970FB6F894DEBF0FBECDBF0E94CF
:1052A00099E90E94663C0E94CE77811106C00E9457
:1052B000596C60E080E00E94BB750E94B27233DBE3
:1052C000DC01CB0182519D4FAF4FBF4F80935703FD
:1052D00090935803A0935903B0935A0310929003EC
:1052E0001092910310925B031A8219821C821B8216
:1052F00087E49DE9282F9E838D8384E0482FC12C6D
:10530000E12CFA8000E01C813E8150E060E070E01A
:1053100088ED98E00E945DA11A8219821C821B828E
:105320008CE498E2282F9E838D8388E8482FFA80AA
:105330001C813E815FEF60E070E088ED98E00E94A4
:105340007FA160E070E088E02A960FB6F894DEBF97
:105350000FBECDBFDF91CF911F910F91FF90EF90C6
:10536000CF90B9CBCF92DF92EF92FF920F931F9322
:10537000CF93DF93CDB7DEB768970FB6F894DEBF53
:105380000FBECDBFD0DA0091570310915803209182
:10539000590330915A03061717072807390718F5DC
:1053A000D901C8014996A11DB11D8093570390935F
:1053B0005803A0935903B0935A039091900380919E
:1053C0009103992341F082508093910381110BC086
:1053D0001092900308C08E5F809391038E3718F06F
:1053E00081E0809390030E945633882309F442C1E0
:1053F0000E943F3C92B392FB992790F981E0982755
:1054000080917C0D85FB222720F9291781F02091BE
:10541000F40E222321F021502093F40E0BC0992387
:1054200011F0806201C08F7D80937C0D03C088E203
:105430008093F40E0F94161C882309F47BC08E0110
:105440000F5F1F4F88E1F80111928A95E9F769EC27
:1054500074E0C8010F94A2750E948A3969EB74E068
:105460008AE00E946C370F941D1C90E0FC0131977C
:10547000EA30F10508F046C08827EA56FF4F8F4F03
:105480000D946E716DEA74E084E10E946C3768EAF5
:1054900074E03AC068E974E084E10E946C3763E923
:1054A00074E032C066E874E084E10E946C3761E821
:1054B00074E02AC062E774E084E10E946C376DE614
:1054C00074E022C06DE574E084E10E946C3768E509
:1054D00074E01AC069E474E084E10E946C3764E40B
:1054E00074E012C06FE274E084E10E946C376AE2FB
:1054F00074E00AC066E174E084E10E946C3761E107
:1055000074E002C069E074E0C8010F94837562E042
:1055100074E088E20E946C37B80182E30E944E3545
:105520008091910360E8681B482F0E945B33DBD7B2
:10553000E0D73DC080917C0D83FD35C080914B0943
:10554000982F907284FF24C091112DC01A82198265
:105550001C821B8285EE95EE282F9E838D838CE026
:10556000482F8F83188619861A86C12CE12CFA8061
:1055700000E01C813E8150E060E070E088ED98E042
:105580000E947FA180914B09806280934B090BC0E0
:10559000992349F08F7D80934B0965EE75EE88ED78
:1055A00098E00E946EA288ED98E00E9429A0E09108
:1055B0008603F0918703309729F08091F30C8F3F99
:1055C00009F0199520ED3CEC4CE45DE36091EB179C
:1055D0007091EC178091ED179091EE170F94247055
:1055E0006B017C0123E333E343E75FE360911E0239
:1055F00070911F0280912002909121020F942470DB
:105600009B01AC01C701B6010F94766C60931E023A
:1056100070931F02809320029093210220ED3CECB6
:105620004CE45DE36091E3177091E4178091E51716
:105630009091E6170F9424706B017C0123E333E310
:1056400043E75FE360911A0270911B0280911C0294
:1056500090911D020F9424709B01AC01C701B6010B
:105660000F94766C60931A0270931B0280931C0255
:1056700090931D0268960FB6F894DEBF0FBECDBFA3
:10568000DF91CF911F910F91FF90EF90DF90CF901E
:105690000895CF93DF931F921F92CDB7DEB780E0BE
:1056A0000F94085A1A821982CE0101960F94115A4A
:1056B00010920F0D0F900F90DF91CF9108950C94E1
:1056C000083C009739F044E150E0BC018BE593E0E1
:1056D0000D94537610925B03089510925B03089526
:1056E0008BE593E00895AC01809176039091770368
:1056F0004817590720F410927703109276032091EF
:10570000750391E0920F909375039831CCF088E186
:105710008093750320917603309177032E5F3F4F7E
:105720004217530728F030937703209376030895A8
:10573000509377034093760388EE80937503089522
:1057400091110DC08091760390917703009739F005
:1057500002979093770380937603209375030895BF
:10576000EF92FF920F931F93CF93DF937C018B01F6
:10577000EA0120918B0330918C0328388FEF380792
:10578000A9F037FF06C0285E3F4F30938C0320936B
:105790008B0320918B0330918C032831310534F039
:1057A0002851310930938C0320938B030E948A394E
:1057B0004EE265E080E40E947F3842E36CE783E0DC
:1057C0000E945C3880918B0390918C0307960F9711
:1057D00090F42BE24BE367E085E00E94D9382AE29F
:1057E0004AE368E086E00E94343AA70166E181E27C
:1057F0000E94F73705C0A70166E181E20E94923757
:1058000080918B0390918C030897089790F42BE27A
:105810004BE767E085E40E94D9382AE24AE768E06E
:1058200086E40E94343AA80166E181E60E94F737D7
:1058300005C0A80166E181E60E949237209739F100
:1058400080918B0390918C0340970897B0F42DE3DF
:105850004AE765E385E00E94D9382CE349E766E32F
:1058600086E00E94343ABE0186E3DF91CF911F911A
:105870000F91FF90EF900C947F37BE0186E3DF918C
:10588000CF911F910F91FF90EF900C946C37DF91A7
:10589000CF911F910F91FF90EF9008950E948A3948
:1058A00043E36CE783E00C945C38AF92BF92CF92F5
:1058B000EF92FF920F931F93CF93DF93CDB7DEB795
:1058C0002A970FB6F894DEBF0FBECDBF8C015A01E8
:1058D00020918B0330918C0328388FEF3807A9F083
:1058E00037FF06C0205F3F4F30938C0320938B031C
:1058F00020918B0330918C032031310534F02051FD
:10590000310930938C0320938B0380918A03882381
:1059100049F180918B0390918C0307960F9710F5B6
:105920006115710511F0FB01199501151105D1F0F3
:105930001A8219821C821B82202F1E830D8388E805
:10594000482F8F838FEF8887CC24C394E12CFA8073
:1059500000E01C813E815FEF60E070E088ED98E040
:105960000E94F1A09BDFA114B10421F483E0A82ED2
:1059700088E0B82E80918B0390918C0307960F9747
:1059800040F52DE34AE765E385E00E94D9382CE332
:1059900049E766E386E00E94343AC5010F94A97591
:1059A000982F990F890FA50166E391E4981B892F21
:1059B0002A960FB6F894DEBF0FBECDBFDF91CF9110
:1059C0001F910F91FF90EF90CF90BF90AF900C94EC
:1059D0006D36C5010F94A975982F990F890FA501F0
:1059E00066E391E4981B892F2A960FB6F894DEBFE0
:1059F0000FBECDBFDF91CF911F910F91FF90EF9020
:105A0000CF90BF90AF900C947C356F927F928F9225
:105A10009F92AF92BF92CF92DF92EF92FF920F933D
:105A20001F93CF93DF93CDB7DEB72A970FB6F894C5
:105A3000DEBF0FBECDBF6C014A0139015701A091F5
:105A40008B03B0918C03A8388FEFB80799F0B7FF9C
:105A500005C05096B0938C03A0938B0380918B0369
:105A600090918C03803191052CF0409790938C039A
:105A700080938B0380918A03882309F43FC080912F
:105A80008B0390918C039C01295F3F4F2F30310590
:105A900080F46115710511F0FB011995C114D10451
:105AA00069F11A8219821C821B822C2DDE82CD8222
:105AB00012C00897089710F50115110511F0F801AB
:105AC000199561147104D1F01A8219821C821B820B
:105AD000262D7E826D8288E8482F8F838FEF8887FE
:105AE000CC24C394E12CFA8000E01C813E815FEF5E
:105AF00060E070E088ED98E00E947FA1CFDE8091A9
:105B00008B0390918C0307960F97D0F42DE34EE30F
:105B100065E385E00E94D9382CE34DE366E386E037
:105B20000E94343AC4010F94A975982F990F890FD8
:105B3000A40166E393E2981B892F0E946D360CC086
:105B4000C4010F94A975982F990F890FA40166E3DA
:105B500093E2981B892FD0D780918B0390918C036F
:105B60000897089768F52DE34AE765E382E40E9409
:105B7000D9382CE349E766E383E40E94343AC5014F
:105B80000F94A975982F990F890FA50166E39FE5DA
:105B9000981B892F2A960FB6F894DEBF0FBECDBF93
:105BA000DF91CF911F910F91FF90EF90DF90CF90F9
:105BB000BF90AF909F908F907F906F900C946D36B8
:105BC000C5010F94A975982F880F980FA50166E35A
:105BD0008FE5891B2A960FB6F894DEBF0FBECDBFA6
:105BE000DF91CF911F910F91FF90EF90DF90CF90B9
:105BF000BF90AF909F908F907F906F907DC7EF92F6
:105C0000FF921F93CF93DF93C82F2FE24CE767E2F9
:105C100083E00E94D938D0E0219714E08CE0E82E90
:105C2000F12CCF3F8FEFD807C1F01D37B1F0CE0177
:105C3000B7010F941D71AC01453051051CF4475D4F
:105C400069E205C08A3030F464E2640F4DE2812FCE
:105C50000E947F381F5F2197E4CFDF91CF911F9182
:105C6000FF90EF900895CF92DF92EF92FF920F9303
:105C70001F93CF93DF93CDB7DEB760970FB6F8943D
:105C8000DEBF0FBECDBF0E94932460939507709333
:105C9000960780939707909398070091110D10E055
:105CA000F801EE0FFF1FEE0FFF1FE551F84E608168
:105CB0007181828193810F94BE6D6B017C01000F15
:105CC000111FF801EF50F84E6081718180E090E083
:105CD0000F94EF6D20E030E040E251E40F94756CDA
:105CE0000F94BE6D8B01D7FE02C0C12CD12C0C15B8
:105CF0001D052CF460E088ED98E00E94D2A12DE70C
:105D00002C9DC0012D9D900D1124B8010F941D7183
:105D1000F09085036F1518F060938503F62E0E94AE
:105D20008A396AEE77E08AE00E946C378E010F5F55
:105D30001F4F80E1F80111928A95E9F7E091110D6A
:105D400084E0E89FF0011124E25EFD4F60817181E3
:105D5000828193810F94BE6DDC01CB0147EE57E049
:105D6000B8010E942A3DE091110DF0E0EE0FFF1FF7
:105D7000EF50F84E45EE57E0BC01808191810E94C2
:105D80002A3DB80188E18AD68F2D39DFB2D36096DB
:105D90000FB6F894DEBF0FBECDBFDF91CF911F913C
:105DA0000F91FF90EF90DF90CF900895FF920F93A7
:105DB0001F93CF93DF93082FEB01FB01019000208D
:105DC000E9F73197E61BF70B9091330242FF49C088
:105DD00091FF28C0E53130F1FF27749786E0282F26
:105DE0002E9FC0012F9F900D11247DDCE091760342
:105DF000F0917703CF01059626E030E0B9010F94CA
:105E00000971C60FD71FCF01B9010F940971892BF2
:105E100011F013E101C014E1FE01E10FF11DF0806A
:105E2000108202C010E0F12C27E0200F6FEF600F0E
:105E30004CE783E00E94343A809176039091770397
:105E4000059666E070E00F940971AE01602F99E04D
:105E5000981B892F27D5FF2091F0C10FD11DF88203
:105E60000EC091FF05C0E53118F01C891C8A01C0E5
:105E700010E0AE01602F84E025D411111C8BDF915E
:105E8000CF911F910F91FF9008956F927F928F9203
:105E90009F92AF92BF92CF92DF92EF92FF920F93B9
:105EA0001F93CF93DF9370918A037111C6C0E09165
:105EB0008B03F0918C03E838FF4F21F410928C0390
:105EC00010928B03A0918B03B0918C03862E062E2B
:105ED000000C9908B7FF0BC0F401EE0FFF1FEE0F87
:105EE000FF1FEA0FFB1FF0938C03E0938B03E091FD
:105EF0008B03F0918C03D401AA0FBB1FAA0FBB1F09
:105F0000EA17FB074CF074E06702E019F10911246D
:105F1000F0938C03E0938B0300918B0310918C031F
:105F200017FF02C00D5F1F4F79015A016C011595D3
:105F3000079515950795702E0E948A39A0917103D7
:105F4000B0917203C801992763E0880F991F6A9581
:105F5000E1F70F978A1B9B0BEC0197FD2396D595D4
:105F6000C795D595C795AC0FBD1F1816190614F423
:105F7000119608C0892B29F4B0937203A093710382
:105F80000BC01197B0937203A09371031092750325
:105F900010927703109276038091710390917203AF
:105FA000282F277033E0969587953A95E1F79BE384
:105FB000692E621ADBE0D21BC82F8C2F90E0881567
:105FC00099054CF4C71511F040E001C044E06D2F75
:105FD0008C2FF5011995CF5FD85FD611EECF28E051
:105FE0004CE760E083E00E94343A2FE34CE761E342
:105FF00083E00E94953929E04CE769E083E00E9444
:10600000953942E36CE783E00E945C38B60181E099
:1060100076D7E114F10489F0802FF701DF91CF9159
:106020001F910F91FF90EF90DF90CF90BF90AF90B6
:106030009F908F907F906F901994DF91CF911F91D7
:106040000F91FF90EF90DF90CF90BF90AF909F9017
:106050008F907F906F900895CF92DF92EF92FF9292
:106060000F93CF93DF93CDB7DEB764970FB6F89455
:10607000DEBF0FBECDBF80917C0390917D03209148
:106080008B0330918C032817390724F490938C03E9
:1060900080938B0380917A0390917B0320918B03F3
:1060A00030918C038217930724F490938C03809390
:1060B0008B0380917E03813041F4E0917F03F09166
:1060C000800380918B0380838EC0823059F4E091ED
:1060D0007F03F091800380918B0390918C039183D7
:1060E000808381C08330A9F4E0907F03F090800327
:1060F00060918B0370918C03072E000C880B990B19
:106100000F94F16D20E030E048EC52E40F94566DAE
:1061100065C0843089F4E0917F03F0918003809121
:106120008B0390918C03092E000CAA0BBB0B808370
:106130009183A283B38357C08530A1F4E0917F039C
:10614000F091800320918B0330918C034FEF429F9D
:10615000C001439F900D112464E670E00F941D71FF
:10616000608341C0863099F4E0907F03F090800313
:1061700060918B0370918C03072E000C880B990B98
:106180000F94F16D20E030E040E752E414C0873016
:10619000A9F4E0907F03F090800360918B037091ED
:1061A0008C03072E000C880B990B0F94F16D20E0E7
:1061B00030E048EC52E40F94247010C0883099F419
:1061C000E0907F03F090800360918B0370918C03CB
:1061D000072E000C880B990B0F94F16DF70160836B
:1061E0007183828393835ADB60918303709184036C
:1061F00084E172D6CE0101967C0184E1F70111920F
:106200008A95E9F720917E0380918B0390918C030E
:10621000C0908103D0908203233091F4BC01990F88
:10622000880B990B0F94F16D20E030E048EC52E4BC
:106230000F94566D00E09601A7010E945D3E04C0D8
:10624000A601B7010E942A3DB7018EE127D46CEF69
:1062500077E0C7010F94A27520917E03C09081035F
:10626000D090820380917803909179032330A1F438
:10627000BC01990F880B990B0F94F16D20E030E071
:1062800048EC52E40F94566D00E09601AE01495F70
:106290005F4F0E945D3E06C0A601BE01695F7F4F51
:1062A0000E942A3DB70186E3F9D380918A038823AF
:1062B00029F061E088ED98E00E94D2A11AD164969D
:1062C0000FB6F894DEBF0FBECDBFDF91CF910F9117
:1062D000FF90EF90DF90CF900895CF92DF92EF92F2
:1062E000FF9280912302882391F10E94ECF58111A5
:1062F0002EC080914B0984FD2AC02091230230E0FA
:10630000A0E6BAEE0F947671C0909507D0909607EC
:10631000E0909707F0909807C60ED71EE81EF91E6A
:106320000E949324C616D706E806F90680F48091E9
:10633000F1179091F2178338910538F09093740318
:106340008093730380E00F94085A80E001C081E0DD
:10635000FF90EF90DF90CF900895CF92EF92FF9251
:106360000F931F93CF93DF93CDB7DEB72A970FB666
:10637000F894DEBF0FBECDBFE091110DF0E0EE0F3F
:10638000FF1FEF50F84E80819181892B11F560E05D
:1063900083E793E00F94F259109285031A821982D1
:1063A0001C821B8283E39EE2282F9E838D8388E8D4
:1063B000482FCC24C394E12CFA8000E01C813E815C
:1063C0005FEF60E070E088ED98E00E947FA180E0E0
:1063D00001C081E02A960FB6F894DEBF0FBECDBF94
:1063E000DF91CF911F910F91FF90EF90CF90089583
:1063F0009091BC0097FFFCCF8093BB0084E8809312
:10640000BC0008958091BC0087FFFCCF84E9809395
:10641000BC0008951F93CF93DF931F92CDB7DEB7D3
:10642000182F84EA8093BC0080EC6983E1DF812F20
:10643000DFDF6981862FDCDF0F90DF91CF911F9125
:10644000E1CFCF93C82F84EA8093BC0088E7D0DFE8
:1064500080E0CEDF81E8CCDF8C2FCADFCF91D2CFB6
:106460001F920F920FB60F9211240BB60F922F931B
:106470003F934F935F936F937F938F939F93AF93CC
:10648000BF93EF93FF9380918E0390918F038115BB
:1064900024E0920711F4B6DF13C0FC01EB56FC4F69
:1064A0008081A6DF8091BC0081608093BC008091D8
:1064B0008E0390918F03019690938F0380938E03A8
:1064C000FF91EF91BF91AF919F918F917F916F91CC
:1064D0005F914F913F912F910F900BBE0F900FBE88
:1064E0000F901F90189580914B09806880934B09FD
:1064F0000895CF92DF92EF92FF922091250930917B
:1065000026092115310509F490C0A0E6BAEE0F94D2
:106510007671C0909507D0909607E0909707F0901D
:106520009807C60ED71EE81EF91E0E9493242091DC
:106530004B09C616D706E806F90608F04BC022FD3F
:1065400027C094E0822F892780934B0990912409DA
:10655000992339F080913202981708F4892F71DF5E
:106560000AC084EA8093BC0088E742DF80E040DF15
:106570008EEA3EDF47DF80912309811109C060E088
:1065800082E048DF60E083E045DF60E084E042DFF6
:1065900090912309992309F448C080914B0981FD0A
:1065A00044C080919103899FC0011124892F990FC4
:1065B000990B809394039C013327220F331F213AB8
:1065C000310514F020EA30E0209393038093920386
:1065D0008ADF2BC022FF29C094E0822F8927809375
:1065E0004B0981FF07C010929403109293031092FD
:1065F000920308C088E2809394038093930386E318
:106600008093920370DF80912409882321F0809188
:10661000320217DF0AC084EA8093BC0088E7E8DE14
:1066200080E0E6DE8FEAE4DEEDDE80914B0987FF55
:106630000FC08F7780934B096091940382E0EADE6C
:106640006091930383E0E6DE6091920384E0E2DEF2
:1066500080914B0982FF04C080912409882309F1AD
:1066600084EA8093BC0088E7C3DE80E0C1DE80E07E
:10667000BFDE80E1BDDE80EBBBDE8091BC0087FF2A
:10668000FCCF84EA8093BC0088E7B2DE80E4B0DE11
:1066900010928F0310928E038091BC0081608093D2
:1066A000BC00FF90EF90DF90CF9008958091BC00E8
:1066B0008095817008958093940360939303409331
:1066C00092030895DF92EF92FF920F931F93CF935F
:1066D000DF93962F969596959695A82FB0E080E833
:1066E000989FA00DB11D11249D012B563C4FAB5E10
:1066F000BB4F677078E0761BE901249615E0FA013C
:10670000E080EE2009F4C6C0C901855993408B3F53
:1067100093400CF0BFC0CD01855993408B3F93400F
:106720000CF0B8C0F12CEDE1EE1AF1081E9DC0018D
:106730001F9D900D11248F5D974FFC01F490062E44
:1067400001C0FF0C0A94EAF7F901E080FE28F0820C
:106750007E01F3E0EF1AF108FC013196E4910E2F6F
:10676000062E01C0000F0A94EAF7F701D0800D2928
:1067700000837E01F2E0EF1AF108FC013296E49109
:106780000E2F062E01C0000F0A94EAF7F701D08001
:106790000D290083FC013396E4910E2F062E01C0D3
:1067A000000F0A94EAF7FE01D2900D290083FC0144
:1067B0003496E491062E01C0EE0F0A94EAF7888120
:1067C000E82BE8832A5F3F4F662309F45FC0FA0194
:1067D000E080F12CFDE1EF1AF1081E9DC0011F9D24
:1067E000900D11248F5D974FFC010491E02FF0E094
:1067F000072E02C0F595E7950A94E2F7FC91EF2B7E
:10680000EC93FC013196E491F0E0072E02C0F5957F
:10681000E7950A94E2F71196FC911197EF2B1196E8
:10682000EC931197FC013296E491F0E0072E02C040
:10683000F595E7950A94E2F71296FC911297EF2BE3
:106840001296EC931297FC013396E491F0E0072E38
:1068500002C0F595E7950A94E2F71396FC91139719
:10686000EF2B1396EC931397FC013496E491F0E030
:10687000072E02C0F595E7950A94E2F714968C91DD
:106880001497E82B1496EC93149716964F5F5F4F6E
:10689000269635CFDF91CF911F910F91FF90EF900A
:1068A000DF900895DF92EF92FF920F931F93CF93A3
:1068B000DF93962F969596959695A82FB0E080E851
:1068C000989FA00DB11D11249D012B563C4FAB5E2E
:1068D000BB4F677078E0761BE901249615E0FA015A
:1068E000E080EE2009F4D2C0C901855993408B3F66
:1068F00093400CF0CBC0CD01855993408B3F934022
:106900000CF0C4C0F12CEDE1EE1AF1081E9DC0019F
:106910001F9D900D11248F5D974FFC01F490EF2D7A
:10692000062E01C0EE0F0A94EAF7FE2EF094F9014C
:10693000E080FE20F0827E01F3E0EF1AF108FC0116
:106940003196E491062E01C0EE0F0A94EAF70E2F5D
:106950000095F701D0800D2100837E01F2E0EF1A4F
:10696000F108FC013296E491062E01C0EE0F0A9464
:10697000EAF70E2F0095F701D0800D210083FC016E
:106980003396E491062E01C0EE0F0A94EAF70E2F1B
:106990000095FE01D2900D210083FC013496E49114
:1069A000062E01C0EE0F0A94EAF7E0958881E823ED
:1069B000E8832A5F3F4F662309F464C0FA01E08050
:1069C000F12CFDE1EF1AF1081E9DC0011F9D900DF5
:1069D00011248F5D974FFC010491E02FF0E0072E0A
:1069E00002C0F595E7950A94E2F7E095FC91EF2354
:1069F000EC93FC013196E491F0E0072E02C0F5958E
:106A0000E7950A94E2F7E0951196FC911197EF2330
:106A10001196EC931197FC013296E491F0E0072E69
:106A200002C0F595E7950A94E2F7E0951296FC917D
:106A30001297EF231296EC931297FC013396E49190
:106A4000F0E0072E02C0F595E7950A94E2F7E0958D
:106A50001396FC911397EF231396EC931397FC0175
:106A60003496E491F0E0072E02C0F595E7950A947C
:106A7000E2F7E09514968C911497E8231496EC9322
:106A8000149716964F5F5F4F269629CFDF91CF91CF
:106A90001F910F91FF90EF90DF900895E82FAB01C9
:106AA000DB010D900020E9F711979D01261B370BA4
:106AB0002431310538F4822F880F280F90E4892F74
:106AC000821B01C084E06E2FFDCDE82FAB01DB01FE
:106AD0000D900020E9F711979D01261B370B2431FB
:106AE000310538F4822F880F280F90E4892F821BFC
:106AF00001C084E06E2FD6CE7F928F929F92AF928C
:106B0000BF92CF92DF92EF92FF920F931F93CF939A
:106B1000DF935A01962F969596959695A82FB0E0FB
:106B200020E8929FA00DB11D1124AD014B565C4F82
:106B3000AB5EBB4F677078E0761BF50124916A016C
:106B4000F4E0CF0ED11C85E0982E222309F4B7C0C3
:106B5000CA01855993408B3F93400CF0B0C0CD01E2
:106B6000855993408B3F93400CF0A9C030E02D51E4
:106B70003109929EC001939E900D11248F5D974F15
:106B8000FC012491062E01C0220F0A94EAF7FA01B3
:106B90003081232B2083E60123977C01FFEFEF1A3E
:106BA000FF0AF7012491062E01C0220F0A94EAF78A
:106BB0003881232B288321968C010E5F1F4FF8010B
:106BC0002491062E01C0220F0A94EAF73881232B64
:106BD0002883EC012396FE018490062E01C0880CC8
:106BE0000A94EAF7F6017290872880829C012C5F54
:106BF0003F4FF9018490062E01C0880C0A94EAF7F1
:106C0000F6017080872880824A5F5F4F662309F40F
:106C10004DC0FC01849190E0072E02C095958795A8
:106C20000A94E2F79C91892B8C93F701E490F12C64
:106C3000072E02C0F594E7940A94E2F711968C911E
:106C40001197E82A1196EC921197F801049110E03F
:106C5000072E02C0159507950A94E2F712968C91BB
:106C60001297082B12960C931297FE01C491D0E054
:106C7000072E02C0D595C7950A94E2F713968C911A
:106C80001397C82B1396CC931397F901249130E0F6
:106C9000072E02C0359527950A94E2F714968C9139
:106CA0001497282B14962C9314971696FFEFAF1A6F
:106CB000BF0AF5012491F6E0CF0ED11C46CFDF913B
:106CC000CF911F910F91FF90EF90DF90CF90BF90E9
:106CD000AF909F908F907F9008957F928F929F9218
:106CE000AF92BF92CF92DF92EF92FF920F931F93DA
:106CF000CF93DF935A01962F969596959695A82F48
:106D0000B0E020E8929FA00DB11D1124AD014B56BB
:106D10005C4FAB5EBB4F677078E0761BF50124914A
:106D20006A01F4E0CF0ED11C85E0982E222309F4ED
:106D3000C5C0CA01855993408B3F93400CF0BEC03B
:106D4000CD01855993408B3F93400CF0B7C030E0A4
:106D50002D513109929EC001939E900D11248F5D9B
:106D6000974FFC012491062E01C0220F0A94EAF7E6
:106D70002095FA01308123232083E60123977C01AB
:106D8000FFEFEF1AFF0AF7012491062E01C0220F30
:106D90000A94EAF7209538812323288321968C01D1
:106DA0000E5F1F4FF8012491062E01C0220F0A9496
:106DB000EAF72095388123232883EC012396FE01EE
:106DC0008490E82D062E01C0EE0F0A94EAF78E2E6D
:106DD0008094F6017290872080829C012C5F3F4F47
:106DE000F9018490E82D062E01C0EE0F0A94EAF70F
:106DF0008E2E8094F6017080872080824A5F5F4FDC
:106E0000662309F452C0FC01849190E0072E02C071
:106E1000959587950A94E2F780959C9189238C93A8
:106E2000F701E490F12C072E02C0F594E7940A9440
:106E3000E2F7E09411968C911197E8221196EC926A
:106E40001197F801049110E0072E02C015950795DF
:106E50000A94E2F7009512968C91129708231296E5
:106E60000C931297FE01C491D0E0072E02C0D59575
:106E7000C7950A94E2F7C09513968C911397C8238F
:106E80001396CC931397F901249130E0072E02C09A
:106E9000359527950A94E2F7209514968C911497CE
:106EA000282314962C9314971696FFEFAF1ABF0A57
:106EB000F5012491F6E0CF0ED11C38CFDF91CF91B0
:106EC0001F910F91FF90EF90DF90CF90BF90AF9008
:106ED0009F908F907F9008951F93CF93DF93182FEB
:106EE000EB01CB010F94A975982F880F980FAE0175
:106EF000612F80E4891BDF91CF911F91FDCD1F93FE
:106F0000CF93DF93182FEB01CB010F94A975982F26
:106F1000880F980FAE01612F80E4891BDF91CF911C
:106F20001F91DBCEAF92BF92CF92DF92EF92FF9292
:106F30000F931F93CF93DF93CDB7DEB72A970FB68A
:106F4000F894DEBF0FBECDBFE82EF62E6A016CE7C7
:106F500070E0CA010F948E758C01009761F15C019D
:106F6000AC18BD08A501B601CE0101966C010F94C5
:106F7000D875F601EA0DFB1D1082F6010190002084
:106F8000E9F73197EC19FD096BEF6F0D8E2F880F24
:106F9000E80FA6018E2D8E1B95DB0F5F1F4FC801DA
:106FA0000F94A97565E06F0D982F990F890FA801AF
:106FB000E81A8E2D0AC0C6010F94A975982F880F64
:106FC000980FA6016F2D8E2D891B96DD2A960FB680
:106FD000F894DEBF0FBECDBFDF91CF911F910F910F
:106FE000FF90EF90DF90CF90BF90AF900895AF9259
:106FF000BF92CF92DF92EF92FF920F931F93CF93A6
:10700000DF93CDB7DEB72A970FB6F894DEBF0FBE79
:10701000CDBFE82EF62E6A016CE770E0CA010F942E
:107020008E758C01009761F15C01AC18BD08A5015B
:10703000B601CE0101966C010F94D875F601EA0DE8
:10704000FB1D1082F60101900020E9F73197EC1941
:10705000FD096BEF6F0D8E2F880FE80FA6018E2DA7
:107060008E1B20DC0F5F1F4FC8010F94A97565E0D0
:107070006F0D982F990F890FA801E81A8E2D0AC05D
:10708000C6010F94A975982F880F980FA6016F2D30
:107090008E2D891B22DE2A960FB6F894DEBF0FBE16
:1070A000CDBFDF91CF911F910F91FF90EF90DF90B7
:1070B000CF90BF90AF900895242F269526952695C2
:1070C000477091E001C0990F4A95EAF7E82FF0E088
:1070D00030E8239FE00DF11D1124EB56FC4F8E1B71
:1070E000282F2E0F621750F09F012559334021158C
:1070F000344024F42081292B2193F2CF089590E08D
:10710000262F269526952695FC0150E8259FE00D13
:10711000F11D11249F01EB56FC4F211534400CF05A
:1071200047C0242F26952695269530E8239F800D6D
:10713000911D1124DC01AB56BC4F81159440C4F560
:1071400067707081EA17FB07A1F450E040955095F5
:10715000477055278FEF90E09C0102C03595279529
:107160004A95E2F701C0880F6A95EAF78223872BD8
:107170001EC02FEF30E001C0220F6A95EAF7272BDF
:1071800020838FEFE058FF4FEA17FB0711F0808351
:10719000F9CF50E040955095477055278FEF90E01C
:1071A00002C0959587954A95E2F79081892B808357
:1071B0000895DF92EF92FF920F931F93CF93DF9387
:1071C0001F92CDB7DEB7E82E162FD42EFF24FA94E7
:1071D000F20E01E0060F4F2D602F298390DF4F2D17
:1071E000602F8D2D8CDF0FEF0D0DFF24F394FE0C1F
:1071F000412F602F8F2D60DF2981422F602F8F2D2F
:107200000F90DF91CF911F910F91FF90EF90DF9042
:1072100053CF0F931F93CF93DF93A82FB0E0962FF8
:10722000969596959695FD0100E8909FE00DF11DCD
:107230001124EB56FC4F922F96959695969510E853
:10724000919FA00DB11D1124AB56BC4FEA17FB074F
:1072500009F45BC06770CFEFD0E08E0102C0000F71
:10726000111F6A95E2F7B801EF01982F491788F0CE
:107270008E0105591340011514405CF4588190FDAE
:1072800002C035E501C03AEA3623352B39939F5FBA
:10729000EDCFBF0160587F4F6A177B07A1F0FB015C
:1072A000982F4917B8F3EF01C559D340C115D44001
:1072B0008CF7308190FD02C055E501C05AEA352BAC
:1072C00031939F5FEECF30E02095309527703327C4
:1072D000EFEFF0E0DF0102C0B595A7952A95E2F740
:1072E0009D01FB01481788F0BF0165597340611586
:1072F00074405CF4508180FD02C095E501C09AEABB
:107300009223952B91938F5FEDCFDF91CF911F91BA
:107310000F91089580E094E0E5E9F3E0DF019C013E
:107320001D9221503040E1F708950F931F93CF93A2
:10733000DF93C82FD0E0962F969596959695FE01EF
:1073400010E8919FE00DF11D1124EB56FC4F922F98
:1073500096959695969530E8939FC00DD11D112472
:10736000CB56DC4F962F9770EC17FD0731F530E0C8
:107370002095309527703327AFEFB0E0BD0102C0F4
:10738000759567952A95E2F701C0AA0F9A95EAF7D5
:10739000A623CE2FDF2F8E1BA0959C2F980F491769
:1073A00008F45DC09E0125593340211534400CF08E
:1073B00056C098819A239993F0CF6FEF70E001C087
:1073C000660F9A95EAF7DF01382F3E1B6095932FE1
:1073D0009A0F491750F08D010559134001151440BB
:1073E00024F49C9196239D93F2CFE058FF4F90E0B8
:1073F000582F5E1BEC17FD0799F0DF01352F390F71
:10740000632F6A0F461740F0BD016559734061153F
:10741000744014F41D92F4CFE058FF4F9058EACF17
:1074200030E020953095277033276FEF70E0DB0157
:1074300002C0B595A7952A95E2F79D01DF018E1B45
:107440002095982F9A0F491750F0BD016559734048
:107450006115744024F49C9192239D93F2CFDF91A7
:10746000CF911F910F9108950F931F93CF93DF93A7
:10747000C82FD0E0962F969596959695FE0130E808
:10748000939FE00DF11D1124EB56FC4F922F969522
:107490009695969550E8959FC00DD11D1124CB5619
:1074A000DC4F6770EC17FD0729F530E0209530952B
:1074B00027703327AFEFB0E0ED0102C0D595C79537
:1074C0002A95E2F701C0AA0F6A95EAF79C2F9A2342
:1074D000DF018E1B282F2A0F421708F45BC09D0185
:1074E00025593340211534400CF054C02C91292BE0
:1074F0002D93F0CF9FEF01C0990F6A95EAF7DF0156
:10750000582F5E1B352F3A0F431750F0BD016559B8
:1075100073406115744024F43C91392B3D93F2CFB4
:10752000E058FF4F90E0582F5E1B6FEFEC17FD0700
:1075300099F0DF01352F390F732F7A0F471740F07D
:107540008D01055913400115144014F46D93F4CFC7
:10755000E058FF4F9058EACF30E0209530952770E3
:1075600033276FEF70E0DB0102C0B595A7952A9530
:10757000E2F79D01DF018E1B982F9A0F491750F0FB
:10758000BD01655973406115744024F49C91922BA0
:107590009D93F2CFDF91CF911F910F910895BF92EC
:1075A000CF92DF92EF92FF920F931F93CF93DF93CF
:1075B000FA019491DA0112963196449150E0495FB4
:1075C0005F4F23E0559547952A95E1F7562F577061
:1075D00078E0751B669566956695082F10E0442344
:1075E00009F442C0683008F03FC09801F0E86F9F8E
:1075F000200D311D1124E901CB5EDB4FF901EB5663
:10760000FC4F7F01FD01B92EBA0EDF01BE1649F114
:10761000970125593340211534401CF59E01255909
:10762000334021153440ECF4249130E06901052EFB
:1076300001C0CC0C0A94EAF7D7018C91C82ACD92EC
:107640007D01552361F0673051F0072E02C035955A
:1076500027950A94E2F73881232B288321963196C7
:10766000D4CF6F5F4150BBCFDF91CF911F910F916E
:10767000FF90EF90DF90CF90BF900895DF92EF9250
:10768000FF920F931F93CF93DF93FA01D4909A0147
:107690002E5F3F4F3196449150E0495F5F4F93E03A
:1076A000559547959A95E1F7562F577098E0F92E22
:1076B000F51A66956695669590E0442309F440C0F6
:1076C000683008F03DC0DC01F0E86F9FA00DB11DEF
:1076D0001124ED01CB5EDB4FAB56BC4FF901ED2C15
:1076E000E20E9F01EE1649F18D0105591340011577
:1076F00014401CF58E010559134001151440ECF49B
:10770000249130E08901052E01C0000F0A94EAF7A8
:1077100000951C9101230D93552369F0673059F0B2
:107720000F2C02C0359527950A94E2F720953881F1
:107730002323288321963196D4CF6F5F4150BDCF4C
:10774000DF91CF911F910F91FF90EF90DF900895FF
:1077500084E15B9AE7EBF5E03197F1F700C00000B8
:107760005B98E7EBF5E03197F1F700C0000081503E
:1077700081F78AE05B9AE7E5F2E03197F1F700C024
:1077800000005B98E7E5F2E03197F1F700C00000F8
:10779000815081F708958091330286FD26C085FFD0
:1077A00023C08FE05B9AEFEEF0E03197F1F700C075
:1077B00000005B98EFEEF0E03197F1F700C00000B9
:1077C000815081F78AE05B9AE7ECF0E03197F1F7BE
:1077D00000C000005B98E7ECF0E03197F1F700C0E3
:1077E0000000815081F70895B3CF08958AE05B9A35
:1077F000E7ECF0E03197F1F700C000005B98E7ECB0
:10780000F0E03197F1F700C00000815081F7089552
:1078100082B381FB992790F981E08927909B826050
:1078200090918803891751F1813059F028F0823006
:1078300091F0833059F020C0923079F09130E1F42A
:1078400014C0992351F09330B9F40FC0913029F04E
:10785000923091F40AC0933031F490918D039F37A8
:1078600059F09F5F07C0911107C090918D03923826
:107870001CF0915090938D0380938803089580911C
:107880008D030E94A5EC89B191E082FB882780F9E5
:10789000892721F020918903922701C090E09093DD
:1078A0008A0380938903811104C080918D0388230A
:1078B00051F00E94932460939507709396078093EC
:1078C00097079093980710928D0308956B9A519A99
:1078D000509AA4E0B1E08C9182608C939FB7F894A9
:1078E000E5E0F1E080818D7F80839FBF8C91816096
:1078F0008C939FB7F89480818E7F80839FBFE1E057
:10790000F1E08081886080839FB7F894E2E0F1E045
:107910008081877F80839FBF539A999898985298C7
:10792000A19AA09A5A9A9A98A29A599A589A739890
:107930008FE99FE00197F1F700C00000739A8FE98B
:107940009FE00197F1F700C000008CE08093B80041
:107950001092B90060E880E00E940A326CE181E098
:107960000E940A326091940382E00E940A32609180
:10797000930383E00E940A326091920384E00E94A4
:107980000A3260E085E00E940A326FEF86E00E94D2
:107990000A3260E087E00E940A326AEA88E00E94C8
:1079A0000A3284EA8093BC0088E70E94F83180E0C4
:1079B0000E94F8318DEF0E94F83182E10E94F83187
:1079C0008EEA0E94F83185ED0E94F83180EA0E942B
:1079D000F83188EA0E94F8318FE30E94F83183ED94
:1079E0000E94F83180E00E94F83180E40E94F83172
:1079F00081EA0E94F83188EC0E94F8318AED0E94F9
:107A0000F83182E10E94F83181E80E94F8318091DA
:107A100032020E94F83189ED0E94F83182E80E941A
:107A2000F8318BED0E94F83184E30E94F83180E256
:107A30000E94F83184EA0E94F8318FEA0E94F831FE
:107A40000E940232E5DE1BDF10928C0310928B0342
:107A50000C9479320F931F93CF93DF939C01FB011A
:107A60008A0197FF06C08DE2808331952195310907
:107A70003196203187E2380774F0C90160E177E27E
:107A80000F941D71CB016AE070E00F941D71805D51
:107A90008083319604C0283E83E0380774F0C90122
:107AA00068EE73E00F941D71CB016AE070E00F94F3
:107AB0001D71805D8083319603C02436310574F0DA
:107AC000C90164E670E00F941D71CB016AE070E0BB
:107AD0000F941D71805D8083319603C02A3031057B
:107AE0006CF0CAE0D0E0C901BE010F941D71CB015A
:107AF000BE010F941D71805D80833196EF01219648
:107B0000C9016AE070E00F941D71805D808311826D
:107B10000115110549F0B801CE010F94A275C801F5
:107B20000F94A975C80FD91FCE01DF91CF911F9176
:107B30000F9108958F929F92AF92BF92CF92DF9252
:107B4000EF92FF920F931F93CF93DF936B017C0112
:107B5000EA018A010F5F1F4F80E8C8168EEED80633
:107B600086E3E806F10490F4C701B60120E13EE0A7
:107B700040E050E00F943071F901211531054105C5
:107B80005105E1F12436310560F002C0E7EEF3E083
:107B9000CF0164E670E00F940971605D6883E801CD
:107BA00003C02A30310568F02AE030E0CF01B90186
:107BB0000F940971CB01B9010F940971805D88831D
:107BC00021969E012F5F3F4FCF016AE070E00F9436
:107BD000097190E3980F9883319741F06AE178E05A
:107BE000C9010F94A275CE0107965AC064E178E0EE
:107BF000C9010F94A275CE01069652C08CE3882E5F
:107C0000912CA12CB12CC701B601A50194010F94B0
:107C100030716B017C01CA01B901A50194010F9477
:107C200030716115710581059105E1F0262F6A30EB
:107C300071058105910550F03AE0862F632F0F946E
:107C4000FD700F94FD70905D9883E801822F6AE0CB
:107C50000F94FD7020E3290FFE012193CF016FE007
:107C600078E01AC02C2DFAE0CF16D104E104F1041B
:107C700040F08C2D6AE00F94FD7090E3980F98838C
:107C8000E801822F6AE00F94FD7020E3290FFE01C6
:107C90002193CF016AE078E00F94A275CE0105969A
:107CA000DF91CF911F910F91FF90EF90DF90CF90D8
:107CB000BF90AF909F908F9008954F925F926F9278
:107CC0007F92AF92BF92CF92DF92EF92FF920F938B
:107CD0001F93CF93DF93EA01590120E030E048EC95
:107CE00052E40F94247020E030E040E05FE30F9412
:107CF000766C0F94BE6D6B017C01002379F0161633
:107D00001706180619061CF48BE2888313C0672B2C
:107D1000682B692B19F480E288835DC0F7FE0BC0E5
:107D20008DE28883F094E094D094C094C11CD11C5F
:107D3000E11CF11C219680EAC81686E8D80681E08D
:107D4000E806F104A4F0C701B60120EA36E841E0F4
:107D500050E00F945271CA01B9012AE030E040E0CE
:107D600050E00F945271605D6883219607C0E0E196
:107D7000CE16E7E2DE06E104F104A4F0C701B60185
:107D800020E137E240E050E00F945271CA01B9019E
:107D90002AE030E040E050E00F945271605D68836B
:107DA000219607C0F8EECF16F3E0DF06E104F104F8
:107DB0009CF0C701B60128EE33E040E050E00F949C
:107DC0005271CA01B9012AE030E040E050E00F945E
:107DD0005271605D68832196C701B60124E630E0E8
:107DE00040E050E00F9452718AE0482E512C612CF3
:107DF000712CCA01B901A30192010F945271605D07
:107E000068838EE28983C701B601A30192010F94B2
:107E10005271162FCA01B901A30192010F94527138
:107E2000605D6A837E0184E0E80EF11C105D1B83B7
:107E3000A114B10449F0B501C7010F94A275C501A1
:107E40000F94A975E80EF91EF7011082C701DF91A2
:107E5000CF911F910F91FF90EF90DF90CF90BF9047
:107E6000AF907F906F905F904F9008950F931F9306
:107E7000CF93DF938C0141505109EB010990002011
:107E8000E9F72197C61BD70B4C175D0708F4EA01E9
:107E9000AE01C8010F940E76F801EC0FFD1F1082A1
:107EA000CE01DF91CF911F910F91089561E088ED90
:107EB00098E00C94D2A161E088ED98E00C941BA2AC
:107EC00060E088ED98E00C94D2A14CE45CE066E3BD
:107ED00085E00C947C3584E090E090938C03809353
:107EE0008B034BE351E16FE670E48BE99FE30E9463
:107EF000552C80E094E00F945179853531F046E3BC
:107F000051E160E084E60E947C3562E271E18AE042
:107F10000E946C376DE071E184E10E946C376CEF78
:107F200070E18EE10E946C3768EE70E188E20E9499
:107F30006C370C94793284E090E090938C038093BA
:107F40008B0344ED50E160EE71E487EF93E40E940F
:107F5000552C80E094E00F945179853531F04FEC49
:107F600050E160E084E60E947C356AEB70E18AE0D3
:107F70000E946C3767EA70E184E10E946C3763E924
:107F800070E18EE10E946C376DE770E188E20E943B
:107F90006C370C94793284E090E090938C0380935A
:107FA0008B0340EF5EE068E371E483E994E40E94B0
:107FB000552C80E094E00F945179853531F04BEEEB
:107FC0005EE060E084E60E947C3565ED7EE08AE05C
:107FD0000E946C3762EC7EE084E10E946C376FEAAD
:107FE0007EE08EE10E946C3769E97EE088E20E94C3
:107FF0006C370C94793284E090E090938C038093FA
:108000008B0340EA5DE063E176E48DEF99E40E9442
:10801000552C4AE95DE060E08EE50E947C3566E81B
:108020007DE08AE00E946C3767E77DE084E10E9492
:108030006C3766E67DE08EE10E946C3762E57DE09C
:1080400088E20E946C370C94793284E090E090933F
:108050008C0380938B0343EA5CE060E070E083E88C
:1080600097E40E94552C4DE95CE060E08EE50E94AB
:108070007C3569E87CE08AE00E946C3769E77CE047
:1080800084E10E946C376DE67CE08EE10E946C37E3
:1080900060E67CE088E20E946C370C94793284E0E0
:1080A00090E090938C0380938B0345E55BE060E068
:1080B00070E08DE899E40E94552C4FE45BE060E0AD
:1080C0008EE50E947C356FE37BE084E10E946C3793
:1080D0006EE27BE08EE10E946C370C9479320F9354
:1080E0001F93CF93DF93CDB7DEB7A0970FB6F89469
:1080F000DEBF0FBECDBF0E94A3578E010F5F1F4F83
:1081000080E2F80111928A95E9F71F9283E28F933A
:1081100060915A0270915B0280915C0290915D02C5
:108120000F94BE6D7F936F938DED90E19F938F932E
:108130001F930F930F947576C8010F94C51B0FB64C
:10814000F894DEBF0FBECDBFA0960FB6F894DEBF89
:108150000FBECDBFDF91CF911F910F9108950F9367
:108160001F93CF93DF93CDB7DEB7A0970FB6F894E8
:10817000DEBF0FBECDBF8E010F5F1F4F80E2F80143
:1081800011928A95E9F76091620270916302809181
:108190006402909165020F94BE6D7F936F9386E7A2
:1081A0009FE09F938F931F930F930F947576C80151
:1081B0000F94C51B6091160D7091170D8091180DCD
:1081C0009091190D0F94BE6D77FF02C060E070E0D2
:1081D000615F7F4F7F936F9360914A0270914B0272
:1081E00080914C0290914D020F94BE6D6A507109BE
:1081F0007F936F9360915A0270915B0280915C0251
:1082000090915D020F94BE6D7F936F9387E69FE020
:108210009F938F931F930F930F947576C8010F94BC
:10822000C51B60916202709163028091640290911B
:1082300065020F94BE6D7F936F938DE59FE09F93D2
:108240008F931F930F930F947576C8010F94C51BDE
:108250000FB6F894DEBF0FBECDBFA0960FB6F89450
:10826000DEBF0FBECDBFDF91CF911F910F9108955B
:10827000EF92FF920F931F93CF93DF93CDB7DEB7AB
:10828000A0970FB6F894DEBF0FBECDBF8E010F5F73
:108290001F4F80E2F80111928A95E9F7609162021E
:1082A0007091630280916402909165020F94BE6D9B
:1082B0007F936F938FE89EE09F938F931F930F930D
:1082C0000F947576C8010F94C51B6091120D7091C3
:1082D000130D8091140D9091150D0F94BE6D7B01BF
:1082E0000F900F900F900F900F900F9077FF02C09C
:1082F000E12CF12C60914E0270914F02809150025E
:10830000909151020F94BE6D6A5071097F936F93E3
:1083100060914A0270914B0280914C0290914D0203
:108320000F94BE6D6E197F0977FF02C06F5F7F4F9C
:10833000CB0195958795B701680F791F7F936F9350
:1083400060915A0270915B0280915C0290915D0293
:108350000F94BE6D7F936F9380E89EE09F938F9301
:108360001F930F930F947576C8010F94C51B6091EE
:1083700062027091630280916402909165020F9491
:10838000BE6D7F936F9386E79EE09F938F931F93BD
:108390000F930F947576C8010F94C51B0FB6F89410
:1083A000DEBF0FBECDBFA0960FB6F894DEBF0FBEE6
:1083B000CDBFDF91CF911F910F91FF90EF90089566
:1083C000EF92FF920F931F93CF93DF93CDB7DEB75A
:1083D000A0970FB6F894DEBF0FBECDBF0E946C4BC6
:1083E0008E010F5F1F4F80E2F80111928A95E9F725
:1083F0006091120D7091130D8091140D9091150DD7
:108400000F94BE6D7B0177FF02C0E12CF12C6091CF
:108410004E0270914F0280915002909151020F9440
:10842000BE6D6A5071097F936F9360914A0270919B
:108430004B0280914C0290914D020F94BE6D6E19CB
:108440007F0977FF02C06F5F7F4FCB0195958795BE
:10845000B701680F791F7F936F931F9283E28F9309
:1084600060915A0270915B0280915C0290915D0272
:108470000F94BE6D7F936F938AE690E19F938F93E5
:108480001F930F930F947576C8010F94C51B0FB6F9
:10849000F894DEBF0FBECDBFA0960FB6F894DEBF36
:1084A0000FBECDBFDF91CF911F910F91FF90EF9045
:1084B00008954091910388E0840F405E682F0E94E8
:1084C0005B330E94733284E090E090938C0380933E
:1084D0008B034AED5FE06FEA70E483E992E40E9467
:1084E000552C80E094E00F945179853531F045EDBD
:1084F0005FE060E084E60E947C3560EC7FE08AE02B
:108500000E946C376AEA7FE084E10E946C3765E97B
:108510007FE08EE10E946C3760E87FE088E20E9495
:108520006C370C9479324091910388E0840F405E5F
:10853000682F0E945B330E94733284E090E0909336
:108540008C0380938B0344E55FE060E070E08BEC8C
:108550009FE30E94552C80E094E00F94517985357B
:1085600031F04FE45FE060E084E60E947C3569E32F
:108570007FE08AE00E946C3763E27FE084E10E9442
:108580006C376EE07FE08EE10E946C3769EF7EE031
:1085900088E20E946C370C9479324091910388E014
:1085A000840F405E682F0E945B330E94733284E028
:1085B00090E090938C0380938B0349E05EE06FEA38
:1085C00070E48DEF92E40E94552C80E094E00F94CB
:1085D0005179853531F044E05EE060E084E60E9448
:1085E0007C3564EF7DE084E10E946C3761EE7DE0D4
:1085F0008EE10E946C370C9479324091910388E0AF
:10860000840F405E682F0E945B330E94733284E0C7
:1086100090E090938C0380938B0380E094E00F9420
:108620005179853539F44CED5DE067EC76E480E016
:1086300090E006C043ED5DE060E176E48BEF9FE300
:108640000E94552C80E094E00F945179853531F0EB
:108650004DEC5DE060E08EE50E947C356DEB7DE0E9
:1086600084E10E946C3769EA7DE08EE10E946C37FC
:108670000C947932CF92EF92FF920F931F93409117
:10868000910388E0840F405E682F0E945B330E9454
:1086900073320F94C141823028F520E030E040E091
:1086A0005FE36091360D7091370D8091380D909198
:1086B000390D0F94766C6093360D7093370D80935F
:1086C000380D9093390DC12CE12CF12C00E010E411
:1086D00026E33DE042E35DE06EE27DE08AE29DE07C
:1086E0000F946F3649E05CE061E478E483E099E45C
:1086F0000E94552C43E05CE060E08EE50E947C35F2
:108700006FEE7BE08AE00E946C376EED7BE084E1E7
:108710000E946C376DEC7BE08EE10E946C376CEB55
:108720007BE088E20E946C371F910F91FF90EF90E1
:10873000CF900C947932CF92EF92FF920F931F93C8
:108740004091910388E0840F405E682F0E945B3364
:108750000E94733249E95BE069E47BE28FE490E4D4
:108760000E94552C43E95BE060E08EE50E947C3579
:1087700062E87BE08AE00E946C3763E77BE084E19B
:108780000E946C3764E67BE08EE10E946C370F94A8
:10879000C141823028F520E030E040E05FE36091A5
:1087A000360D7091370D8091380D9091390D0F94E1
:1087B000766C6093360D7093370D8093380D9093DF
:1087C000390DC12CE12CF12C00E81FE326E33DE03C
:1087D00042E35DE06EE27DE08AE29DE00F946F3659
:1087E0001F910F91FF90EF90CF900C947932CF9220
:1087F000EF92FF920F931F934091910388E0840FB3
:10880000405E682F0E945B330E94733280918B031D
:1088100090918C0388389F4F21F410928C03109212
:108820008B038091F30C81110AC080918B0390918E
:108830008C03892B21F00F94C141843088F0109271
:108840008C0310928B039091DE118091DD119813AF
:108850003BC048E550E16FE275E489E592E43AC037
:1088600060918B0370918C03072E000C880B990B81
:108870000F94F16D2DEC3CEC4CE45DE30F9424700F
:108880009B01AC016091320D7091330D8091340DDC
:108890009091350D0F94756C6093320D7093330D7C
:1088A0008093340D9093350DC12CE12CF12C00E711
:1088B00012E426E33DE042E35DE06EE27DE08AE221
:1088C0009DE00F946F36BBCF41E650E160E070E071
:1088D00080E090E00E94552C80E094E00F94517964
:1088E000853531F043E550E160E084E60E947C3557
:1088F00061E470E18AE00E946C376DE270E184E12E
:108900000E946C376BE170E18EE10E946C3766E08B
:1089100070E188E20E946C371F910F91FF90EF90F9
:10892000CF900C947932CF92EF92FF920F931F93D6
:108930004091910388E0840F405E682F0E945B3372
:108940000E94733280918B0390918C0388389F4FE3
:1089500021F410928C0310928B038091F30C8111FF
:108960000AC080918B0390918C03892B21F00F9486
:10897000C141843068F09091DE118091DD1198132F
:108980003FC044E65EE06FE275E48DEC92E43EC0E9
:1089900060918B0370918C03072E000C880B990B50
:1089A0000F94F16D2DEC3CEC4CE45DE30F942470DE
:1089B0009B01AC016091320D7091330D8091340DAB
:1089C0009091350D0F94756C6093320D7093330D4B
:1089D0008093340D9093350D10928C0310928B037D
:1089E000C12CE12CF12C00E712E426E33DE042E348
:1089F0005DE06EE27DE08AE29DE00F946F36BBCFD2
:108A00004DE65EE060E070E080E090E00E94552C72
:108A100080E094E00F945179853531F04FE55EE0C8
:108A200060E084E60E947C3569E47EE08AE00E9492
:108A30006C3763E37EE084E10E946C3762E27EE0A3
:108A40008EE10E946C3762E17EE088E20E946C3722
:108A50001F910F91FF90EF90CF900C947932EF928D
:108A60000F931F93CF93DF93CDB7DEB7A0970FB6C9
:108A7000F894DEBF0FBECDBF2091320D3091330D83
:108A80004091340D5091350D6091260D7091270D58
:108A90008091280D9091290D0F94756C6093260D8F
:108AA0007093270D8093280D9093290D1092320D0D
:108AB0001092330D1092340D1092350DEE24E39484
:108AC0000091110D26E33DE042E35DE06EE27DE0C2
:108AD0008AE29DE00F94CE408E010F5F1F4F80E22F
:108AE000F80111928A95E9F7609162027091630230
:108AF00080916402909165020F94BE6D7F936F9395
:108B00008CEF9FE09F938F931F930F930F94757635
:108B1000C8010F94C51B6091160D7091170D8091BF
:108B2000180D9091190D0F94BE6D77FF02C060E093
:108B300070E0615F7F4F7F936F936091120D709132
:108B4000130D8091140D9091150D0F94BE6D77FF4C
:108B500002C060E070E0665F7F4F7F936F9360912B
:108B60005A0270915B0280915C0290915D020F94B9
:108B7000BE6D7F936F938DEE9FE09F938F931F93B6
:108B80000F930F947576C8010F94C51B6091620214
:108B90007091630280916402909165020F94BE6DA2
:108BA0007F936F9383EE9FE09F938F931F930F9319
:108BB0000F947576C8010F94C51B0FB6F894DEBFED
:108BC0000FBECDBFA0960FB6F894DEBF0FBECDBFCF
:108BD000DF91CF911F910F91EF9008952DEC3CEC18
:108BE0004CEC5DE36091260D7091270D8091280D6E
:108BF0009091290D0F94766C6093260D7093270D3C
:108C00008093280D9093290D0F94266480E094E0C2
:108C10000F945179853511F40C94A7570C94A357F0
:108C2000DDDF0C94596CEF92FF920F931F93CF935B
:108C3000DF93CDB7DEB7A0970FB6F894DEBF0FBEB7
:108C4000CDBF0E94596C8E010F5F1F4F80E2F8016B
:108C500011928A95E9F76091120D7091130D809130
:108C6000140D9091150D0F94BE6D7B0177FF02C01E
:108C7000E12CF12C6091160D7091170D8091180D5B
:108C80009091190D0F94BE6D77FF02C060E070E007
:108C90006B5F7F4F7F936F9360914A0270914B029D
:108CA00080914C0290914D020F94BE6D6E197F0918
:108CB00077FF02C06F5F7F4F759567956E0D7F1DC3
:108CC0007F936F9360915A0270915B0280915C0276
:108CD00090915D020F94BE6D7F936F9383E49DE04E
:108CE0009F938F931F930F930F947576C8010F94E2
:108CF000C51B8FE39DE00F94D81B0FB6F894DEBF21
:108D00000FBECDBFA0960FB6F894DEBF0FBECDBF8D
:108D1000DF91CF911F910F91FF90EF900895EF9207
:108D2000FF920F931F934091910388E0840F405E60
:108D3000682F0E945B330E94733285EDE82E8CE031
:108D4000F82E00E61FE32FE73AE441ED5CE0B801BE
:108D500085E290E40E94052D4BEC5CE060E08EE53E
:108D60000E947C356BEB7CE084E10E946C3769EEFD
:108D700077E08EE10E944E356CEA7CE088E20E944A
:108D80006C371F910F91FF90EF900C94793226DF92
:108D900061E088ED98E00C94D2A1EF92FF920F93DE
:108DA0001F93CF93DF93CDB7DEB7A0970FB6F8949C
:108DB000DEBF0FBECDBF1092260D1092270D109270
:108DC000280D1092290D83E29AE00F94D81B8E0192
:108DD0000F5F1F4F80E2F80111928A95E9F76091C9
:108DE000120D7091130D8091140D9091150D0F942B
:108DF000BE6D7B0177FF02C0E12CF12C60914E0229
:108E000070914F0280915002909151020F94BE6D6B
:108E10006A5071097F936F9360914A0270914B027F
:108E200080914C0290914D020F94BE6D6E197F0996
:108E300077FF02C06F5F7F4FCB0195958795B70194
:108E4000680F791F7F936F931F9283E28F936091D6
:108E50005A0270915B0280915C0290915D020F94C6
:108E6000BE6D7F936F9380E19AE09F938F931F93E2
:108E70000F930F947576C8010F94C51B60E088EDC1
:108E800098E00E94D2A10FB6F894DEBF0FBECDBF0E
:108E9000A0960FB6F894DEBF0FBECDBFDF91CF9185
:108EA0001F910F91FF90EF9008950F931F93CF9311
:108EB000DF93CDB7DEB72A970FB6F894DEBF0FBEAB
:108EC000CDBF162F042F28E1829FC0011124BC01C1
:108ED0006F5F774F48E050E0CE0101960F944179E3
:108EE0001986402FBE016F5F7F4F812F0E94D62EC3
:108EF0002A960FB6F894DEBF0FBECDBFDF91CF919B
:108F00001F910F9108954F925F926F927F92AF924F
:108F1000BF92CF92DF92EF92FF920F931F93CF9366
:108F2000DF93CDB7DEB72A970FB6F894DEBF0FBE3A
:108F3000CDBF80919A0790919B079A83898360E0C7
:108F4000CE0101960F94F25920E030E040EA51E45E
:108F50006091EB177091EC178091ED179091EE17DF
:108F60000F94756C0F94BE6D6B017C016091F117CD
:108F70007091F21780E090E00F94EF6D20E030E008
:108F800040E251E40F94756C20E030E040EA51E497
:108F90000F94756C0F94BE6D2B013C015B01D7FEE5
:108FA00002C0C12CD12CAC14BD0454F580E090E07B
:108FB000A0E8BFE380930F1790931017A0931117A9
:108FC000B09312171A8219821C821B828AE393E4DF
:108FD000282F9E838D8384E0482F8F8318861986DF
:108FE0001A86CC24C394E12CFA8000E01C813E81D7
:108FF00050E060E070E088ED98E00E94F1A062012E
:109000002DE72C9DC0012D9D900D1124B5010F94CD
:109010001D71F09085036F1518F060938503F62E8F
:109020000E944E2C46E45CE060E08EE50E947C35B8
:1090300069E37CE08AE00E946C3763E27CE084E1D3
:109040000E946C3762E17CE08EE10E946C378F2DCC
:109050000E94FF2D0E9479322A960FB6F894DEBF47
:109060000FBECDBFDF91CF911F910F91FF90EF9079
:10907000DF90CF90BF90AF907F906F905F904F90B8
:1090800008952F923F924F925F926F927F928F92AC
:109090009F92AF92BF92CF92DF92EF92FF920F9387
:1090A0001F93CF93DF9300D01F92CDB7DEB783E23B
:1090B000282E87E1382ED1011C964D905D906D9041
:1090C0007C901F978090F3169090F416A090F51660
:1090D000B090F6168091E7169091E816A091E916E7
:1090E000B091EA1689839A83AB83BC83C0901F1723
:1090F000D0902017E0902117F0902217A701960139
:1091000060E078E08FEC96E40F94566DD1011C96E8
:109110006D937D938D939C931F97A701960160E0BB
:1091200070E081EE95E40F94566D6093F3167093A2
:10913000F4168093F5169093F61680E090E0A0E880
:10914000BFE38093E7169093E816A093E916B093D7
:10915000EA160F94084A0AE21DE0F8011486158603
:109160001686178641E06091110D86E39DE00F940D
:109170008D4180E090ECA3E2B4E4F8018487958708
:10918000A687B787D1011C96ED90FD900D911C919B
:109190001F97C12C26E33DE042E35DE06EE27DE0F7
:1091A000CF010F946F36F101448655866686778627
:1091B0008092F3169092F416A092F516B092F616DD
:1091C00089819A81AB81BC818093E7169093E816E0
:1091D000A093E916B093EA160F900F900F900F909E
:1091E000DF91CF911F910F91FF90EF90DF90CF9083
:1091F000BF90AF909F908F907F906F905F904F90B7
:109200003F902F9008958F929F92AF92BF92CF92EE
:10921000DF92EF92FF920F931F93CF93DF93CDB71F
:10922000DEB72A970FB6F894DEBF0FBECDBF0E94FF
:109230004E2C46EB5BE060E08EE50E947C3562EAF6
:109240007BE084E10E946C379091DE118091DD110A
:109250009817C1F183E00F94F4494B015C0120E0C1
:1092600030EC43E254E460911F1770912017809115
:109270002117909122170F9424700F94F46F6B01B3
:109280007C01ADE7B0E0A50194010F948B71A701BB
:1092900096010F945271822F0E94FF2D2A960FB6CD
:1092A000F894DEBF0FBECDBFDF91CF911F910F911C
:1092B000FF90EF90DF90CF90BF90AF909F908F90F6
:1092C0000C9479320E94CB3B809177029091780286
:1092D000880F991F63E070E00F941D7182E00F9476
:1092E000F04A1A8219821C821B828BE993E4282F90
:1092F0009E838D8384E0482F8F831886CC24C3946B
:10930000E12CFA8000E01C813E8150E060E070E0DA
:1093100088ED98E00E94F1A09DCF80917C0D85FDA5
:1093200023C040E050E06BE57FE380E090E00E94E6
:10933000552C48E25BE060E08EE50E947C3562E1FE
:109340007BE084E10E946C3763E07BE08EE10E9469
:109350006C3760EF7AE088E20E946C370E947932C5
:109360008AE39DE00D94485D80FF04C08091F60E75
:109370008823C9F040E050E06BE57FE380E090E0B7
:109380000E94552C4AEE5AE060E08EE50E947C3542
:109390006AED7AE08EE10E946C370E9479328AE3AE
:1093A0009DE00D94575C84E090E090938C03809353
:1093B0008B034EEC5AE060E070E084E399E80E9491
:1093C000552C48EC5AE060E08EE50E947C3564EB59
:1093D0007AE08AE00E946C3765EA7AE084E10E94D4
:1093E0006C3760E97AE08EE10E946C3763E87AE0DE
:1093F00088E20E946C370C947932CF92EF92FF9200
:109400000F931F93CF93DF93CDB7DEB72A970FB695
:10941000F894DEBF0FBECDBF80E098E00F94517985
:109420008130B1F5609177027091780282E00F94FB
:10943000F04A60E080E00E94BB7565E580E094E062
:109440000F946C791A8219821C821B8283E897E43C
:10945000282F9E838D8388E8482FC12CE12CFA8029
:1094600000E01C813E815FEF60E070E088ED98E0F5
:109470000E94F1A02A960FB6F894DEBF0FBECDBFB2
:10948000DF91CF911F910F91FF90EF90CF900895B2
:1094900084E090E090938C0380938B0349E35DE03C
:1094A00069E47BE28FE79AE40E94552C43E35DE098
:1094B00060E08EE50E947C3562E27DE08AE00E94F9
:1094C0006C3760E17DE084E10E946C3761E07DE013
:1094D0008EE10E946C3765EF7CE088E20E946C3779
:1094E0002A960FB6F894DEBF0FBECDBFDF91CF91A5
:1094F0001F910F91FF90EF90CF900C947932CF9203
:10950000EF92FF920F931F93CF93DF93CDB7DEB708
:109510002A970FB6F894DEBF0FBECDBF40919103DE
:1095200088E0840F405E682F0E945B330E94733294
:1095300080E098E00F94517925E63FE345E557E454
:10954000682F8CEE9CE00E94452F46EE5CE060E0C8
:109550008EE50E946D360E94793280918A038823BD
:1095600009F445C0609177027091780282E00F940F
:10957000F04A80918B0390918C0397FD039695950B
:1095800087959595879560E00E94BB7565E580E0BD
:1095900094E00F946C791A8219821C821B828FE8E6
:1095A00096E4282F9E838D8384E0482FCC24C39497
:1095B000E12CFA8000E01C813E8150E060E070E028
:1095C00088ED98E00E94F1A068ED7CE089EE97E0DC
:1095D0002A960FB6F894DEBF0FBECDBFDF91CF91B4
:1095E0001F910F91FF90EF90CF900D9483752A9665
:1095F0000FB6F894DEBF0FBECDBFDF91CF911F91A4
:109600000F91FF90EF90CF90089584E090E09093B9
:109610008C0380938B0346E951E160E070E08BE6B8
:109620009FE30E94552C80E094E00F94517985359A
:1096300031F041E951E160E084E60E947C356CE75D
:1096400071E18AE00E946C376CE671E184E10E946E
:109650006C3767E571E18EE10E946C3764E471E17B
:1096600088E20E946C370C947932EF92FF920F934C
:109670001F938CE7E82E8AE0F82E06E51FE320E032
:1096800030E043E75AE06DEC76E487EF93E40E9424
:10969000052D62E67AE08AE00E946C376EE47AE09B
:1096A00084E10E946C376CE37AE08EE10E946C37B3
:1096B00060E37AE088E20E946C371F910F91FF907F
:1096C000EF900C947932E7EEF7E08091700380839D
:1096D000809122028183089587E796E10D94D81B3B
:1096E000CF92DF92EF92FF920F931F93CF93DF936E
:1096F000CDB7DEB7A0970FB6F894DEBF0FBECDBFD3
:1097000080918B0390918C030396079748F080918A
:10971000F30C811105C00F94C141833008F4E1C0FE
:109720000091110D10E0F801EE0FFF1FEE0FFF1F6B
:10973000E551F84EC080D180E280F38020E030E037
:1097400048EC52E4C701B6010F944F6D87FD02C18A
:10975000000F111FF801EF50F84E80819181BC017C
:1097600080E090E00F94EF6D20E030E040EA51E4BB
:109770000F94756C9B01AC01C701B6010F944F6D3E
:1097800087FDE8C080918A0381110BC0E091110D23
:10979000F0E0EE0FFF1FEF50F84E80819181892B92
:1097A000A1F460E070E08AE293E40F94C841E09194
:1097B000110DF0E0EE0FFF1FEF50F84E11821082F6
:1097C00061E088ED98E00E94D2A10091110D10E0B7
:1097D000F801EE0FFF1FEF50F84E6081718180E0BD
:1097E00090E00F94EF6D6B017C0120E030E040EFE2
:1097F00052E40F944F6D87FDB8C0000F111F000F8A
:10980000111F0551184E20E030E040EA51E4C70135
:10981000B6010F94756C9B01AC01F80160817181F8
:10982000828193810F944F6D87FD9FC00E948A397A
:1098300068E576E18AE00E946C3766E476E188E2CA
:109840000E946C3766E376E186E30E946C378E01F6
:109850000F5F1F4F80E2F80111928A95E9F7E091BE
:10986000110D84E0E89FF0011124E25EFD4F60815C
:109870007181828193810F94BE6DDC01CB0141E344
:1098800056E1B8010E942A3DE091110DF0E0EE0F83
:10989000FF1FEF50F84E44E356E1BC0180819181F7
:1098A0000E942A3DB80184E10E944E358091110D3D
:1098B00090E00F94C84D482F6EE18EE30E948DAA70
:1098C0000E947932A0960FB6F894DEBF0FBECDBFCE
:1098D000DF91CF911F910F91FF90EF90DF90CF908C
:1098E000089560918B0370918C03072E000C880BF8
:1098F000990B0F94F16D2DEC3CEC4CEC5DE30F9467
:1099000024709B01AC016091360D7091370D8091F0
:10991000380D9091390D0F94766C6093360D7093DD
:10992000370D8093380D9093390DC090110DE12CB7
:10993000F12C00E211E426E33DE042E35DE06EE25B
:109940007DE08AE29DE00F946F3610928C031092B6
:109950008B03E6CE0E94932460939507709396073D
:1099600080939707909398070DCF0E94932460935C
:10997000950770939607809397079093980756CF13
:10998000CF92EF92FF920F931F93CF93DF93CDB7B8
:10999000DEB72A970FB6F894DEBF0FBECDBF20E02A
:1099A00030E046EB5FE466E086E895E10E94452FF3
:1099B00080918A03882309F460C080918B03909181
:1099C0008C039C012D5F3F4F2730310530F461E05F
:1099D00088ED98E00E94D2A150C09C01245031092A
:1099E0002430310538F41A8219821C821B8280E8E7
:1099F00096EC30C09C01285031092430310538F4F0
:109A00001A8219821C821B828DE496EC23C09C0171
:109A10002C5031092430310538F41A8219821C8205
:109A20001B828AE196EC16C09C012051310924303A
:109A3000310538F41A8219821C821B8281E895EC68
:109A400009C044970497C8F41A8219821C821B82A9
:109A500084EB95EC282F9E838D838CE0482FCC24BB
:109A6000C394E12CFA8000E01C813E8150E060E06C
:109A700070E088ED98E00E947FA12A960FB6F894D6
:109A8000DEBF0FBECDBFDF91CF911F910F91FF9031
:109A9000EF90CF900C947932CF92EF92FF920F9388
:109AA0001F93CF93DF93CDB7DEB72A970FB6F89405
:109AB000DEBF0FBECDBF26EB34E546E651E560E1E3
:109AC00089E096E10E94452F80918A03882309F45A
:109AD000F1C080918B0390918C0397FD039695952F
:109AE000879595958795009731F461E088ED98E02A
:109AF0000E94D2A1DFC08130910539F41A82198207
:109B00001C821B828DE693E522C082309105B1F460
:109B100083E69BE4E82E9A8389831C821B828DEA6C
:109B200093E5282F9E838D8388E8482FCC24C39407
:109B3000FA8000E01C813E815FEFB6C08330910562
:109B400079F41A8219821C821B8283E293E5282F02
:109B50009E838D8388E8482FCC24C394E12CE8CFE2
:109B60008430910539F41A8219821C821B8283EE9B
:109B700092E5EDCF8530910539F41A8219821C8265
:109B80001B828BE195ECE3CF86309105B1F41A820C
:109B900019821C821B8287E592E5282F9E838D8384
:109BA00018861F82CC24C394E12CFA8000E01C812B
:109BB0003E8140E0588564E078C08730910539F4F3
:109BC0001A8219821C821B8283EB96EC60C088305B
:109BD000910539F41A8219821C821B8286EE96EC5A
:109BE000B6CF8930910539F41A8219821C821B8202
:109BF00087EE95EC4CC08A30910539F41A821982AF
:109C00001C821B8280EC9CE435C08B30910539F4BA
:109C10001A8219821C821B828EE495EC38C08C302B
:109C20009105A9F41A8219821C821B8248EF5FE910
:109C3000242F5E834D83482F98878F83CC24C39431
:109C4000E12CFA8000E01C813E8158852DC08D30CA
:109C5000910539F41A8219821C821B8286EB9EE4DC
:109C600009C08E30910559F41A8219821C821B8218
:109C70008AEC9EE4282F9E838D8382E00CC00F9790
:109C8000C9F41A8219821C821B8289E69EE4282F5D
:109C90009E838D838CE0482FCC24C394E12CFA80E2
:109CA00000E01C813E8150E060E070E088ED98E0CB
:109CB0000E947FA12A960FB6F894DEBF0FBECDBFDB
:109CC000DF91CF911F910F91FF90EF90CF900C9467
:109CD0007932EF92FF920F931F9386E0E82E86E190
:109CE000F82E06E51FE320E030E042E056E16DE8A3
:109CF0007EE480E090E00E94052D61EF75E18AE04E
:109D00000E946C3765EE75E184E10E946C371F910B
:109D10000F91FF90EF900C94793261E088ED98E01C
:109D20000E94D2A160E084E690E00F946C7960E03C
:109D300085E690E00F946C7960E086E690E00F9401
:109D40006C7960E080E094E00F946C796FEF7FEFC6
:109D500087E094E00F947F7960E080E098E00F94D2
:109D60006C79F894EE27FF270994089541EB55E1AB
:109D700066E57FE380E090E00E94552C6CE975E198
:109D80008EE10E946C376DE875E188E20E946C37C5
:109D90000C9479328F929F92AF92BF92EF92FF9282
:109DA0000F931F93CF93DF93CDB7DEB768970FB6AE
:109DB000F894DEBF0FBECDBF4EED55E166E57FE303
:109DC00080E090E00E94552C6EEC75E18AE00E94E4
:109DD0006C378E010F5F1F4F88E1F80111928A9551
:109DE000E9F76091BE087091BF088091C00890911A
:109DF000C1083CE3832E912CA12CB12CA501940128
:109E00000F943071DA01C9014CEC55E1B8010E94A0
:109E10002A3D7C016091BE087091BF088091C00806
:109E20009091C108A50194010F9430716A307105B9
:109E30008105910530F480E3F7018083C701019625
:109E40007C016091BE087091BF088091C00890911C
:109E5000C1082CE3822E912CA12CB12CA5019401D8
:109E60000F943071DC01CB0140E050E0B7010E945B
:109E70002A3DB80184E10E944E3562EC75E18EE125
:109E80000E946C376091BA087091BB088091BC0841
:109E90009091BD08A50194010F943071DA01C901B8
:109EA00040EC55E1B8010E942A3D7C016091BA085E
:109EB0007091BB088091BC089091BD08A5019401E8
:109EC0000F9430716A3071058105910530F480E39B
:109ED000F7018083C70101967C016091BA087091F7
:109EE000BB088091BC089091BD082CE330E040E0B5
:109EF00050E00F943071DC01CB0140E050E0B7013D
:109F00000E942A3D7C016AEB75E10F94A27595E0F1
:109F1000E90EF11C6091B6087091B7088091B808FD
:109F20009091B90824E630E040E050E00F943071A1
:109F3000DA01C90148EB55E1B7010E942A3DB80199
:109F400088E20E944E350E94793268960FB6F894E6
:109F5000DEBF0FBECDBFDF91CF911F910F91FF905C
:109F6000EF90BF90AF909F908F900895EF92FF92E7
:109F70000F931F93CF93DF93CDB7DEB7A0970FB6A4
:109F8000F894DEBF0FBECDBFF62EE42E8E010F5F1C
:109F90001F4F90E2F80111929A95E9F7811103C0E1
:109FA0006DE775E11BC0813019F460E775E116C0FB
:109FB000823019F460E675E111C0833019F462E56E
:109FC00075E10CC0843019F464E475E107C0853094
:109FD00019F468E375E102C064E375E1C8010F9408
:109FE000A2754E2DB8018F2D0E94D62EA0960FB6C9
:109FF000F894DEBF0FBECDBFDF91CF911F910F91BF
:10A00000FF90EF900895EF92FF920F931F93CF93DD
:10A01000DF93CDB7DEB764970FB6F894DEBF0FBEFF
:10A02000CDBFF62EE42E8E010F5F1F4F94E1F80195
:10A0300011929A95E9F790E29983811104C068EF33
:10A0400074E1C8011DC0813061F48091330281FD4B
:10A0500005C066EF74E1C8010F94A27569EE74E162
:10A060000DC0823079F48091330281FF05C067EE24
:10A0700074E1C8010F94A27566ED74E1CE010296F9
:10A080000F94A2754E2DB8018F2D0E94D62E649686
:10A090000FB6F894DEBF0FBECDBFDF91CF911F91F9
:10A0A0000F91FF90EF900895EF92FF920F931F93FF
:10A0B000CF93DF93CDB7DEB764970FB6F894DEBFCA
:10A0C0000FBECDBFF62EE42E8E010F5F1F4F94E121
:10A0D000F80111929A95E9F790E29983811103C0F2
:10A0E00061EC74E12EC0813061F49091330290767E
:10A0F00029F46FEB74E1C8010F94A27561EB74E170
:10A100001BC0823061F48091330285FF05C06FEA85
:10A1100074E1C8010F94A27564EA74E10DC0833044
:10A1200071F48091330286FF05C062EA74E1C801D0
:10A130000F94A2756EE974E1CE01029603C069E93D
:10A1400074E1C8010F94A2754E2DB8018F2D0E94A5
:10A15000D62E64960FB6F894DEBF0FBECDBFDF914A
:10A16000CF911F910F91FF90EF900895DF92EF92A2
:10A17000FF920F931F93CF93DF93CDB7DEB7A097D6
:10A180000FB6F894DEBF0FBECDBF182F062FD42E0A
:10A19000CE0101967C0180E2F70111928A95E9F7E0
:10A1A000111103C06DE774E11BC0113019F462E7AF
:10A1B00074E116C0123019F467E674E111C013306F
:10A1C00019F46BE574E10CC0143019F468E474E11F
:10A1D00007C0153019F468E374E102C064E374E168
:10A1E000C7010F94A275212F30E022503109E09170
:10A1F0007003F0E02E173F0711F48EE389834D2D95
:10A20000B701802F0E94D62EA0960FB6F894DEBF1D
:10A210000FBECDBFDF91CF911F910F91FF90EF90B7
:10A22000DF900895EF92FF920F931F93CF93DF93E8
:10A23000CDB7DEB764970FB6F894DEBF0FBECDBFC3
:10A24000F62EE42E8E010F5F1F4F94E1F80111925C
:10A250009A95E9F790E29983811104C06CE174E169
:10A26000C80120C0813061F48091330280FD05C0B7
:10A270006AE174E1C8010F94A2756CE074E110C04A
:10A28000823061F48091330280FF05C06AE074E19E
:10A29000C8010F94A27560E074E102C06CEF73E135
:10A2A000CE0102960F94A2754E2DB8018F2D0E94FB
:10A2B000D62E64960FB6F894DEBF0FBECDBFDF91E9
:10A2C000CF911F910F91FF90EF900895EF92FF9221
:10A2D0000F931F93CF93DF93CDB7DEB7A0970FB641
:10A2E000F894DEBF0FBECDBFF62EE42E8E010F5FB9
:10A2F0001F4F90E2F80111929A95E9F7811103C07E
:10A300006BE873E14DC0813019F46CE773E148C02C
:10A31000823019F46FE673E143C0833019F463E6C9
:10A3200073E13EC0843019F462E573E139C08530D1
:10A3300019F466E473E134C0863019F466E373E11E
:10A340002FC0873019F467E273E12AC0883019F40E
:10A3500063E173E125C0893019F46FEF72E120C029
:10A360008A3019F46FEE72E11BC08B3019F464EE81
:10A3700072E116C08C3019F467ED72E111C08D30B6
:10A3800019F46FEC72E10CC08E3019F461EC72E1DB
:10A3900007C08F3019F463EB72E102C06FEA72E11B
:10A3A000C8010F94A2754E2DB8018F2D0E94D62E94
:10A3B000A0960FB6F894DEBF0FBECDBFDF91CF9150
:10A3C0001F910F91FF90EF900895EF92FF920F93DE
:10A3D0001F93CF93DF93CDB7DEB7A0970FB6F89456
:10A3E000DEBF0FBECDBFF62EE42E8E010F5F1F4FD6
:10A3F00090E2F80111929A95E9F7811103C06AE998
:10A4000072E13AC0813019F46EE872E135C08230F1
:10A4100019F460E872E130C0833019F46EE672E13D
:10A420002BC0843019F464E672E126C0853019F43B
:10A4300063E572E121C0863019F462E472E11CC068
:10A44000873019F462E372E117C0883019F464E2CE
:10A4500072E112C0893019F466E172E10DC0909189
:10A46000330290FF04C08A30E1F09BE001C09AE023
:10A4700089131AC063EF71E1C8010F94A2754E2DC4
:10A48000B8018F2D0E94D62EA0960FB6F894DEBF8D
:10A490000FBECDBFDF91CF911F910F91FF90EF9035
:10A4A000089564E072E1E8CF6FEE71E1E5CFEF92DD
:10A4B000FF920F931F93CF93DF93CDB7DEB7A09793
:10A4C0000FB6F894DEBF0FBECDBF44E660E082E376
:10A4D00092E00E943AA6882349F0809132028111CD
:10A4E00001C081E0809332020E94213280918A0370
:10A4F000882359F06091320286E094E00F946C79E1
:10A5000061E088ED98E00E94D2A10E948A3964E25D
:10A5100075E18AE00E946C3764E175E186E30E9490
:10A520006C378E010F5F1F4F80E2F80111928A9500
:10A53000E9F76091320270E080E090E00F94EF6DF7
:10A5400020E030E048EC52E40F94247020E030E04A
:10A550004FE753E40F94566D20E030E040E05FE3B6
:10A560000F94766C0F94BE6DDC01CB0142E155E196
:10A57000B8010E942A3DB80186E10E944E356091E3
:10A58000320270E080E090E00F94EF6D20E030E068
:10A590004FE753E40F94566D7B018C0128E240E7AE
:10A5A00062E280E10E94A9A90E947932A0960FB6CA
:10A5B000F894DEBF0FBECDBFDF91CF911F910F91F9
:10A5C000FF90EF900895CF93DF931F92CDB7DEB742
:10A5D00020E030E043E050E563E081E095E10E9457
:10A5E000452F80918A03882349F120918B03309174
:10A5F0008C03A90144505109809133024430510524
:10A6000010F48D7F06C0285031092430310518F42C
:10A610008260809333026091330281E094E0698329
:10A620000F9451796981681721F081E094E00F94CB
:10A630006C7961E088ED98E00E94D2A10F90DF91E3
:10A64000CF910C947932CF93DF931F92CDB7DEB7C1
:10A6500020E030E044E550E564E08AEC94E10E94BB
:10A66000452F80918A03882399F120918B033091A3
:10A670008C03A901445051098091330244305105A3
:10A6800010F48F7910C0A901485051094430510588
:10A6900018F48F7B806207C02C50310924303105BB
:10A6A00020F48F7D8064809333026091330281E0D7
:10A6B00094E069830F9451796981681721F081E0F2
:10A6C00094E00F946C7961E088ED98E00E94D2A14B
:10A6D0000F90DF91CF910C947932CF93DF931F923B
:10A6E000CDB7DEB720E030E042E151E563E085E23E
:10A6F00094E10E94452F80918A03882349F120919B
:10A700008B0330918C03A90144505109809133028D
:10A710004430510510F48E7F06C028503109243092
:10A72000310518F48160809333026091330281E037
:10A7300094E069830F9451796981681721F081E071
:10A7400094E00F946C7961E088ED98E00E94D2A1CA
:10A750000F90DF91CF910C947932AF92BF92CF924C
:10A76000EF92FF920F931F93CF93DF93CDB7DEB796
:10A770002A970FB6F894DEBF0FBECDBF809122029C
:10A780002FEF829FC001112424E6A22EB12CB50127
:10A790000F941D7188E00E946B2526E834E546EB96
:10A7A00050E566E085E994E10E94452F80918A0397
:10A7B000882309F49AC080918B0390918C039C01AB
:10A7C0002D5F3F4F27303105E0F4809170038823DF
:10A7D00029F060E070E088E00E946B2590917003A2
:10A7E0008091E707981305C0909122028091E807B5
:10A7F00098130F94266461E088ED98E00E94D2A13E
:10A8000074C09C01245031092430310508F04CC03B
:10A81000E09114098AE0E89FF0011124E852F74F13
:10A82000118210821A8219821C821B828CE290E3B0
:10A83000282F9E838D8388E8482FCC24C394E12C55
:10A84000FA8000E01C813E815FEF60E070E088EDFF
:10A8500098E00E947FA18AE894E19093840380931A
:10A86000830388E894E1909382038093810382E2DA
:10A8700092E09093800380937F0381E080937E0336
:10A880008091220290E090938C0380938B039093AD
:10A8900079038093780310927D0310927C03B09229
:10A8A0007B03A0927A0321C09C01285031092430F7
:10A8B000310518F41092700316C09C012C50310918
:10A8C0002430310510F481E00CC09C012051310985
:10A8D0002430310510F482E004C04497049728F432
:10A8E00083E0809370030E94CB3B2A960FB6F894C6
:10A8F000DEBF0FBECDBFDF91CF911F910F91FF90B3
:10A90000EF90CF90BF90AF900C9479320F931F933C
:10A91000CF93DF93CDB7DEB760970FB6F894DEBF65
:10A920000FBECDBF8E010F5F1F4F90E1F801119256
:10A930009A95E9F7882379F0813069F480912202B1
:10A9400046E854E1B80190E00E942A3DA80166E380
:10A9500085E00E94623360960FB6F894DEBF0FBEAA
:10A96000CDBFDF91CF911F910F9108950F931F934A
:10A97000CF93DF93CDB7DEB7A0970FB6F894DEBFC5
:10A980000FBECDBF8E010F5F1F4F90E2F8011192F5
:10A990009A95E9F7813051F48091330280FF03C02A
:10A9A00062EF73E172C064EE73E16FC0823031F424
:10A9B0008091220242EE53E1B8015CC0833079F409
:10A9C0008091330286FF03C06EED73E15EC085FFA8
:10A9D00003C063ED73E159C06AEC73E156C0843083
:10A9E00051F48091330281FF03C062EC73E14DC0EA
:10A9F00069EB73E14AC0863009F56091320270E07C
:10AA000080E090E00F94EF6D20E030E048EC52E4FD
:10AA10000F94247020E030E04FE753E40F94566D1C
:10AA200020E030E040E05FE30F94766C0F94BE6D61
:10AA3000DC01CB0147EB53E1B8011DC0873009F5BC
:10AA400080912302882339F040EB53E1B80190E074
:10AA50000E942A3D07C069EA73E1C8010F94A275FC
:10AA6000CE01079620912B02222341F047EA53E1C1
:10AA7000BC01822F90E00E942A3D0AC063EA73E184
:10AA800005C08D3051F464E973E1C8010F94A275DB
:10AA9000A80166E384E00E946233A0960FB6F894A2
:10AAA000DEBF0FBECDBFDF91CF911F910F910895F3
:10AAB0000F931F93CF93DF93CDB7DEB7A0970FB659
:10AAC000F894DEBF0FBECDBF8E010F5F1F4F90E227
:10AAD000F80111929A95E9F79091330290FD04C024
:10AAE0008C3010F08F5F36C08230C9F460911E0246
:10AAF00070911F0280912002909121020F94BE6DEF
:10AB0000DC01CB014AEA52E1B8010E942A3D4DEA3C
:10AB100052E1BC018091F1179091F2172BC0833064
:10AB2000C9F460911A0270911B0280911C029091ED
:10AB30001D020F94BE6DDC01CB0145EA52E1B80164
:10AB40000E942A3D48EA52E1BC018091E9179091A8
:10AB5000EA1710C08930A9F480910F0DF4E68F9F99
:10AB6000C00111246FEF70E00F941D71CB0143EA17
:10AB700052E1B8010E942A3DA80166E384E00E94E8
:10AB80006233A0960FB6F894DEBF0FBECDBFDF9143
:10AB9000CF911F910F9108950F931F93CF93DF9340
:10ABA000CDB7DEB760970FB6F894DEBF0FBECDBF4E
:10ABB00020918B0330918C03A9014D5F5F4F47308B
:10ABC000510508F44CC08091110D082F10E0F801D8
:10ABD000EE0FFF1FEF50F84E37FD9A013595279580
:10ABE0003595279540815181240F351F37FD2AC0A7
:10ABF0000F94E9596091110D062F10E0F801EE0F46
:10AC0000FF1FEF50F84E20918B0330918C0337FFDC
:10AC100002C02D5F3F4F359527953595279540818B
:10AC20005181240F351FAC014E50510924173507AF
:10AC300034F0862F0F94E9599C012F503109922F3F
:10AC4000832F02C090E080E0000F111FF801EF5049
:10AC5000F84E9083818310928C0310928B03809125
:10AC60008A03882329F061E088ED98E00E94D2A150
:10AC70000E948A396BED71E184E10E946C376BECC4
:10AC800071E186E30E946C378E010F5F1F4F80E1F8
:10AC9000F80111928A95E9F7E091110D84E0E89F9F
:10ACA000F0011124E25EFD4F608171818281938108
:10ACB0000F94BE6DDC01CB0148EC51E1B8010E945C
:10ACC0002A3DF80101900020E9F7BF0161507109A8
:10ACD000E091110DF0E0EE0FFF1FEF50F84E46EC43
:10ACE00051E1808191810E942A3DB8018EE10E944C
:10ACF0004E358091110D90E00F94C84D482F68E2B9
:10AD00008EE30E948DAA0E94793260960FB6F89465
:10AD1000DEBF0FBECDBFDF91CF911F910F91089580
:10AD20000F931F93CF93DF93CDB7DEB760970FB626
:10AD3000F894DEBF0FBECDBF80918B0390918C0342
:10AD40009C012D5F3F4F27303105F0F097FDC90181
:10AD500095958795959587952091E9173091EA17F4
:10AD6000820F931F97FD06C08A3B91052CF089EB5B
:10AD700090E002C080E090E09093EA178093E9179A
:10AD800010928C0310928B0380918A03882329F000
:10AD900061E088ED98E00E94D2A10E948A3964EBBC
:10ADA00071E184E10E946C3764EA71E186E30E94FC
:10ADB0006C378E010F5F1F4F80E1F80111928A9569
:10ADC000E9F760911A0270911B0280911C02909128
:10ADD0001D020F94BE6DDC01CB0141EA51E1B801C7
:10ADE0000E942A3DF80101900020E9F7BF0161505F
:10ADF00071094FE951E18091E9179091EA170E949A
:10AE00002A3DB8018EE10E944E358FEF9FEF0F94DF
:10AE1000C84D482F68E28EE30E948DAA0E947932C5
:10AE200060960FB6F894DEBF0FBECDBFDF91CF9115
:10AE30001F910F910895BF92CF92DF92EF92FF92F0
:10AE40000F931F93CF93DF93CDB7DEB72A970FB63B
:10AE5000F894DEBF0FBECDBF47E956E16EE876E15C
:10AE600081E896E10E94B02B80918A03882309F43F
:10AE700059C080918B0390918C039C01295F3F4FB7
:10AE80002F30310538F51A8219828CE69BE4082FA1
:10AE90009C838B8386E59FE3282F9E838D8388E8A0
:10AEA000D82E4D2DCC24C394E12CFA801C813E81F8
:10AEB0005FEF60E070E088ED98E00E947FA11A8269
:10AEC00019821C821B8285E39BE4282F9E838D833D
:10AED0004D2D14C09C012850310928303105D0F483
:10AEE0001A8219821C821B8283E298E5282F9E8396
:10AEF0008D8388E8482FCC24C394E12CFA8000E0AD
:10AF00001C813E815FEF60E070E088ED98E00E9478
:10AF10007FA108C04097089728F461E088ED98E089
:10AF20000E94D2A12A960FB6F894DEBF0FBECDBF05
:10AF3000DF91CF911F910F91FF90EF90DF90CF9015
:10AF4000BF900C94793280E796E10D94D81B8CE683
:10AF500096E10D94D81BCF92EF92FF920F931F931F
:10AF6000CF93DF93CDB7DEB72A970FB6F894DEBF45
:10AF70000FBECDBF60E070E0CB010F94C8411092CE
:10AF8000360D1092370D1092380D1092390D41E0A8
:10AF90006091110D86E39DE00F948D418091110D1C
:10AFA00090E0FC01EE0FFF1FEF50F84E24E4289FC5
:10AFB000D001299FB00D1124A656B84F8D919C91B8
:10AFC000918380838091330280FF16C083E29DEEDF
:10AFD000E82E9A8389831C821B828AE29DEE282FA9
:10AFE0009E838D8388E8482FCC24C394FA8000E0A8
:10AFF0001C813E815FEF13C01A8219821C821B8262
:10B0000080E79BE4282F9E838D8384E0482FCC2407
:10B01000C394E12CFA8000E01C813E8150E060E0A6
:10B0200070E088ED98E00E947FA12A960FB6F89410
:10B03000DEBF0FBECDBFDF91CF911F910F91FF906B
:10B04000EF90CF900895CF92EF92FF920F931F93BE
:10B05000CF93DF93CDB7DEB72A970FB6F894DEBF54
:10B060000FBECDBF8091330280FD02C06BE001C0F6
:10B070006CE028E535E545EE51E588E296E10E9471
:10B08000452F80918A03882309F4F3C080918B03B4
:10B0900090918C0397FD0396959587959595879547
:10B0A000009731F461E088ED98E00E94D2A1E1C000
:10B0B0008130910539F41A8219821C821B828CE43A
:10B0C0009DE4C4C08230910549F41092110D1A829A
:10B0D00019821C821B828CEC95E509C08330910596
:10B0E000A9F41A8219821C821B8280E996E5282F16
:10B0F0009E838D8384E0482FCC24C394E12CFA8076
:10B1000000E01C813E8150E064E0AEC084309105D7
:10B1100029F40E94CB3B0E946C4BABC0853091055B
:10B1200021F40E94CB3B0FDFA4C08630910541F48F
:10B130000E94CB3B08DF81E296E10F94D81B99C0B7
:10B1400087309105C9F41092110D80E00E94DF6BE9
:10B150001A8219821C821B8286E59BE5282F9E831A
:10B160008D8388E8482FCC24C394E12CFA8000E03A
:10B170001C813E815FEF77C08830910521F41092E9
:10B18000110DE9DE76C08930910509F04BC01A82B5
:10B1900019821C821B828CE290E3282F9E838D8370
:10B1A00088E8482FCC24C394E12CFA8000E01C816D
:10B1B0003E815FEF60E070E088ED98E00E947FA143
:10B1C00087E196E1909384038093830385E196E180
:10B1D00090938203809381038FE09DE0909380039E
:10B1E00080937F0385E080937E0380910F0D24E69A
:10B1F000829FC00111246FEF70E00F941D71709356
:10B200008C0360938B03709379036093780310929F
:10B210007D0310927C0384E690E090937B038093FF
:10B220007A0327C02091330220FF05C08A309105A0
:10B2300079F12BE001C02AE030E028173907C9F482
:10B240001A8219821C821B8288EB9BEE282F9E8318
:10B250008D8382E0482FCC24C394E12CFA8000E057
:10B260001C813E8150E060E070E088ED98E00E9433
:10B270007FA12A960FB6F894DEBF0FBECDBFDF9137
:10B28000CF911F910F91FF90EF90CF900C94793256
:10B290001A8219821C821B8285E39BE4D7CFEBE1E3
:10B2A000FCE12491222341F03091C00035FFFCCF16
:10B2B0002093C6003196F5CFE3E5F9E124912223EE
:10B2C00041F03091C00035FFFCCF2093C60031968D
:10B2D000F5CFFC018191882339F09091C00095FF52
:10B2E000FCCF8093C600F6CF8091C00085FFFCCFD5
:10B2F0008AE08093C600089508950E94492B0E9419
:10B300006C4B8CEF9BE10F94D81B60E088ED98E0CC
:10B310000C94D2A14F925F926F927F928F929F92E4
:10B32000AF92BF92CF92DF92EF92FF920F931F9353
:10B33000CF93DF93CDB7DEB762970FB6F894DEBF39
:10B340000FBECDBF0E94932460939507709396071C
:10B3500080939707909398076091110D84E4689FFC
:10B36000F0011124E656F84F808191819A838983F8
:10B37000CE0101960F94F259C090110DD12CF60117
:10B38000EE0FFF1FEE0FFF1FE551F84E20E030E0FB
:10B3900040EA51E460817181828193810F94756CE0
:10B3A0000F94BE6D2B013C01F601EE0FFF1FEF5015
:10B3B000F84E6081718180E090E00F94EF6D20E0A5
:10B3C00030E040EA51E40F94756C0F94BE6D4B0170
:10B3D0005C01720157FE02C0E12CF12C2DE72E9D7D
:10B3E000C0012F9D900D11240F941D71D0908503E5
:10B3F0006D1518F060938503D62E40E050E064E6AA
:10B400007FE580E090E00E94552CC40109968E15DE
:10B410009F051CF046ED5BE102C047EC5BE16AE092
:10B4200083E00E947C3542EB5BE164E183E00E94B3
:10B430007C358D2D0E94FF2DC4010497E816F90676
:10B440000CF41BC1B4016C5F7F4F6E157F050CF4CB
:10B4500014C10F94084A60E070E0CB010F94C8411A
:10B460001092360D1092370D1092380D1092390D42
:10B4700041E06091110D86E39DE00F948D41409075
:10B480002F175090301760903117709032178091BD
:10B49000F3169091F416A091F516B091F6168B87DD
:10B4A0009C87AD87BE878091E7169091E816A091A2
:10B4B000E916B091EA168F87988BA98BBA8BC0904A
:10B4C0001F17D0902017E0902117F0902217A701A6
:10B4D000960160E078E08FEC96E40F94566D4B0196
:10B4E0005C0160932F1770933017809331179093FE
:10B4F0003217A701960160E070E081EE95E40F94A9
:10B50000566D6093F3167093F4168093F51690932E
:10B51000F61680E090E0A0E8BFE38093E7169093F2
:10B52000E816A093E916B093EA16C090110D94E0C6
:10B53000C99EF0011124E15FF84E208131814281E2
:10B54000538160E070E080E89FE30F94566D9B01AB
:10B55000AC016091360D7091370D8091380D90914E
:10B56000390D0F94756C6093360D7093370D809381
:10B57000380D9093390D8501740126E33DE042E3D7
:10B580005DE06EE27DE08AE29DE00F946F36C09050
:10B59000110DA4E0CA9EF0011124E15FF84E208154
:10B5A00031814281538160E070EC8CE394E40F942C
:10B5B000566D9B01AC016091360D7091370D8091F5
:10B5C000380D9091390D0F94756C6093360D709312
:10B5D000370D8093380D9093390DE0902F17F09030
:10B5E0003017009131171091321726E33DE042E306
:10B5F0005DE06EE27DE08AE29DE00F946F3640925E
:10B600002F175092301760923117709232178B8536
:10B610009C85AD85BE858093F3169093F416A09318
:10B62000F516B093F6168F859889A989BA89809303
:10B63000E7169093E816A093E916B093EA161A82DB
:10B6400019821C821B8285EF92E6282F9E838D83B0
:10B6500088E8482F8F838FEF888719861A86C12C38
:10B66000E12CFA8000E01C813E815FEF60E070E039
:10B6700088ED98E00E94F1A002C00E9479326296A3
:10B680000FB6F894DEBF0FBECDBFDF91CF911F91F3
:10B690000F91FF90EF90DF90CF90BF90AF909F9071
:10B6A0008F907F906F905F904F9008954F925F9230
:10B6B0006F927F92AF92BF92CF92DF92EF92FF9202
:10B6C0000F931F93CF93DF93CDB7DEB72A970FB6B3
:10B6D000F894DEBF0FBECDBF0E9493246093950700
:10B6E0007093960780939707909398076091110D38
:10B6F00084E4689FF0011124E656F84F808191811F
:10B700009A838983CE0101960F94F2590091110D0D
:10B7100010E0F801EE0FFF1FEE0FFF1FE551F84E8E
:10B7200020E030E040EA51E46081718182819381C0
:10B730000F94756C0F94BE6D6B017C01000F111F8F
:10B74000F801EF50F84E6081718180E090E00F9435
:10B75000EF6D20E030E040EA51E40F94756C20E09A
:10B7600030E040E251E40F94756C0F94BE6D2B01F4
:10B770003C015B01D7FE02C0C12CD12CAC14BD042E
:10B7800074F4C20143968C159D054CF080917C0D9C
:10B7900084FD4CC00E94ECF5882309F447C02DE7D6
:10B7A0002C9DC0012D9D900D1124B5010F941D718C
:10B7B00010918503611718F060938503162F40E000
:10B7C00050E064E67FE580E090E00E94552C89E03F
:10B7D000480E511C4C145D041CF04FE45BE102C0A8
:10B7E0004CE35BE16AE083E00E947C3549E25BE187
:10B7F00064E183E00E947C35812F0E94FF2D0E942E
:10B8000079322A960FB6F894DEBF0FBECDBFDF9116
:10B81000CF911F910F91FF90EF90DF90CF90BF904D
:10B82000AF907F906F905F904F90089560E070E0D0
:10B83000CB010F94C8411A8219821C821B8288E0B6
:10B8400090E6282F9E838D8384E0482F8F8318866F
:10B8500019861A86CC24C394E12CFA8000E01C815E
:10B860003E8150E060E070E088ED98E00E94F1A039
:10B87000620195CFEF92FF920F931F93CF93DF93C7
:10B880001F921F92CDB7DEB74091910388E0840FDD
:10B89000405E682F0E945B330E9473326091110DED
:10B8A00084E4689FF0011124E656F84F808191816D
:10B8B0009A838983CE0101960F94F25988E9E82E84
:10B8C0008BE1F82E04E61FE520E030E042E95BE181
:10B8D00067EB7CE580E090E00E94052D62E87BE16B
:10B8E00084E10E946C370E9479320F900F90DF91B3
:10B8F000CF911F910F91FF90EF90089584E090E019
:10B9000090938C0380938B034EE759E166E57FE3C8
:10B9100080E090E00E94552C6DE679E184E10E9480
:10B920006C376CE579E18EE10E946C370C947932CA
:10B9300084E090E090938C0380938B034CE858E173
:10B9400066E57FE380E090E00E94552C6CE778E1AB
:10B9500084E10E946C376DE678E18EE10E946C37DD
:10B960006DE578E188E20E946C370C947932CF92D1
:10B97000EF92FF920F931F93CF93DF93CDB7DEB774
:10B980002A970FB6F894DEBF0FBECDBF0F9496492D
:10B990001A8219821C821B8289ED96E7282F9E83CA
:10B9A0008D8382E0482FCC24C394E12CFA8000E000
:10B9B0001C813E8150E060E070E088ED98E00E94DC
:10B9C000F1A02A960FB6F894DEBF0FBECDBFDF916F
:10B9D000CF911F910F91FF90EF90CF900C94AD31CC
:10B9E0008F929F92AF92BF92CF92EF92FF920F935E
:10B9F0001F93CF93DF93CDB7DEB72A970FB6F89496
:10BA0000DEBF0FBECDBF28EF31E64FED50E666E05A
:10BA10008BEE97E10E94452F80918A03882309F4D9
:10BA200070C0A0908B03B0908C03450183E0880E1A
:10BA3000911C61E087E08816910428F488ED98E075
:10BA40000E94D2A15EC088ED98E00E94D2A11A8225
:10BA500019821C821B828CE290E3282F9E838D83A7
:10BA600088E8482F8F838FEF8887CC24C394E12CFC
:10BA7000FA8000E01C813E815FEF60E070E088EDBD
:10BA800098E00E947FA18FED97E1909384038093CB
:10BA900083038DED97E1909382038093810320913E
:10BAA000110D30E0C501B7FCC401959587959595BA
:10BAB0008795815092E2929FF001939FF00D11249F
:10BAC000E80FF11DEE0FFF1FE656F84FF0938003CD
:10BAD000E0937F0382E080937E0380819181909345
:10BAE0008C0380938B039093790380937803109257
:10BAF0007D0310927C038CE291E090937B03809312
:10BB00007A032A960FB6F894DEBF0FBECDBFDF9141
:10BB1000CF911F910F91FF90EF90CF90BF90AF907A
:10BB20009F908F900C9479328F929F92AF92BF9298
:10BB3000CF92DF92EF92FF920F931F93CF93DF93F9
:10BB4000CDB7DEB7A0970FB6F894DEBF0FBECDBF5E
:10BB500010E29E012F5F3F4F7901F901212F1192D1
:10BB60002A95E9F79091900338E1839F60011124B1
:10BB7000FE013B965F01992321F1C601805F974F3B
:10BB80000F94597900E026E73BE1A7010E945D3E52
:10BB90008C0180E20A151B0520F4F80181938F01C6
:10BBA000F9CF60E77BE1C8010F94A275C601825FFF
:10BBB000974F0F945E79B8016B5F7F4F4EE65BE164
:10BBC00033C0C601875F974F0F945E794CE65BE107
:10BBD000B7010E942A3D4C01FFEF8F1A9F0AFC011A
:10BBE0001083C601855F974F0F945E794AE65BE14B
:10BBF000B4010E942A3D8C0180E20A151B0520F445
:10BC0000F80181938F01F9CF64E67BE1C8010F94BD
:10BC1000A275C601835F974F0F945179B8016B5F8E
:10BC20007F4F42E65BE190E00E942A3DA70166E378
:10BC300084E00E946233A0960FB6F894DEBF0FBE78
:10BC4000CDBFDF91CF911F910F91FF90EF90DF90CB
:10BC5000CF90BF90AF909F908F9008950F931F93B8
:10BC6000CF93DF93CDB7DEB72A970FB6F894DEBF38
:10BC70000FBECDBF162F042F28E1829FC0011124D3
:10BC8000BC016F5F774F48E050E0CE0101960F9402
:10BC900041791986402FBE016F5F7F4F812F0E942F
:10BCA000D62E2A960FB6F894DEBF0FBECDBFDF9119
:10BCB000CF911F910F910895DF92EF92FF920F9312
:10BCC0001F93CF93DF93CDB7DEB7A0970FB6F8944D
:10BCD000DEBF0FBECDBF182F062FD42E80E098E018
:10BCE0000F9451799E012F5F3F4F790190E2F90146
:10BCF00011929A95E9F7111103C06FEF77E104C033
:10BD0000811730F464EF77E1C7010F94A27513C077
:10BD1000212F30E02150310988E1829FF001839F7B
:10BD2000F00D1124BF016F5F774F48E050E0C7016D
:10BD30000F94417919864D2DB701802F0E94D62E80
:10BD4000A0960FB6F894DEBF0FBECDBFDF91CF91A6
:10BD50001F910F91FF90EF90DF900895EF92FF9267
:10BD60000F931F93CF93DF93CDB7DEB7A0970FB696
:10BD7000F894DEBF0FBECDBFF62EE42E8E010F5F0E
:10BD80001F4F90E2F80111929A95E9F7811103C0D3
:10BD90006CEA77E120C0813019F460EA77E11BC0DA
:10BDA000823019F46EE877E116C0833019F465E843
:10BDB00077E111C0843019F461E877E10CC0853077
:10BDC00019F46AE777E107C0863019F46AE677E18B
:10BDD00002C066E677E1C8010F94A2754E2DB80146
:10BDE0008F2D0E94D62EA0960FB6F894DEBF0FBE00
:10BDF000CDBFDF91CF911F910F91FF90EF900895EC
:10BE0000DF92EF92FF920F931F93CF93DF93CDB703
:10BE1000DEB7A0970FB6F894DEBF0FBECDBF182FC8
:10BE2000062FD42E80E098E00F945179E82FCE01B0
:10BE300001967C0180E2D7011D928A95E9F71111E4
:10BE400003C06AE077E10AC0212F30E0F0E0CF01C3
:10BE500001962817390731F460E077E1C7010F94A4
:10BE6000A2751FC0CF0102962817390719F463EF96
:10BE700076E1F4CF33962E173F0719F464EE76E19E
:10BE8000EDCF2150310988E1829FB001839F700D71
:10BE900011246F5F774F48E050E0C7010F9441795C
:10BEA00019864D2DB701802F0E94D62EA0960FB671
:10BEB000F894DEBF0FBECDBFDF91CF911F910F91E0
:10BEC000FF90EF90DF9008950F94084A60917702F9
:10BED0007091780282E00F94F04A60E070E08AE2AC
:10BEE00093E40F94C84160E088ED98E00C94D2A1EF
:10BEF000CF92EF92FF920F931F93CF93DF931F92F6
:10BF00001F92CDB7DEB70F94084A60917702709107
:10BF1000780282E00F94F04A60E088ED98E00E9499
:10BF2000D2A11092360D1092370D1092380D10924A
:10BF3000390D41E06091110D86E39DE00F948D4134
:10BF40008091F80C882349F02091F40C3091F50C85
:10BF50004091F60C5091F70C18C0E091110D84E05F
:10BF6000E89FF0011124E15FF84E20813181428188
:10BF7000538160912D0270912E0280912F02909139
:10BF800030020F94566D9B01AC016091360D70919B
:10BF9000370D8091380D9091390D0F94756C609329
:10BFA000360D7093370D8093380D9093390D20E046
:10BFB00030E040E752E4609141027091420280918A
:10BFC0004302909144020F94566DC090110D7B0175
:10BFD0008C0126E33DE042E35DE06EE27DE08AE233
:10BFE0009DE00F946F3680917C0D83FD07C01A820F
:10BFF000198260E0CE0101960F94F2590F900F90D4
:10C00000DF91CF911F910F91FF90EF90CF90089506
:10C01000CF92EF92FF920F931F934091910388E08C
:10C02000840F405E682F0E945B330E947332E09160
:10C03000110DF0E0EE0FFF1FEF50F84E808191815F
:10C04000892B41F08091F30C811104C00F94C14100
:10C05000823058F192E2E92E9BE1F92E04E61FE5C9
:10C0600020E030E04CE15BE160E973E680E090E0E5
:10C070000E94052D68E07BE18AE00E946C3763EF47
:10C080007AE184E10E946C3765EE7AE18EE10E94EC
:10C090006C3764ED7AE188E20E946C371F910F9152
:10C0A000FF90EF90CF900C947932C090110D84E006
:10C0B000C89EF0011124E15FF84E20813181428158
:10C0C000538160E070E080E09FE30F94566D9B0128
:10C0D000AC016091360D7091370D8091380D9091C3
:10C0E000390D0F94766C6093360D7093370D8093F5
:10C0F000380D9093390DE12CF12C00E010E426E38B
:10C100003DE042E35DE06EE27DE08AE29DE00F9477
:10C110006F36A0CF4FE75AE166E57FE380E090E01D
:10C120000E94552C6CE67AE184E10E946C3769EE3E
:10C1300077E08EE10E944E350C9479328F929F9277
:10C14000AF92BF92CF92DF92EF92FF927B0160E0BD
:10C1500070E00F94C8724B015C01B70180E090E081
:10C160000F94EF6D9B01AC01C501B4010F942470D5
:10C170006B017C0120E03FEF4FE757E40F944F6DD8
:10C1800087FF0FC020E030E0A901C701B6010F947E
:10C190004F6D87FD09C0C701B6010F94C36DCB0178
:10C1A00005C08FEF9FEF02C080E090E0FF90EF901E
:10C1B000DF90CF90BF90AF909F908F900895CF92D7
:10C1C000DF92EF92FF920F931F93CF93DF93CDB740
:10C1D000DEB764970FB6F894DEBF0FBECDBF182F41
:10C1E000D62EC42ECE0101967C0184E1F701119276
:10C1F0008A95E9F7111106C062ED77E1C7010F9446
:10C20000A27522C064EC77E1C7010F94A275D70133
:10C210000D900020E9F7AD01415051091150153042
:10C2200058F484E0189FF0011124E152FD4F608121
:10C2300071818281938103C060E070E0CB0100E0F6
:10C2400020E030E00E945D3E4C2DB7018D2D0E9414
:10C25000D62E64960FB6F894DEBF0FBECDBFDF9129
:10C26000CF911F910F91FF90EF90DF90CF900895A5
:10C27000DF92EF92FF920F931F93CF93DF93CDB78F
:10C28000DEB764970FB6F894DEBF0FBECDBF9E0138
:10C290002F5F3F4F790194E1F90111929A95E9F7E7
:10C2A00081110EC06091110DF4E46F9FB001112453
:10C2B0006B52784F44E150E0C9010E94363F85C07F
:10C2C0008130E9F5809190038823E1F0E091110D30
:10C2D00014E41E9FF0011124E656F84F4EEB57E18F
:10C2E000B901868197810E942A3DE091110D1E9F20
:10C2F000F0011124E656F84F4EEB57E1BC01808562
:10C30000918561C000E010E0C90132E2D32E209196
:10C31000110DF801D29EE00DF11D1124EE0FFF1F4B
:10C32000E656F84F41EC57E1BC01808191810E94B3
:10C330002A3D0F5F1F4F0330110549F746C0823079
:10C3400071F4E091110D24E4E29FF0011124E6560E
:10C35000F84F4CEB57E1B70182A993A934C0833061
:10C3600099F4E091110D34E4E39FF0011124E656B5
:10C37000F84F67A970AD81AD92AD00E029EB37E1D0
:10C38000A7010E945D3E21C0843071F4E091110D3F
:10C3900084E4E89FF0011124E656F84F84A947EBA6
:10C3A00057E1B90190E00FC0853079F4E091110DAB
:10C3B00024E4E29FF0011124E656F84F45EB57E1E3
:10C3C000B70185A996A90E942A3DA70166E384E0EA
:10C3D0000E94623364960FB6F894DEBF0FBECDBFE5
:10C3E000DF91CF911F910F91FF90EF90DF90089513
:10C3F0000F931F93CF93DF93CDB7DEB72A970FB676
:10C40000F894DEBF0FBECDBF882301F18E010F5F10
:10C410001F4F9AE0F80111929A95E9F7E091110DFA
:10C4200092E2E99FF0011124E80FF11DEE0FFF1FCA
:10C43000E856F84F4BED57E1B801808191810E9499
:10C440002A3DA80166E384E00E9462332A960FB673
:10C45000F894DEBF0FBECDBFDF91CF911F910F913A
:10C4600008958F929F92AF92BF92CF92DF92EF92F8
:10C47000FF920F931F93CF93DF93CDB7DEB7A097B3
:10C480000FB6F894DEBF0FBECDBFE82E80E098E077
:10C490000F945179EE2009F495C08E1508F475C0FB
:10C4A00010E29E012F5F3F4F6901F901212F119288
:10C4B0002A95E9F7EA948091900338E1E39E7001B0
:10C4C0001124FE013B965F01882321F1C701805FA3
:10C4D000974F0F94597900E023E637E1A6010E94B7
:10C4E0005D3E8C0180E20A151B0520F4F801819362
:10C4F0008F01F9CF6DE577E1C8010F94A275C701EF
:10C50000825F974F0F945E79B8016B5F7F4F4BE569
:10C5100057E133C0C701875F974F0F945E7949E5B4
:10C5200057E1B6010E942A3D4C01FFEF8F1A9F0A86
:10C53000FC011083C701855F974F0F945E7947E533
:10C5400057E1B4010E942A3D8C0180E20A151B05C7
:10C5500020F4F80181938F01F9CF61E577E1C801FB
:10C560000F94A275C701835F974F0F945179B8015B
:10C570006B5F7F4F4FE457E190E00E942A3DA60198
:10C5800066E384E00E9462331DC0F12C90E09C01C0
:10C590002F5F3F4FE216F30619F46BE377E10FC00C
:10C5A0009C012E5F3F4FE216F30619F467E277E134
:10C5B00006C00396E816F90629F463E177E186E3FD
:10C5C0000E946C37A0960FB6F894DEBF0FBECDBFA9
:10C5D000DF91CF911F910F91FF90EF90DF90CF905F
:10C5E000BF90AF909F908F9008958F929F92AF923F
:10C5F000BF92CF92DF92EF92FF920F931F93CF9350
:10C60000DF93CDB7DEB72A970FB6F894DEBF0FBE23
:10C61000CDBF0E94932460939507709396078093F3
:10C620009707909398079091DE118091DD119813F0
:10C6300031C01A8219821C821B828AE39CE5282F52
:10C640009E838D8384E0482F8F83188619861A86EF
:10C65000CC24C394E12CFA8000E01C813E8150E0A0
:10C6600060E070E088ED98E00E94F1A0409A2A9680
:10C670000FB6F894DEBF0FBECDBFDF91CF911F91F3
:10C680000F91FF90EF90DF90CF90BF90AF909F9071
:10C690008F90089540E050E064E67FE580E090E010
:10C6A0000E94552C4FE95BE164E183E00E947C35F8
:10C6B00083E00F94F4494B015C0120E030EC4CE343
:10C6C00054E460911F177091201780912117909169
:10C6D00022170F9424700F94F46F6B017C01A3E870
:10C6E000BFEFA50194010F949771A70196010F94D4
:10C6F0005271822F0E94FF2D2A960FB6F894DEBF4A
:10C700000FBECDBFDF91CF911F910F91FF90EF90A2
:10C71000DF90CF90BF90AF909F908F900C94793224
:10C720004F925F926F927F928F929F92AF92BF9241
:10C73000CF92DF92EF92FF920F931F93CF93DF93ED
:10C74000CDB7DEB72E970FB6F894DEBF0FBECDBFC4
:10C750000E94AD31882309F4CEC040902F1750902D
:10C76000301760903117709032178090F3169090C8
:10C77000F416A090F516B090F6168091E7169091F9
:10C78000E816A091E916B091EA168B879C87AD87D1
:10C79000BE87C0901F17D0902017E0902117F0900F
:10C7A0002217A701960160E078E08FEC96E40F94E1
:10C7B000566D60932F1770933017809331179093B5
:10C7C0003217A701960160E070E081EE95E40F94C6
:10C7D000566D6093F3167093F4168093F51690934C
:10C7E000F61680E090E0A0E8BFE38093E716909310
:10C7F000E816A093E916B093EA160F94084A10922F
:10C80000360D1092370D1092380D1092390D41E00F
:10C810006091110D86E39DE00F948D41C090110D44
:10C8200094E0C99EF0011124E15FF84E208131812E
:10C830004281538160E070EC83E294E40F94566D82
:10C840009B01AC016091360D7091370D8091380DD0
:10C850009091390D0F94766C6093360D7093370D6F
:10C860008093380D9093390DE0902F17F09030178A
:10C87000009131171091321726E33DE042E35DE06D
:10C880006EE27DE08AE29DE00F946F3640922F17B2
:10C890005092301760923117709232178092F316CF
:10C8A0009092F416A092F516B092F6168B859C85A0
:10C8B000AD85BE858093E7169093E816A093E916A0
:10C8C000B093EA161A8219821C821B8282E994E6CE
:10C8D000282F9E838D8388E8482FCC24C394E12C95
:10C8E000FA8000E01C813E815FEF60E070E088ED3F
:10C8F00098E00E94F1A02E960FB6F894DEBF0FBE0E
:10C90000CDBFDF91CF911F910F91FF90EF90DF90FE
:10C91000CF90BF90AF909F908F907F906F905F90DF
:10C920004F9008958F929F92AF92BF92CF92DF92D5
:10C93000EF92FF920F931F93CF93DF93CDB7DEB7A4
:10C940002A970FB6F894DEBF0FBECDBF0E94932486
:10C950006093950770939607809397079093980735
:10C960009091DE118091DD1198133BC00E94CB3B6A
:10C970008091770290917802880F991F63E070E0B0
:10C980000F941D7182E00F94F04A1A8219821C8262
:10C990001B828EE597E6282F9E838D8384E0482FA7
:10C9A000CC24C394E12CFA8000E01C813E8150E04D
:10C9B00060E070E088ED98E00E94F1A02A960FB642
:10C9C000F894DEBF0FBECDBFDF91CF911F910F91C5
:10C9D000FF90EF90DF90CF90BF90AF909F908F909F
:10C9E000089540E050E064E67FE580E090E00E943A
:10C9F000552C40EC5AE164E183E00E947C3583E0F1
:10CA00000F94F4494B015C0120E030EC43E254E424
:10CA100060911F1770912017809121179091221714
:10CA20000F9424700F94F46F6B017C01ADE7B0E0BC
:10CA3000A50194010F948B71A70196010F94527177
:10CA4000822F0E94FF2D2A960FB6F894DEBF0FBEEC
:10CA5000CDBFDF91CF911F910F91FF90EF90DF90AD
:10CA6000CF90BF90AF909F908F900C9479322F927F
:10CA70003F924F925F926F927F928F929F92AF926E
:10CA8000BF92CF92DF92EF92FF920F931F93CF93BB
:10CA9000DF93CDB7DEB7A9970FB6F894DEBF0FBE10
:10CAA000CDBF80917C0D85FD29C04091910388E028
:10CAB000840F405E682F0E945B330E94733284E0D3
:10CAC00090E090938C0380938B0340E050E066E508
:10CAD0007FE380E090E00E94552C67E479E18FE0ED
:10CAE0000E946C3764E379E189E10E946C370E940F
:10CAF00079328AE39DE00F94485DC7C180FF04C08E
:10CB00008091F60E8823A1F040E050E066E57FE3D7
:10CB100080E090E00E94552C64E279E180E10E947F
:10CB20006C370E9479328AE39DE00F94575CADC167
:10CB30008AE39DE00F942E5D40E062ED72E08AE3AF
:10CB40009DE00F94595D80E098E00F9451798DA39A
:10CB5000212C8AE0382E80E59CE09CA38BA39BE0EF
:10CB6000C92E98E0D92E10E0DE0111967D01EDA1CD
:10CB70001E1709F468C1D701E0E21D92EA95E9F7B2
:10CB800068E179E1C7010F94A275B7018AE39DE0DE
:10CB90000F94776162E179E1C7010F94A275F70103
:10CBA00001900020E9F7CF0101975C0148E050E0D7
:10CBB000B6016A5071090F944179D50118961C92FB
:10CBC00060E179E1C7010F948375B7018AE39DE0C5
:10CBD0000F94776163E079E1C7010F94A275F701C3
:10CBE00001900020E9F731975F01AE18BF08C60138
:10CBF00002970F945E79B7016A0D7B1D41E059E100
:10CC00000E942A3DB7018AE39DE00F947761EFED22
:10CC1000F2E0FAA3E9A38BA09CA0A12CB12C64EFB5
:10CC200078E1C7010F94A275F70101900020E9F7A0
:10CC3000A9A1BAA14D905D906D907D90BAA3A9A3D2
:10CC4000AF014150510900E022EF38E1C301B201C8
:10CC50000E945D3EBC01C501820D931D68A779A7A6
:10CC60000F945E7940EF58E168A579A50E942A3DAE
:10CC7000B7018AE39DE00F9477616DED78E1C7011C
:10CC80000F94A275F70101900020E9F7AF01415020
:10CC900051092BED38E1C301B2010E945D3E9FA313
:10CCA0008EA3C4010F945E79BC0180E090E00F94E4
:10CCB000EF6D20E030E040E85BE30F94247029ED55
:10CCC00038E14EA15FA10E945D3EB7018AE39DE07D
:10CCD0000F94776167EC78E1C7010F94A275F701B3
:10CCE00001900020E9F7AF014150510925EC38E1EE
:10CCF000C301B2010E945D3E3C01C40102960F9443
:10CD00005179682F70E080E090E00F94EF6D20E0A3
:10CD100030E040E85EE30F94247023EC38E1A30197
:10CD20000E945D3EB7018AE39DE00F947761B2E017
:10CD3000AB0EB11CE3E08E0E911CFAE0AF16B1040D
:10CD400009F06DCF62EB78E1C7010F94A275F7018E
:10CD500001900020E9F731975F01AE18BF08C601C6
:10CD60000F945E79B7016A0D7B1D40EB58E10E947C
:10CD70002A3DB7018AE39DE00F94776165EA78E187
:10CD8000C7010F94A275F70101900020E9F73197D0
:10CD90005F01AE18BF08C60102960F945179B70122
:10CDA0006A0D7B1D43EA58E190E00E942A3DB701DD
:10CDB0008AE39DE00F9477616DE978E1C7010F94F4
:10CDC000A275F70101900020E9F731975F01AE18D5
:10CDD000BF08C60103960F945E79B7016A0D7B1DEB
:10CDE0004BE958E10E942A3DB7018AE39DE00F9488
:10CDF000776161E978E1C7010F94A275F7010190AD
:10CE00000020E9F731975F01AE18BF08C60105960B
:10CE10000F945979A7014A0D5B1D2FE838E10E9454
:10CE20005D3EB7018AE39DE00F9477611F5F88E163
:10CE3000C80ED11CABA1BCA1D096BCA3ABA3B0E2E1
:10CE40002B0E311C94CE8AE39DE00F945F621A8210
:10CE500019821C821B8288E99CE5282F9E838D8382
:10CE600088E8482F8F838FEF888719861A86CC240D
:10CE7000C394E12CFA8000E01C813E815FEF60E00A
:10CE800070E088ED98E00E94F1A0A9960FB6F894A2
:10CE9000DEBF0FBECDBFDF91CF911F910F91FF90ED
:10CEA000EF90DF90CF90BF90AF909F908F907F904A
:10CEB0006F905F904F903F902F900895CF92EF9298
:10CEC000FF920F931F93CF93DF93CDB7DEB72A97CF
:10CED0000FB6F894DEBF0FBECDBFE091110DF0E0AC
:10CEE000EE0FFF1FEF50F84E80819181892B09F4DE
:10CEF0006BC04091910388E0840F405E682F0E94D0
:10CF00005B330E94733299EBE92E9AE1F92E04E625
:10CF10001FE520E030E043EB5AE168E77FE586E576
:10CF20009FE30E94052D60EA7AE184E10E946C375C
:10CF30006BE87AE18EE10E946C370F94C141823038
:10CF4000A0F5C090110D84E0C89EF0011124E15FAE
:10CF5000F84E208131814281538160E070E080E0B1
:10CF60009FE30F94566D9B01AC016091360D70915B
:10CF7000370D8091380D9091390D0F94766C609338
:10CF8000360D7093370D8093380D9093390DE12C49
:10CF9000F12C00E81FE326E33DE042E35DE06EE2B2
:10CFA0007DE08AE29DE00F946F362A960FB6F894E2
:10CFB000DEBF0FBECDBFDF91CF911F910F91FF90CC
:10CFC000EF90CF900C9479320E94785F1A82198288
:10CFD0001C821B8289ED96E7282F9E838D8388E82B
:10CFE000482FCC24C394E12CFA8000E01C813E81C0
:10CFF0005FEF60E070E088ED98E00E94F1A02A9673
:10D000000FB6F894DEBF0FBECDBFDF91CF911F9159
:10D010000F91FF90EF90CF900895CF92EF92FF92F3
:10D020000F931F93CF93DF93CDB7DEB7AA970FB6B9
:10D03000F894DEBF0FBECDBF109285038E010F5F47
:10D040001F4F80E2F80111928A95E9F70E946C4B1C
:10D050006091120D7091130D8091140D9091150D2A
:10D060000F94BE6D7B0177FF02C0E12CF12C609123
:10D07000160D7091170D8091180D9091190D0F9448
:10D08000BE6D6B5F7F4F7F936F9360914A0270918B
:10D090004B0280914C0290914D020F94BE6D6E191F
:10D0A0007F0977FF02C06F5F7F4FCB019595879512
:10D0B000B701680F791F7F936F9360915A02709147
:10D0C0005B0280915C0290915D020F94BE6D7F9334
:10D0D0006F9386E09CE19F938F931F930F930F9420
:10D0E0007576C8010F94C51B1AA219A21CA21BA217
:10D0F0008DE799E5282F9EA38DA388E8482F8FA35D
:10D100008FEF88A7CC24C394E12CFAA000E01CA1E7
:10D110003EA15FEF60E070E088ED98E00E947FA1A3
:10D120000FB6F894DEBF0FBECDBFAA960FB6F89427
:10D13000DEBF0FBECDBFDF91CF911F910F91FF904A
:10D14000EF90CF9008952F923F924F925F926F92FF
:10D150007F928F929F92AF92BF92CF92DF92EF9287
:10D16000FF920F931F93CF93DF93CDB7DEB7C654D3
:10D17000D1090FB6F894DEBF0FBECDBF80917C0DF4
:10D1800085FD29C04091910388E0840F405E682F9F
:10D190000E945B330E94733284E090E090938C0392
:10D1A00080938B0340E050E066E57FE380E090E011
:10D1B0000E94552C60E67AE18FE00E946C376DE4A6
:10D1C0007AE189E10E946C370E9479328AE39DE01E
:10D1D0000F94485DDAC280FF04C08091F60E882368
:10D1E000A1F040E050E066E57FE380E090E00E943F
:10D1F000552C6DE37AE180E10E946C370E94793210
:10D200008AE39DE00F94575CC0C28AE39DE00F94CF
:10D210002E5D41E062ED72E08AE39DE00F94595D7E
:10D2200080911F0F81111BC084E090E090938C03CC
:10D2300080938B0340E050E066E57FE380E090E080
:10D240000E94552C6CE27AE18FE00E946C376DE110
:10D250007AE189E10E946C370E94793296C2E5E159
:10D26000FCE18491882341F09091C00095FFFCCFB0
:10D270008093C6003196F5CFE8E0FAE184918823E7
:10D2800041F09091C00095FFFCCF8093C60031968D
:10D29000F5CF8091C00085FFFCCF8AE08093C60067
:10D2A00081E080939907FE01B19680E2DF011D9233
:10D2B0008A95E9F7EE24EA94FE2E1F2FFE0131969F
:10D2C0005F0120E030E040E250E06F2D712F8CE1F3
:10D2D0009FE00F94BF23181619060CF01EC221966A
:10D2E0001FAE21976AE070E08F2D912F0F942A7660
:10D2F000009711F0DC011C926DEF79E18F2D912FD9
:10D300000F949975892B11F4E394DBCFBFE0BE1520
:10D31000C0F26DE370E08F2D912F0F942A76009765
:10D3200081F26C01EFEFCE1ADE0ADC011C9268EF8D
:10D3300079E18F2D912F0F949975892B09F05DC09C
:10D34000B8E1EB9EB00111246F5F774F48E050E0E9
:10D35000C6010F946379E5E1FCE18491882341F0F3
:10D360009091C00095FFFCCF8093C6003196F5CF19
:10D37000E7EEF9E18491882341F09091C00095FF98
:10D38000FCCF8093C6003196F5CFF60181918823BA
:10D3900039F09091C00095FFFCCF8093C600F6CF86
:10D3A0008091C00085FFFCCF8AE08093C600F0E347
:10D3B000EF9E400111242FED32E025963FAF2EAFB6
:10D3C00025978E2D90E0805B9F4FDC0195E0AA0FA2
:10D3D000BB1F9A95E1F72796BFAFAEAF2797F40131
:10D3E000E05BF34F2396FFAFEEAF239794012E5AE5
:10D3F000334F4901612C712C37C16BED79E18F2DD1
:10D40000912F0F949975892BE1F461E070E0C601CA
:10D410000E949E609C01215031092B33314040F025
:10D420008F2D912F0E944F591092990782ED90E015
:10D43000A8E1EA9E90011124BC01C901875F974FC2
:10D440007BC06BEC79E18F2D912F0F949975892B0F
:10D45000C9F461E070E0C6010E949E60893C9105BC
:10D4600040F08F2D912F0E944F59109299078CE315
:10D4700090E0B8E1EB9E90011124BC01C901855FE9
:10D48000974F5AC061EC79E18F2D912F0F949975C8
:10D49000892B11F561E070E0C6010E949E608F3F0C
:10D4A000910540F08F2D912F0E944F5910929907AE
:10D4B00084E607C061E070E0C6010E949E60853688
:10D4C00088F7E8E1EE9E90011124682FC901835F7F
:10D4D000974F0F946C796BCF6CEB79E18F2D912F77
:10D4E0000F949975892B59F561E070E0C6010E948F
:10D4F0009E609C0121503109283E3340A8F0EBE1A9
:10D50000FCE18491882341F09091C00095FFFCCF0D
:10D510008093C6003196F5CF8F2D912F0E944F59E1
:10D520001092990784E690E0F8E1EF9E90011124B3
:10D53000BC01C901825F974F0F947F7938CF63EBAD
:10D5400079E18F2D912F0F949975892B09F02FCFA9
:10D5500060E070E0C6010F94C8722B013C012DEC15
:10D560003CEC4CEC5DE30F944F6D87FD00C120E077
:10D5700030E040E251E4C301B2010F94526F18163B
:10D580000CF4F5C028E1E29EC0011124B301A20110
:10D59000805F974F0F947A790ACF61E070E0C601FF
:10D5A0000E949E609C01215031092B33314040F094
:10D5B0008F2D912F0E944F591092990782ED90E084
:10D5C000BC0127968EAD9FAD2797860D971D0F94B2
:10D5D0007F7963E979E1C5010F94A275F5010190A6
:10D5E0000020E9F7AF014150510900E020E030E0B0
:10D5F000C201B1010E945D3EB5018F2D912F0F94A4
:10D600003576892B09F458C061E879E1C5010F949A
:10D61000A275F50101900020E9F7AF0141505109D1
:10D6200000E020E030E0C201B1010E945D3EB501A2
:10D630008F2D912F0F943576892B09F456C0F3E086
:10D640008F0E911C23962EAD3FAD23972D5F3F4F3C
:10D6500023963FAF2EAF239732E0630E711C4AE052
:10D660006416710409F42DCE66EA79E1C5010F94C0
:10D67000A275F50101900020E9F72596AEADBFAD8A
:10D6800025972D903D904D905D902596BFAFAEAF04
:10D690002597AF014150510900E020E030E0C20180
:10D6A000B1010E945D3EB5018F2D912F0F9435760B
:10D6B000892B09F08ECF71CF60E071E0C6010E9426
:10D6C0009E608130E4E19E0740F08F2D912F0E94F3
:10D6D0004F591092990780E896E0BC0123968EADD1
:10D6E0009FAD23970F947F798FCF64E070E0C601E0
:10D6F0000E949E609C0121503109243B310540F07D
:10D700008F2D912F0E944F591092990784E690E037
:10D71000682FC4010F946C7992CF61E06E0D21F0F7
:10D7200080E098E00F946C798AE39DE00F945F624B
:10D730001A8219821C821B828EE79CE5282F9E8309
:10D740008D8388E8482F8F838FEF888719861A8604
:10D75000CC24C394E12CFA8000E01C813E815FEF71
:10D7600060E070E088ED98E00E94F1A00EC08F2D7F
:10D77000912F0E944F591092990786E6482E542CFB
:10D7800086E3682E80E4782EFDCECA5BDF4F0FB6AD
:10D79000F894DEBF0FBECDBFDF91CF911F910F91E7
:10D7A000FF90EF90DF90CF90BF90AF909F908F90C1
:10D7B0007F906F905F904F903F902F9008958111D0
:10D7C00001C02BCC0895CF92EF92FF920F931F933D
:10D7D000CF93DF93CDB7DEB72A970FB6F894DEBFAD
:10D7E0000FBECDBF45EF5BE16CEE7BE185EE9BE1CB
:10D7F0000E94B02B80918A03882341F180918B0392
:10D8000090918C0307960F9780F50E94ECF581119B
:10D810002CC003DC1A8219821C821B828AE899E5DB
:10D82000282F9E838D8388E8482FCC24C394E12C35
:10D83000FA8000E01C813E815FEF34C0409708977A
:10D8400028F461E088ED98E00E94D2A12A960FB6F4
:10D85000F894DEBF0FBECDBFDF91CF911F910F9126
:10D86000FF90EF90CF900C94793280918B03909140
:10D870008C039C012850310928303105F8F61A82B2
:10D8800019821C821B828EE297E7282F9E838D834C
:10D8900082E0482FCC24C394E12CFA8000E01C8164
:10D8A0003E8150E060E070E088ED98E00E947FA14A
:10D8B000CDCF8F929F92AF92BF92CF92DF92EF9295
:10D8C000FF920F931F93CF93DF93CDB7DEB72997C6
:10D8D0000FB6F894DEBF0FBECDBFE5E1FCE1849149
:10D8E000882341F09091C00095FFFCCF8093C60043
:10D8F0003196F5CFE8ECF6E18491882341F09091E0
:10D90000C00095FFFCCF8093C6003196F5CF809183
:10D91000C00085FFFCCF8AE08093C6008E010F5FB8
:10D920001F4F89E0F80111928A95E9F764EC76E1DE
:10D93000C8010F94A27544E050E061E078E0C801AE
:10D940000F94637962ED70E089E098E00F947F793D
:10D950006CE370E08BE098E00F947F7964E68DE0F3
:10D9600098E00F946C7964E670E08EE098E00F9494
:10D970007F7946E656E666E370E480E198E00F942E
:10D980007A7962ED70E080E09AE00F947F7963EC41
:10D9900070E082E09AE00F947F7966EE70E084E0B8
:10D9A0009AE00F947F7960EF70E086E09AE00F9440
:10D9B0007F7960EF70E088E09AE00F947F7960E80B
:10D9C00076E080E59CE00F947F7960E876E083E57F
:10D9D0009CE00F947F7960E876E086E59CE00F9408
:10D9E0007F7960E876E089E59CE00F947F7960E8D4
:10D9F00076E08CE59CE00F947F7964E682E59CE01C
:10DA00000F946C7964E685E59CE00F946C7964E68C
:10DA100088E59CE00F946C7964E68BE59CE00F94BC
:10DA20006C7964E68EE59CE00F946C7960EC76E1AD
:10DA3000C8010F94A27544E050E069E178E0C801A4
:10DA40000F94637964E071E081E298E00F947F794C
:10DA50006AE570E083E298E00F947F7964E685E2FE
:10DA600098E00F946C796BE670E086E298E00F9492
:10DA70007F7946E656E666E370E488E298E00F9424
:10DA80007A796FEF70E080E29AE00F947F7965EF2A
:10DA900070E082E29AE00F947F7964E071E084E2C2
:10DAA0009AE00F947F7964E071E086E29AE00F9447
:10DAB0007F7964E071E088E29AE00F947F7960E812
:10DAC00076E080E89CE00F947F7960E876E083E878
:10DAD0009CE00F947F7960E876E086E89CE00F9404
:10DAE0007F7960E876E089E89CE00F947F7960E8D0
:10DAF00076E08CE89CE00F947F7964E682E89CE015
:10DB00000F946C7964E685E89CE00F946C7964E688
:10DB100088E89CE00F946C7964E68BE89CE00F94B5
:10DB20006C7964E68EE89CE00F946C796CEB76E19E
:10DB3000C8010F94A27544E050E061E378E0C801A9
:10DB40000F9463796FEF70E089E398E00F947F7929
:10DB50006CE370E08BE398E00F947F7962E38DE3F0
:10DB600098E00F946C7964E670E08EE398E00F948F
:10DB70007F7946E656E666E370E480E498E00F9429
:10DB80007A796FEF70E080E49AE00F947F7965EF27
:10DB900070E082E49AE00F947F7964E071E084E4BD
:10DBA0009AE00F947F7964E071E086E49AE00F9444
:10DBB0007F7964E071E088E49AE00F947F7960E80F
:10DBC00076E080EB9CE00F947F7960E876E083EB71
:10DBD0009CE00F947F7960E876E086EB9CE00F9400
:10DBE0007F7960E876E089EB9CE00F947F7960E8CC
:10DBF00076E08CEB9CE00F947F7964E682EB9CE00E
:10DC00000F946C7964E685EB9CE00F946C7964E684
:10DC100088EB9CE00F946C7964E68BEB9CE00F94AE
:10DC20006C7964E68EEB9CE00F946C7969EB76E19D
:10DC3000C8010F94A27543E050E069E478E0C801A0
:10DC40000F94637964E071E081E598E00F947F7947
:10DC50006EE670E083E598E00F947F7964E685E5F1
:10DC600098E00F946C7964E670E086E598E00F9494
:10DC70007F7946E656E666E370E488E598E00F941F
:10DC80007A7964E071E080E69AE00F947F7964E04D
:10DC900071E082E69AE00F947F7964E071E084E6B7
:10DCA0009AE00F947F7964E071E086E69AE00F9441
:10DCB0007F7964E071E088E69AE00F947F7960E80C
:10DCC00076E080EE9CE00F947F7960E876E083EE6A
:10DCD0009CE00F947F7960E876E086EE9CE00F94FC
:10DCE0007F7960E876E089EE9CE00F947F7960E8C8
:10DCF00076E08CEE9CE00F947F7964E682EE9CE007
:10DD00000F946C7964E685EE9CE00F946C7964E680
:10DD100088EE9CE00F946C7964E68BEE9CE00F94A7
:10DD20006C7964E68EEE9CE00F946C7963EB76E19F
:10DD3000C8010F94A27546E050E061E678E0C801A2
:10DD40000F9463796AEF70E089E698E00F947F7929
:10DD50006CE370E08BE698E00F947F7964E68DE6E3
:10DD600098E00F946C7964E670E08EE698E00F948A
:10DD70007F7946E656E666E370E480E798E00F9424
:10DD80007A796AEF70E080E89AE00F947F7960EF2B
:10DD900070E082E89AE00F947F796FEF70E084E89A
:10DDA0009AE00F947F7964E071E086E89AE00F943E
:10DDB0007F7964E071E088E89AE00F947F7960E809
:10DDC00076E080E19DE00F947F7960E876E083E182
:10DDD0009DE00F947F7960E876E086E19DE00F9406
:10DDE0007F7960E876E089E19DE00F947F7960E8D3
:10DDF00076E08CE19DE00F947F7964E682E19DE01E
:10DE00000F946C7964E685E19DE00F946C7964E68B
:10DE100088E19DE00F946C7964E68BE19DE00F94BE
:10DE20006C7964E68EE19DE00F946C796EEA76E1A0
:10DE3000C8010F94A27545E050E069E778E0C80199
:10DE40000F94637964E071E081E898E00F947F7942
:10DE50006EE670E083E898E00F947F7964E685E8E9
:10DE600098E00F946C7964E670E086E898E00F948F
:10DE70007F7946E656E666E370E488E898E00F941A
:10DE80007A7964E071E080EA9AE00F947F7964E047
:10DE900071E082EA9AE00F947F7964E071E084EAAD
:10DEA0009AE00F947F7964E071E086EA9AE00F943B
:10DEB0007F7964E071E088EA9AE00F947F7960E806
:10DEC00076E080E49DE00F947F7960E876E083E47B
:10DED0009DE00F947F7960E876E086E49DE00F9402
:10DEE0007F7960E876E089E49DE00F947F7960E8CF
:10DEF00076E08CE49DE00F947F7964E682E49DE017
:10DF00000F946C7964E685E49DE00F946C7964E687
:10DF100088E49DE00F946C7964E68BE49DE00F94B7
:10DF20006C7964E68EE49DE00F946C7966EA76E1A4
:10DF3000C8010F94A27548E050E061E978E0C8019B
:10DF40000F9463796BEE70E089E998E00F947F7924
:10DF500066E470E08BE998E00F947F7964E68DE9E0
:10DF600098E00F946C7964E670E08EE998E00F9485
:10DF70007F7946E656E666E370E480EA98E00F941F
:10DF80007A796BEE70E080EC9AE00F947F796BEE1B
:10DF900070E082EC9AE00F947F796BEE70E084EC95
:10DFA0009AE00F947F796BEE70E086EC9AE00F9424
:10DFB0007F796BEE70E088EC9AE00F947F7960E0F7
:10DFC0007AE080E79DE00F947F7960E07AE083E774
:10DFD0009DE00F947F7960E07AE086E79DE00F9402
:10DFE0007F7960E07AE089E79DE00F947F7960E0D7
:10DFF0007AE08CE79DE00F947F7964E682E79DE00C
:10E000000F946C7964E685E79DE00F946C7964E683
:10E0100088E79DE00F946C7964E68BE79DE00F94B0
:10E020006C7964E68EE79DE00F946C7963EA76E1A3
:10E03000C8010F94A27543E050E069EA78E0C80196
:10E040000F9463796CED70E081EB98E00F947F7929
:10E0500064E670E083EB98E00F947F7964E685EBEB
:10E0600098E00F946C7964E670E086EB98E00F948A
:10E070007F7946E656E666E370E488EB98E00F9415
:10E080007A796CED70E080EE9AE00F947F796CED18
:10E0900070E082EE9AE00F947F7966EE70E084EE95
:10E0A0009AE00F947F7960EF70E086EE9AE00F942B
:10E0B0007F7960EF70E088EE9AE00F947F7960E0FE
:10E0C00078E080EA9DE00F947F7960E078E083EA71
:10E0D0009DE00F947F7960E078E086EA9DE00F9400
:10E0E0007F7960E078E089EA9DE00F947F7960E0D5
:10E0F00078E08CEA9DE00F947F7964E682EA9DE007
:10E100000F946C7964E685EA9DE00F946C7964E67F
:10E1100088EA9DE00F946C7964E68BEA9DE00F94A9
:10E120006C7964E68EEA9DE00F946C796EE976E195
:10E13000C8010F94A27545E050E061EC78E0C80199
:10E140000F9463796DEC70E089EC98E00F947F791F
:10E1500062E370E08BEC98E00F947F7964E68DECDD
:10E1600098E00F946C7964E670E08EEC98E00F9480
:10E170007F7946E656E666E370E480ED98E00F941A
:10E180007A796DEC70E080E09BE00F947F7963EC2E
:10E1900070E082E09BE00F947F7962ED70E084E0B4
:10E1A0009BE00F947F7962ED70E086E09BE00F9436
:10E1B0007F7967ED70E088E09BE00F947F7960E8FD
:10E1C00076E080ED9DE00F947F7960E876E083ED66
:10E1D0009DE00F947F7960E876E086ED9DE00F94F6
:10E1E0007F7960E876E089ED9DE00F947F7960E8C3
:10E1F00076E08CED9DE00F947F7964E682ED9DE002
:10E200000F946C7964E685ED9DE00F946C7964E67B
:10E2100088ED9DE00F946C7964E68BED9DE00F94A2
:10E220006C7964E68EED9DE00F946C7969E080E096
:10E2300098E00F946C79A12C8AE0B82E9FE5C92E46
:10E240009CE0D92E760100E010E045018AE0880EBE
:10E25000911C60E070E0C401800F911F0F947F79E2
:10E2600060E070E0C7010F947F7960E0C70102961B
:10E270000F946C790E5F1F4FF3E0EF0EF11C063127
:10E28000110539F780E3C80ED11CE0E2AE0EB11CD7
:10E29000FFE0CF16FEE0DF06A9F629960FB6F89448
:10E2A000DEBF0FBECDBFDF91CF911F910F91FF90C9
:10E2B000EF90DF90CF90BF90AF909F908F90089598
:10E2C000CF92DF92EF92FF920F931F93CF93DF9342
:10E2D000C82F88E1C89F80011124E091110DD4E47A
:10E2E000DE9FF0011124E656F84F60817181C8016C
:10E2F000875F974F0F947F79E091110DDE9FF001BA
:10E300001124E656F84F62A973A9C801855F974F9B
:10E310000F947F79E091110DDE9FF0011124E656F4
:10E32000F84F65A976A9C801825F974F0F947F794E
:10E33000E091110DDE9FF0011124E656F84F64A91B
:10E34000C801835F974F0F946C79E091110DDE9FA8
:10E35000F0011124E656F84F47A950AD61AD72ADFA
:10E36000C801805F974F0F947A79EC2EF12C80E5ED
:10E37000E80EF11C54E0EE0CFF1C5A95E1F780E327
:10E38000C89FE0011124C05BD34F00E010E062E2BF
:10E39000C62E71E1D72E8091110DF801C89EE00DB7
:10E3A000F11D1124EE0FFF1FE656F84F60817181B9
:10E3B000C8018E0D9F1D880F991F0F947F79809142
:10E3C000110DF801D89EE00DF11D1124EE0FFF1F75
:10E3D000EE0FFF1FE656F84F20E030E040E853E430
:10E3E00062857385848595850F9424700F94C36D21
:10E3F000CE010F947F798091110DF801D89EE00D28
:10E40000F11D1124EE0FFF1FEE0FFF1FE656F84F10
:10E4100020E030E040E752E4668D778D80A191A145
:10E420000F94566D20E030E040E850E40F942470E3
:10E430000F94C36DCE0102960F946C790F5F1F4F3E
:10E4400023960530110509F0A6CFDF91CF911F91DA
:10E450000F91FF90EF90DF90CF900895EF92FF9291
:10E460000F931F93CF93DF93CDB7DEB729970FB6E6
:10E47000F894DEBF0FBECDBF80E098E00F945179D5
:10E48000182F803109F41FE02CE739E54CE55EE5F3
:10E4900062E0610F88E098E10E94452F80918A0335
:10E4A000882309F450C060918B0370918C03CB01D9
:10E4B00003968730910508F441C077FDBC017B01CC
:10E4C000F594E794F594E7940FEF0E0D011334C023
:10E4D00087E0E9E9F2E0DE01119601900D928A955C
:10E4E000E1F719861886812F90E040E050E0BE01E8
:10E4F000695F7F4F01960E942A3D2091110D34E4FF
:10E50000239FC0011124BE016F5F7F4F8B52984F34
:10E510000F943E7688E1189F90011124B9016F5F36
:10E52000774F48E050E0CE0101960F9463796E2D4D
:10E5300080E098E00F946C79802FC2DE61E088ED76
:10E5400098E00E94D2A10E94793229960FB6F894E1
:10E55000DEBF0FBECDBFDF91CF911F910F91FF9016
:10E56000EF900895CF92DF92EF92FF920F931F9357
:10E57000CF93DF9389E899E00F945E7990939B079E
:10E5800080939A078C3221E092071CF46BE371E0D0
:10E590000AC09C012C533140243C3E4708F484C0FF
:10E5A000BC01615F7F4F80E00F94A8598BE899E030
:10E5B0000F945E799093CD078093CC078EE899E015
:10E5C0000F945E799093D0078093CF078DE899E000
:10E5D0000F9451798093CE0780E999E00F9459798F
:10E5E0006093D1077093D2078093D3079093D40799
:10E5F0008AE9C82E87E0D82E94EAE92E97E0F92E12
:10E6000000E51FE0C0E0DCE0CE010F945E79F6018A
:10E61000819391936F01C8010F945E79BC0180E0F2
:10E6200090E00F94EF6D20E030E040E85BE30F9462
:10E630002470F70161937193819391937F01C801D5
:10E6400002960F945179682F70E080E090E00F946B
:10E65000EF6D20E030E040E85EE30F94247020E0AE
:10E6600030E040E752E40F942470F701608B718B27
:10E67000828B938B22960D5F1F4FCA30FCE0DF0721
:10E6800019F648E050E061E879E085ED97E00F94F5
:10E6900041791092DD07DF91CF911F910F91FF908B
:10E6A000EF90DF90CF9008956AE471E07CCFCF9235
:10E6B000DF92EF92FF920F931F93CF93DF936091BE
:10E6C0009A0770919B0789E899E00F947F79609190
:10E6D0009A0770919B076C3281E078071CF46BE31A
:10E6E00071E007C06C3381E078070CF079C0615F9E
:10E6F0007F4F80E00F94A8596091CC077091CD07AF
:10E700008BE899E00F947F796091CE078DE899E0CE
:10E710000F946C796091CF077091D0078EE899E0E3
:10E720000F947F794091D1075091D2076091D30720
:10E730007091D40780E999E00F947A798AE9C82E1C
:10E7400087E0D82E94EAE92E97E0F92E00E51FE045
:10E75000C0E0DCE0F601619171916F01CE010F9490
:10E760007F79F70161917191819191917F0120E011
:10E7700030E040E853E40F9424700F94C36DC80157
:10E780000F947F7920E030E040E752E4F7016089A0
:10E790007189828993890F94566D20E030E040E8BA
:10E7A00050E40F9424700F94C36DC80102960F9427
:10E7B0006C7922960D5F1F4FCA30FCE0DF0751F6DF
:10E7C00048E050E061E879E085ED97E0DF91CF9196
:10E7D0001F910F91FF90EF90DF90CF900D94637990
:10E7E0006AE471E086CFCF92EF92FF920F931F936E
:10E7F000CF93DF93CDB7DEB72A970FB6F894DEBF7D
:10E800000FBECDBF28E331E64EEA5EE567E084E562
:10E8100098E10E94452F80918A03882309F49CC1C6
:10E8200080918B0390918C039C012D5F3F4F27308B
:10E83000310538F461E088ED98E00E94D2A137DF1D
:10E840008BC19C01245031092430310538F41A82DF
:10E8500019821C821B8280EF9CE56BC19C012850B1
:10E8600031092430310508F04CC01A8219821C820B
:10E870001B828CE290E3282F9E838D8388E8482FAB
:10E880008F838FEF8887CC24C394E12CFA8000E03B
:10E890001C813E815FEF60E070E088ED98E00E94AF
:10E8A0007FA183E498E1909384038093830381E4C0
:10E8B00098E190938203809381038091110D24E469
:10E8C000829FC00111249C012453384F3093800350
:10E8D00020937F0322E020937E03FC01E656F84F4D
:10E8E00082A993A990938C0380938B0390937903CF
:10E8F0008093780310927D0310927C0389EB90E063
:10E900000AC19C012C5031092430310508F05CC04B
:10E910001A8219821C821B828CE290E3282F9E832C
:10E920008D8388E8482F8F838FEF8887CC24C3940A
:10E93000E12CFA8000E01C813E815FEF60E070E036
:10E9400088ED98E00E947FA18FE298E19093840384
:10E95000809383038CE298E19093820380938103F8
:10E960008091110D24E4829FC00111249C012F523B
:10E97000384F3093800320937F0323E020937E035E
:10E98000FC01E656F84F20E030E048EC52E467A97D
:10E9900070AD81AD92AD0F94247020E030E040E086
:10E9A0005FE30F94766C0F94BE6D70938C0360934D
:10E9B0008B03709379036093780310927D03109218
:10E9C0007C0380E197E2A7C09C01205131092430EB
:10E9D000310508F04CC01A8219821C821B828CE21D
:10E9E00090E3282F9E838D8388E8482F8F838FEFB5
:10E9F0008887CC24C394E12CFA8000E01C813E81FE
:10EA00005FEF60E070E088ED98E00E947FA182E215
:10EA100098E1909384038093830380E298E190933C
:10EA20008203809381038091110D24E4829FC001B1
:10EA300011249C012253384F3093800320937F038D
:10EA400021E020937E03FC01E656F84F84A990E074
:10EA500090938C0380938B03909379038093780336
:10EA600010927D0310927C0384E690E054C09C01D8
:10EA7000245131092430310508F052C01A8219821C
:10EA80001C821B828CE290E3282F9E838D8388E872
:10EA9000482F8F838FEF8887CC24C394E12CFA8092
:10EAA00000E01C813E815FEF60E070E088ED98E05F
:10EAB0000E947FA182E198E1909384038093830375
:10EAC00080E198E190938203809381038091110DFE
:10EAD00024E4829FC00111249C012153384F3093BC
:10EAE000800320937F0322E020937E03FC01E656FF
:10EAF000F84F85A996A990938C0380938B039093EC
:10EB000079038093780381E090E090937D03809374
:10EB10007C0388EE93E090937B0380937A031CC080
:10EB200048970497C8F41A8219821C821B828EE2CD
:10EB300092E7282F9E838D8388E8482FCC24C394A6
:10EB4000E12CFA8000E01C813E815FEF60E070E024
:10EB500088ED98E00E947FA12A960FB6F894DEBF58
:10EB60000FBECDBFDF91CF911F910F91FF90EF901E
:10EB7000CF900C9479325F926F927F928F929F9296
:10EB8000AF92BF92CF92DF92EF92FF920F931F93BB
:10EB9000CF93DF93B82E562E062F10E0682E712CDF
:10EBA00028E1829F70011124C701875F974F0F945E
:10EBB0005E79BC0184E4809FF001819FF00D1124F7
:10EBC000E656F84F718360836C3241E074071CF4A1
:10EBD0006BE371E009C0CB018C539140843C9E47AC
:10EBE00008F4E4C0615F7F4F852D0F94A859C701D9
:10EBF000855F974F0F945E798A3B91054CF424E42E
:10EC0000209FF001219FF00D1124E656F84F0AC015
:10EC100084E4809FF001819FF00D1124E656F84FA7
:10EC200089EB90E093AB82ABC701825F974F0F9463
:10EC30005E7924E4209F6001219FD00C1124E6011D
:10EC4000C656D84F9EAB8DABC701835F974F0F94CD
:10EC500051798CABC701805F974F0F9459796FAB97
:10EC600078AF89AF9AAFC6018B52984F6C01B7014C
:10EC70006F5F774F48E050E00F944179CD5BDF4FF5
:10EC80001882B60189EE97E00F943E7690E3B99E24
:10EC9000E0011124C05BD34FE4E45E9E40011124E7
:10ECA000A4014C55584F5A0150E5650E711C85E082
:10ECB000660C771C8A95E1F7E12CF12CC701860DD3
:10ECC000971D0F945E799701280D391DF901E656BD
:10ECD000F84F6F0191838083852D0F94E9590E972A
:10ECE000F60120813181281739073CF0852D0F94DA
:10ECF000E9590F97F60191838083CE010F945E79D5
:10ED0000BC0180E090E00F94EF6D20E030E040E83F
:10ED10005BE30F942470F501619371938193919358
:10ED20005F01CE0102960F945179682F70E080E068
:10ED300090E00F94EF6D20E030E040E85EE30F9448
:10ED4000247020E030E040E752E40F942470F50195
:10ED5000608B718B828B938BF2E0EF0EF11C23960C
:10ED60002AE0E216F10409F0A9CF84E4809FF001C3
:10ED7000819FF00D1124E656F84F82A993A98A3B92
:10ED8000910524F089EB90E093AB82ABDF91CF91BA
:10ED90001F910F91FF90EF90DF90CF90BF90AF90B9
:10EDA0009F908F907F906F905F9081CC6AE471E02C
:10EDB0001BCFCF92EF92FF920F931F93CF93DF93CE
:10EDC000CDB7DEB72A970FB6F894DEBF0FBECDBF22
:10EDD00080E098E00F94517924E93DE54EE25EE54C
:10EDE000682F89E79BE10E94452F80918A03882341
:10EDF00031F180918B0390918C0397FD039695954B
:10EE00008795959587956091110DB5DE1A821982C7
:10EE10001C821B8286E59BE5282F9E838D8384E0E0
:10EE2000482FCC24C394E12CFA8000E01C813E8161
:10EE300050E060E070E088ED98E00E94F1A02A9632
:10EE40000FB6F894DEBF0FBECDBFDF91CF911F91FB
:10EE50000F91FF90EF90CF900C947932CF92EF9278
:10EE6000FF920F931F93CF93DF93CDB7DEB72A970F
:10EE70000FB6F894DEBF0FBECDBF80E098E00F94D0
:10EE80005179182F64E0680F21E332E640E05FE536
:10EE900082E89AE10E94452F80918A03882309F431
:10EEA0006EC080918B0390918C03AC014D5F5F4FDE
:10EEB0004730510530F461E088ED98E00E94D2A11E
:10EEC0005EC0212F30E097FDCA01959587959595F5
:10EED0008795A9014F5F5F4F4817590739F41A8288
:10EEE00019821C821B8283EF93E70CC0A9014E5F3D
:10EEF0005F4F48175907D1F41A8219821C821B826E
:10EF000087E395E6282F9E838D8388E8482FCC24BD
:10EF1000C394E12CFA8000E01C813E815FEF60E049
:10EF200070E088ED98E00E947FA129C02D5F3F4FDF
:10EF30002817390739F41A8219821C821B8283EA46
:10EF400098E6E0CF6091110D815015DE1A8219828A
:10EF50001C821B828AE890E6282F9E838D8384E0A2
:10EF6000482FCC24C394E12CFA8000E01C813E8120
:10EF700050E060E070E088ED98E00E94F1A02A96F1
:10EF80000FB6F894DEBF0FBECDBFDF91CF911F91BA
:10EF90000F91FF90EF90CF900C9479328F929F92C7
:10EFA000AF92BF92CF92DF92EF92FF920F931F9397
:10EFB000CF9380E098E00F945179C82F8EEF8C0F9B
:10EFC0008F3008F07AC0C150EC2EF12C28E1C29F9E
:10EFD00080011124C801875F974F0F945E790197D4
:10EFE0008B33914008F069C0C801855F974F0F943B
:10EFF0005E79893C910508F060C0C801835F974F36
:10F000000F945179853608F058C0C801825F974F38
:10F010000F945E790197883E934008F04EC0C80176
:10F02000805F974F0F9459794B015C012DEC3CECBC
:10F030004CEC5DE30F944F6D87FD3FC020E030E066
:10F0400040E251E4C501B4010F94526F1816ACF1BF
:10F0500080E3C89F800111240E5A134F20E5E20E71
:10F06000F11C85E0EE0CFF1C8A95E1F7C12CD12C38
:10F07000C6018E0D9F1D0F945E7901978B339140D1
:10F08000E0F4C80102970F945E7981309441A8F4AE
:10F09000C8010F94517990E00197843B910568F481
:10F0A00082E0C80ED11C0D5F1F4F2AE0C216D104AA
:10F0B000F9F6C11188CF81E001C080E0CF911F91A6
:10F0C0000F91FF90EF90DF90CF90BF90AF909F9007
:10F0D0008F900895CF92DF92EF92FF926B017C01A7
:10F0E00020E030E040E85EE30F94756C9F772DECF4
:10F0F0003CEC4CE45DE30F944F6D87FD37C02AE98B
:10F1000039E949E15FE3C701B6010F94756C9F7758
:10F110002DEC3CEC4CEC5DE30F944F6D87FD28C06B
:10F120002DEC3CEC4CE45FE3C701B6010F94756C29
:10F130009F772DEC3CEC4CEC5DE30F944F6D87FD1D
:10F1400019C020E030E040E85FE3C701B6010F944A
:10F15000756C9F772DEC3CEC4CEC5DE30F944F6DA0
:10F16000881F8827881F880F880F05C081E003C08B
:10F1700082E001C083E0FF90EF90DF90CF90089590
:10F1800060E088ED98E00C94A6A50E94492B61E010
:10F1900088ED98E00C941BA28FEF8093F30C1092F3
:10F1A00087031092860380914B098D7F80934B09D2
:10F1B00080917C0D83FF02C084FF05C061E088ED73
:10F1C00098E00C941BA281E08093E207F7CFCF92E6
:10F1D000EF92FF920F931F93CF93DF93CDB7DEB7DC
:10F1E0002A970FB6F894DEBF0FBECDBF1A821982E0
:10F1F0001C821B8289EF9BE7282F9E838D8388E8E2
:10F20000482FCC24C394E12CFA8000E01C813E817D
:10F210005FEF60E070E088ED98E00E947FA12A96A1
:10F220000FB6F894DEBF0FBECDBFDF91CF911F9117
:10F230000F91FF90EF90CF900895CF92EF92FF92B1
:10F240000F931F93CF93DF93CDB7DEB72A970FB6F7
:10F25000F894DEBF0FBECDBF1A8219821C821B82BA
:10F2600089E29FE7282F9E838D838CE0482FCC2452
:10F27000C394E12CFA8000E01C813E8150E060E004
:10F2800070E088ED98E00E947FA12A960FB6F8946E
:10F29000DEBF0FBECDBFDF91CF911F910F91FF90C9
:10F2A000EF90CF9008958091910360E8681B482FFC
:10F2B0000E945B330E94733249E151E26BE57FE3C8
:10F2C00080E090E00E94552C6DE071E28AE00E949F
:10F2D0006C376CEF70E284E10E946C3765EF70E28E
:10F2E0008EE10E946C3762EE70E288E20E946C3719
:10F2F0000C9479328091910360E8681B482F0E943A
:10F300005B330E94733243ED50E26BE57FE380E0B4
:10F3100090E00E94552C6CEC70E28FE00E946C37FC
:10F3200069EB70E289E10E946C3768EA70E283E27F
:10F330000E946C370C947932EF92FF920F93CF9327
:10F34000DF93CDB7DEB7A0970FB6F894DEBF0FBE40
:10F35000CDBF9E012F5F3F4F790190E2F9011192DD
:10F360009A95E9F7813061F4609145027091460207
:10F37000809147029091480200E026E73DE12DC0D0
:10F380008230F1F420E030E040E752E46091410245
:10F390007091420280914302909144020F94566D05
:10F3A00020E030E040E05FE30F94766C0F94BE6D98
:10F3B000DC01CB014FE65DE1B7010E942A3D10C0A0
:10F3C000833099F460912D0270912E0280912F026A
:10F3D0009091300200E02CE63DE1A7010E945D3EE5
:10F3E000A70166E385E00E946233A0960FB6F89409
:10F3F000DEBF0FBECDBFDF91CF910F91FF90EF9099
:10F4000008950F931F93CF93DF93CDB7DEB7A097E7
:10F410000FB6F894DEBF0FBECDBF8E010F5F1F4F3A
:10F4200090E2F80111929A95E9F7813041F44CE2AB
:10F430005DE1B801809158029091590259C0823023
:10F44000C9F460911E0270911F0280912002909178
:10F4500021020F94BE6DDC01CB0147E25DE1B801F2
:10F460000E942A3D4AE25DE1BC018091F117909132
:10F47000F2173EC08330C9F460911A0270911B02EA
:10F4800080911C0290911D020F94BE6DDC01CB0196
:10F4900042E25DE1B8010E942A3D45E25DE1BC0126
:10F4A0008091E9179091EA1723C0843079F4809114
:10F4B0000F0DF4E68F9FC00111246FEF70E00F94E1
:10F4C0001D71CB0140E25DE1B80112C0853041F40D
:10F4D0004EE15DE1B801809156029091570208C05B
:10F4E000873069F4809122024CE15DE1B80190E03F
:10F4F0000E942A3DA80166E384E00E946233A09640
:10F500000FB6F894DEBF0FBECDBFDF91CF911F9134
:10F510000F91089580914B098D7F80934B098091C5
:10F520007003833029F460E070E088E00E946B256E
:10F5300061E088ED98E00C94D2A18AE39DE00D94FF
:10F540006663CF92EF92FF920F931F93CF93DF9357
:10F55000CDB7DEB72A970FB6F894DEBF0FBECDBF8A
:10F560002CE939E747EB5DE764E088EB9DE10E9419
:10F57000452F80918A03882309F42CC180918B0345
:10F5800090918C039C012D5F3F4F2730310530F463
:10F5900061E088ED98E00E94D2A11CC19C0124503A
:10F5A000310924303105F0F51A8219821C821B8240
:10F5B0008CE290E3282F9E838D8388E8482F8F83E9
:10F5C0008FEF8887CC24C394E12CFA8000E01C8163
:10F5D0003E815FEF60E070E088ED98E00E947FA1DF
:10F5E00089EA9DE1909384038093830386EA9DE1F9
:10F5F000909382038093810385E492E0909380034B
:10F6000080937F0383E080937E0320E030E048EC2A
:10F6100052E46091450270914602809147029091B8
:10F620004802BCC09C01285031092430310508F043
:10F6300074C01A8219821C821B828CE290E3282FEC
:10F640009E838D8388E8482F8F838FEF8887CC2413
:10F65000C394E12CFA8000E01C813E815FEF60E002
:10F6600070E088ED98E00E947FA188E99DE1909389
:10F6700084038093830381E99DE1909382038093C7
:10F68000810381E492E09093800380937F0386E07E
:10F6900080937E0320E030E040E752E46091410235
:10F6A0007091420280914302909144020F94566DF2
:10F6B00020E030E040E05FE30F94766C0F94BE6D85
:10F6C00070938C0360938B0370937903609378033A
:10F6D00010927D0310927C0320E030E040E752E47A
:10F6E00060912F17709130178091311790913217D8
:10F6F0000F94247020E030E040E752E40F94566D00
:10F7000020E030E040E05FE30F94766C0F94BE6D34
:10F7100070937B0360937A035DC00C97049708F0A5
:10F7200059C01A8219821C821B828CE290E3282F16
:10F730009E838D8388E8482F8F838FEF8887CC2422
:10F74000C394E12CFA8000E01C813E815FEF60E011
:10F7500070E088ED98E00E947FA18CE79DE1909396
:10F7600084038093830389E79DE1909382038093D0
:10F7700081038DE292E09093800380937F0383E086
:10F7800080937E0320E030E048EC52E460912D024B
:10F7900070912E0280912F02909130020F9424706C
:10F7A00020E030E040E05FE30F94766C0F94BE6D94
:10F7B00070938C0360938B03709379036093780349
:10F7C00010927D0310927C0388E893E190937B0371
:10F7D00080937A032A960FB6F894DEBF0FBECDBF92
:10F7E000DF91CF911F910F91FF90EF90CF900C94EC
:10F7F0007932CF92EF92FF920F931F93CF93DF93C3
:10F80000CDB7DEB72A970FB6F894DEBF0FBECDBFD7
:10F810008091330280FF07C080917C0D8871883110
:10F8200021F069E003C068E001C06AE021E03AE746
:10F830004AEF5DE78AEF9DE10E94452F80918A03A0
:10F84000882309F471C180918B0390918C0397FDFB
:10F8500003969595879595958795009731F461E086
:10F8600088ED98E00E94D2A15FC18130910599F5A1
:10F870001A8219821C821B828CE290E3282F9E83BD
:10F880008D8388E8482FCC24C394E12CFA8000E0D3
:10F890001C813E815FEF60E070E088ED98E00E949F
:10F8A0007FA18EEE9DE190938403809383038CEE81
:10F8B0009DE1909382038093810388E592E0909389
:10F8C000800380937F0382E080937E0380915802BF
:10F8D000909159028FC08230910539F41A821982B1
:10F8E0001C821B828CE790E89FC08330910539F41D
:10F8F0001A8219821C821B8280E996E595C08430A9
:10F90000910509F041C01A8219821C821B828CE287
:10F9100090E3282F9E838D8388E8482FCC24C394BE
:10F92000E12CFA8000E01C813E815FEF60E070E036
:10F9300088ED98E00E947FA182EE9DE19093840380
:10F940008093830380EE9DE19093820380938103F3
:10F950008FE09DE09093800380937F0385E0809308
:10F960007E0380910F0D24E6829FC00111246FEF6A
:10F9700070E00F941D7170938C0360938B037093F0
:10F980007903609378039CC08530910509F043C0EA
:10F990001A8219821C821B828CE290E3282F9E839C
:10F9A0008D8388E8482FCC24C394E12CFA8000E0B2
:10F9B0001C813E815FEF60E070E088ED98E00E947E
:10F9C0007FA182ED9DE1909384038093830380ED7A
:10F9D0009DE1909382038093810386E592E090936A
:10F9E000800380937F0382E080937E0380915602A0
:10F9F0009091570290938C0380938B03909379039B
:10FA0000809378038AE090E090937D0380937C0359
:10FA100088EE93E05BC086309105A9F41A821982C2
:10FA20001C821B8281EA9AE7282F9E838D83188689
:10FA30001F82CC24C394E12CFA8000E01C813E811B
:10FA400040E058856BC08730910509F044C01A82A8
:10FA500019821C821B828CE290E3282F9E838D8367
:10FA600088E8482FCC24C394E12CFA8000E01C8164
:10FA70003E815FEF60E070E088ED98E00E947FA13A
:10FA800085EC9DE1909384038093830383EC9DE157
:10FA9000909382038093810382E292E090938003AB
:10FAA00080937F0381E080937E038091220290E027
:10FAB00090938C0380938B039093790380937803C6
:10FAC00010927D0310927C0384E690E090937B0378
:10FAD00080937A0329C02091330220FF25C0209112
:10FAE0007C0D2871283179F58830910511F029E0D5
:10FAF0002BC083E29DEEE82E9A8389831C821B82B1
:10FB00008AE29DEE282F9E838D8388E8482FCC249F
:10FB1000C394FA8000E01C813E815FEF60E070E0FA
:10FB200088ED98E00E947FA12A960FB6F894DEBF78
:10FB30000FBECDBFDF91CF911F910F91FF90EF903E
:10FB4000CF900C94793228E030E02817390761F71C
:10FB50001A8219821C821B828BE195EC282F9E83CE
:10FB60008D8388E8482FCC24C394E12CD2CFEF9228
:10FB7000FF920F931F93CF93DF93CDB7DEB7A0977C
:10FB80000FB6F894DEBF0FBECDBFF62EE42E8E0169
:10FB90000F5F1F4F90E2F80111929A95E9F78111DA
:10FBA00003C063E67DE111C0813019F464E57DE1B5
:10FBB0000CC0823019F466E47DE107C0833019F48B
:10FBC00062E37DE102C06EE27DE1C8010F94A2759F
:10FBD0004E2DB8018F2D0E94D62EA0960FB6F89408
:10FBE000DEBF0FBECDBFDF91CF911F910F91FF9070
:10FBF000EF900895EF92FF920F931F93CF93DF93AF
:10FC0000CDB7DEB7A0970FB6F894DEBF0FBECDBF5D
:10FC1000F62EE42E8E010F5F1F4F90E2F801119235
:10FC20009A95E9F7811103C063E17DE135C0813028
:10FC300019F46DE07DE130C0823019F461E07DE1BE
:10FC40002BC0833019F460EF7CE126C0843019F4B6
:10FC500066EE7CE121C0853019F468ED7CE11CC0C2
:10FC6000863019F46DEC7CE117C0873019F46EEB27
:10FC70007CE112C09091330290FF0CC090917C0DFA
:10FC800098719831F1F4883011F099E01BC060EB65
:10FC90007CE102C060EA7CE1C8010F94A2754E2DA0
:10FCA000B8018F2D0E94D62EA0960FB6F894DEBF15
:10FCB0000FBECDBFDF91CF911F910F91FF90EF90BD
:10FCC000089598E09813E6CF64EA7CE1E5CFEF92DF
:10FCD000FF920F931F9387EAE82E8FE1F82E00E63C
:10FCE0001FE324E339E84EE95FE16EE67FE880E058
:10FCF00090E00E94052D6FE87FE18AE00E946C375A
:10FD00006EE77FE184E10E946C3769E67FE18EE176
:10FD10000E946C3768E57FE188E20E946C371F9192
:10FD20000F91FF90EF900C947932EF92FF920F9326
:10FD30001F93CF93DF93CDB7DEB765970FB6F894D7
:10FD4000DEBF0FBECDBF8BEFE82E8EE1F82E05ECA7
:10FD500018E720E030E042EF5EE166E57FE380E017
:10FD600090E00E94052D6DED7EE18AE00E946C37E7
:10FD70006DEC7EE184E10E946C3763EC7EE18EE104
:10FD80000E946C378FE798E09F938F9385ED97E003
:10FD90009F938F938AEB9EE19F938F938E010F5FCA
:10FDA0001F4F1F930F930F947576B80188E20E943E
:10FDB0004E350E9479320FB6F894DEBF0FBECDBF2C
:10FDC00065960FB6F894DEBF0FBECDBFDF91CF9121
:10FDD0001F910F91FF90EF900895EF92FF921F9364
:10FDE000CF93DF931F921F92CDB7DEB71091110D05
:10FDF000E12EF12CF701EE0FFF1FEE0FFF1FE5586C
:10FE0000F74F608171818281938164D992E29E9DD6
:10FE100090019F9D300D1124F901E80FF11DEE0FA7
:10FE2000FF1FE656F84F808191819A838983612F65
:10FE3000CE0101960F94F25960E088ED98E00E949F
:10FE4000D2A10F900F90DF91CF911F91FF90EF9073
:10FE50000895EF92FF920F931F934091910388E0D2
:10FE6000840F405E682F0E945B330E9473328AE8E1
:10FE7000E82E8EE1F82E06E51FE320E030E046E8AC
:10FE80005EE16CEC78E784EE92E80E94052D65E770
:10FE90007EE184E10E946C374DEC55E060E28CE33A
:10FEA0000E94CF3A1F910F91FF90EF900C947932FE
:10FEB000CF92DF92EF92FF920F931F93CF93DF9336
:10FEC000CDB7DEB7A0970FB6F894DEBF0FBECDBF9B
:10FED000809170038330B9F480914B0981FD13C088
:10FEE0002091910330E0220F331F40912202429F64
:10FEF000C001439F900D112464E670E00F941D71C2
:10FF000088E00E946B254CE55EE16AE87AE780E0D4
:10FF100090E00E94552C4DE06CE783E00E945C3835
:10FF20008E010F5F1F4F80E2F80111928A95E9F769
:10FF30008091550990915609A0915709B09158099F
:10FF4000C0905909D0905A09E0905B09F0905C0983
:10FF5000BC01CD016C197D098E099F0928EE33E0A3
:10FF600040E050E00F94307169017A0166E57EE16E
:10FF7000C8010F94A275AE014A5F5F4FC701B60179
:10FF80000E9400A9FCE3CF16D104E104F10418F4A7
:10FF900062E57EE102C060E57EE10F948375B80101
:10FFA00085E00E944E3560911E0270911F02809183
:10FFB0002002909121020F94BE6DDC01CB014DE433
:10FFC0005EE1B8010E942A3D7C0160911A027091A5
:10FFD0001B0280911C0290911D020F94BE6DDC01EA
:10FFE000CB014BE45EE1B7010E942A3DB8018AE1F2
:10FFF0000E944E3510914B0913FF57C020E030E0AE
:020000021000EC
:1000000040E752E46091EB177091EC178091ED1787
:100010009091EE170F94526F181684F020E030E0A4
:1000200040E252E46091E3177091E4178091E51784
:100030009091E6170F94526F18169CF566E37EE1D7
:1000400080E10E946C3720E030E040E752E46091AC
:10005000EB177091EC178091ED179091EE170F94BC
:10006000756C9B01AC0160E070E088EF92E40F9446
:10007000756C0F94BE6D77FD06C06D3771052CF061
:100080006CE770E002C060E070E08091850390E072
:10009000681779071CF060938503CB010E94FF2D40
:1000A0001AC0177F10934B0916C011FD0AC040916A
:1000B000910388E0840F405E682F0E945B330E94AA
:1000C000733267E47DE080E10E944E3567E27EE1B5
:1000D00088E20E946C370E947932A0960FB6F8949D
:1000E000DEBF0FBECDBFDF91CF911F910F91FF906B
:1000F000EF90DF90CF9008950F931F93CF93DF93EE
:10010000CDB7DEB760970FB6F894DEBF0FBECDBF98
:1001100080918B0390918C039C012D5F3F4F273082
:100120003105D0F197FDC9019595879595958795EE
:100130002091F1173091F217820F931F97FD22C083
:1001400080E00F94E95920918B0330918C0337FFA5
:1001500002C02D5F3F4F35952795359527954091E6
:10016000F1175091F217240F351F0E9728173907F2
:1001700034F080E00F94E9599C012F503109922FFF
:10018000832F02C090E080E09093F1178093F217E4
:1001900010928C0310928B0380918A03882329F09C
:1001A00061E088ED98E00E94D2A10E948A3964E162
:1001B0007EE184E10E946C3764E07EE186E30E9488
:1001C0006C378E010F5F1F4F80E1F80111928A9505
:1001D000E9F760911E0270911F02809120029091B8
:1001E00021020F94BE6DDC01CB0141E05EE1B8015C
:1001F0000E942A3DF80101900020E9F7BF016150FB
:1002000071094FEF5DE18091F1179091F2170E9413
:100210002A3DB8018EE10E944E3580E090E00F94B7
:10022000C84D482F68E28EE30E948DAA0E94793261
:1002300060960FB6F894DEBF0FBECDBFDF91CF91B1
:100240001F910F910895CF93DF930E948A394EE258
:1002500065E080E40E947F3842E36CE783E00E941F
:100260005C3880917C0D83FD02C0D3E001C0D4E0F6
:100270004D2F6FED75E888ED98E00E9428A4C0E04E
:100280004C2F69E771E888ED98E00E9498A5CF5F50
:10029000CD13F6CFDF91CF910C947932CF93DF93CA
:1002A0000E948A394EE265E080E40E947F3842E392
:1002B0006CE783E00E945C3880917C0D83FD02C076
:1002C000D2E001C0D4E04D2F66E176E888ED98E0F9
:1002D0000E9428A4C0E04C2F62E172E888ED98E00B
:1002E0000E9498A5CF5FCD13F6CFDF91CF910C94EC
:1002F0007932CF92EF920F931F93CF93DF93EB015D
:10030000811115C0C88094E2E92E04E81CE124E2C2
:1003100044E369E087E00E94F4A3888146ED55E05C
:100320006DE182FF02C08EE11CC08EE126C090917B
:100330007C0D93FF2AC0813011F092E027C0C88065
:1003400084E2E82E0DE71CE124E244E369E087E45F
:100350000E94F4A3888182FF0CC04DEC55E06DE152
:100360008EE5DF91CF911F910F91EF90CF900C947C
:100370003E3B4DEC55E06DE18EE5DF91CF911F9155
:100380000F91EF90CF900C94CF3A91E0891320C059
:10039000088127E040E366E388E00E94C6A28881E6
:1003A00082FF0BC048E75CE166E387E10E946D369F
:1003B0004DEB55E066E38CE0D4CF43E75CE166E3C8
:1003C00087E10E947C354DEB55E066E38CE0D5CFAC
:1003D0009F5F891320C0088127E040E366E388E43B
:1003E0000E94C6A2888182FF0BC04EE65CE166E3F4
:1003F00087E50E946D3644EC55E066E38CE4B1CFAE
:1004000049E65CE166E387E50E947C3544EC55E013
:1004100066E38CE4B2CFDF91CF911F910F91EF9003
:10042000CF900895CF92EF920F931F93CF93DF93C6
:10043000EB0181111CC0C8800F94C141811103C020
:1004400008E51CE102C000E61CE184E2E82E24E29B
:1004500044E369E087E00E94F4A388814DED55E014
:100460006DE182FF02C08EE122C08EE138C0909122
:100470007C0D93FF80C08130D1F5088124E244E3F4
:1004800069E087E40E94C6A2888182FF18C041E526
:100490005CE16FE081E60E94F73748E45CE168E1E7
:1004A00081E60E94F7374FE855E061E28EE5DF9183
:1004B000CF911F910F91EF90CF900C943E3B41E470
:1004C0005CE16FE081E60E94923748E35CE168E11D
:1004D00081E60E9492374FE855E061E28EE5DF91B8
:1004E000CF911F910F91EF90CF900C94CF3A823023
:1004F00001F5088127E040E366E388E00E94C6A298
:10050000888182FF0BC043E35CE166E387E10E94E0
:100510006D364DEB55E066E38CE0C9CF4EE25CE111
:1005200066E387E10E947C354DEB55E066E38CE0A5
:10053000D6CF833019F5088127E040E366E388E4ED
:100540000E94C6A2888182FF0BC048E25CE166E39C
:1005500086E50E946D364DEC55E066E38AE4A7CF50
:1005600042E25CE166E386E50E947C354DEC55E0B5
:1005700066E38AE4B4CF813009F4BBCFDF91CF9139
:100580001F910F91EF90CF90089561E088ED98E072
:100590000E94D2A180917C0D8F7E80937C0DE09192
:1005A000110D84E0E89FF0011124E958F74F808194
:1005B0009181A281B381892B8A2B8B2B19F081E049
:1005C0008093E2070C94AD31CF92EF92FF920F939C
:1005D0001F93CF93DF93CDB7DEB72A970FB6F8946A
:1005E000DEBF0FBECDBF4091910388E0840F405E17
:1005F000682F0E945B330E9473328091F30C8F3F0F
:10060000B1F40E948A3969E67EE184E10E946C3788
:100610002A960FB6F894DEBF0FBECDBFDF91CF9103
:100620001F910F91FF90EF90CF900C94793260E082
:1006300088ED98E00E941BA21A8219821C821B82FC
:1006400088E59FE7282F9E838D8384E0482FC12C67
:10065000E12CFA8000E01C813E8150E060E070E017
:1006600088ED98E00E947FA12A960FB6F894DEBF2D
:100670000FBECDBFDF91CF911F910F91FF90EF90F3
:10068000CF900895BF92CF92DF92EF92FF920F9397
:100690001F93CF93DF93CDB7DEB72A970FB6F894A9
:1006A000DEBF0FBECDBF9091DE118091DD1198139A
:1006B00032C081E00E94DF6B1A8219821C821B8289
:1006C0008DEE9EE7282F9E838D8388E8D82E4D2DB2
:1006D000C12CE12CFA8000E01C813E815FEF60E0DC
:1006E00070E088ED98E00E947FA11A8219821C8236
:1006F0001B828AE899E5282F9E838D834D2DCC247B
:10070000C394FA801C813E815FEF60E070E088ED69
:1007100098E00E947FA12A960FB6F894DEBF0FBE24
:10072000CDBFDF91CF911F910F91FF90EF90DF90A0
:10073000CF90BF9008954F925F926F927F928F9269
:100740009F92AF92BF92CF92DF92EF92FF920F9360
:100750001F93CF93DF93CDB7DEB7A8970FB6F8946A
:10076000DEBF0FBECDBF80917C0D84FF3FC080EC0B
:1007700098E7E82E9A8389831C821B828EE491E895
:10078000282F9E838D8344E0D42EB12C4D2DDF8203
:10079000B88619861A86CC24C394FA8000E01C819E
:1007A0003E8150E060E070E088ED98E00E947FA11B
:1007B0000E94D4EF8111ECC11A8219821C821B8223
:1007C0008EE290EF282F9E838D834D2DDF82B88699
:1007D00019861A86E12CFA801C813E8150E060E087
:1007E00070E088ED98E00E947FA1D2C132E5E32E4F
:1007F0003FE1F32E00EC18E723E231E84DE45FE13E
:1008000060E070E089EF9BE70E94052D8091370F33
:100810009091380FA091390FB0913A0FBC01CD01E2
:1008200065587F4F8F4F9F4F2CE730E040E050E0FE
:100830000F94307160913F0F7091400F8091410F84
:100840009091420F0F943071122FCE0101967C01CE
:1008500080E2D7011D928A95E9F78091F30C8330ED
:1008600051F0843031F163E47FE184E10E946C3720
:1008700067E47DE03EC06BE37FE184E10E946C377A
:1008800060911E0270911F028091200290912102BE
:100890000F94BE6DDC01CB0146E35FE1B7010E941E
:1008A0002A3D49E35FE1BC018091F1179091F21775
:1008B0001DC063E27FE184E10E946C3760911A02FF
:1008C00070911B0280911C0290911D020F94BE6DCD
:1008D000DC01CB014EE15FE1B7010E942A3D41E21C
:1008E0005FE1BC018091E9179091EA170E942A3DCF
:1008F000B7018EE10E944E350E949324C0905909A1
:10090000D0905A09E0905B09F0905C096C197D0960
:100910008E099F090F94EF6D4B015C0120E030E0E0
:100920004AE754E40F94566D6B017C016091370FD8
:100930007091380F8091390F90913A0F0F94EF6DAD
:100940009B01AC01C501B4010F9424704B015C0103
:1009500060913F0F7091400F8091410F9091420F35
:100960000F94EF6D9B01AC01C501B4010F94566D5E
:100970006DA37EA38FA398A720E030E04AE754E45C
:100980000F94566D69A37AA38BA39CA320E030EC4F
:1009900049E754E46091DE077091DF078091E0073A
:1009A0009091E1070F94247029A13AA14BA15CA179
:1009B0000F94766C20E030E04AE754E40F94566DD3
:1009C0004B015C012B013C01E89477F82FEF3FEFDE
:1009D0004FE75FE7C301B2010F94D27081110AC0E3
:1009E0002FEF3FEF4FE75FE7C301B2010F944F6D69
:1009F00018164CF08092DE079092DF07A092E00775
:100A0000B092E1070CC08DA19EA1AFA1B8A58093C3
:100A1000DE079093DF07A093E007B093E1074090D3
:100A200073085090740860907508709076084114AF
:100A3000510461047104E9F420E030E040E752E43D
:100A4000C701B6010F944F6D87FF13C089A19AA10A
:100A5000ABA1BCA18093DE079093DF07A093E007D2
:100A6000B093E1074CE05FE16AE085E00E947C35ED
:100A70008AC0C301B20196958795779567950F94C3
:100A8000EF6D4B015C019B01AC01C701B6010F94F6
:100A90004F6D87FF43C0A5019401C701B6010F94B4
:100AA000566D4B015C0120E030E040E85FE30F94BD
:100AB000526F181634F4812C912C80E8A82E8FE305
:100AC000B82E2091DE073091DF074091E00750916A
:100AD000E107C501B4010F94247069A37AA38BA325
:100AE0009CA3C301B2010F94EF6D2B013C01A50142
:100AF000940160E070E080E89FE30F94756C9B01C7
:100B0000AC01C301B2010F9424709B01AC0169A137
:100B10007AA18BA19CA10F94766C08C06091DE072E
:100B20007091DF078091E0079091E1070F94C36D0A
:100B30000F94EF6D4B015C019B01AC01C701B60145
:100B40000F94526F18164CF0A7019601C501B4011D
:100B50000F94756C0F94C36D04C061E070E080E089
:100B600090E0AE014F5F5F4F0E949A3D42E05FE12F
:100B70006AE085E00E947C35AE014F5F5F4F6AE01E
:100B800081E40E946233812F0E94FF2D0E947932FE
:100B9000A8960FB6F894DEBF0FBECDBFDF91CF9100
:100BA0001F910F91FF90EF90DF90CF90BF90AF908B
:100BB0009F908F907F906F905F904F900895FB0172
:100BC000811107C011821082138212828AE992E990
:100BD0000EC090917C0D93FF13C0813011F092E014
:100BE00010C011821082138212828DE199E79583E1
:100BF000848388E89FEF978386831086118614C0CC
:100C000091E0891307C0118210821382128287EE4D
:100C100098E7EDCF9F5F891307C01182108213827E
:100C2000128286E59FE3E3CFCF010895FB01811196
:100C300007C0118210821382128285EC92E815C0DF
:100C400090917C0D93FF23C0813039F41182108282
:100C50001382128282E493E808C0823079F4118210
:100C600010821382128287EE98E79583848388E846
:100C70009FEF97838683108611860BC0833049F4DB
:100C800011821082138212828DE199E7EECF8130BA
:100C900031F3CF010895BF92CF92DF92EF92FF928E
:100CA0000F931F93CF93DF93CDB7DEB7E5970FB6C2
:100CB000F894DEBF0FBECDBFF82EB62EE42E8E0107
:100CC0000F5F1F4F85E3F80111928A95E9F7F11044
:100CD0000DC08091F30E811103C065EB7FE102C06E
:100CE0006EEA7FE1C8010F94A2755BC0E7EEF7E002
:100CF00020E030E080818F110EC087E1829FB0013B
:100D0000839F700D11246751784F44E150E0C80172
:100D10000F94537606C02F5F3F4F779626303105EC
:100D200049F7898181112BC024E1A8016FEF6F0D74
:100D30008AE39DE00F94B9638F2D66E00F94FD70F8
:100D4000F7E19F9FC00111249C012951384F69018F
:100D5000F901F08244E150E0B8018751984F0F94B7
:100D60005376F601168A80917C0D86FB992790F9BF
:100D700091839091F60E992311F085FD27C0E2FE34
:100D800010C0809172088F110CC080918808882350
:100D900041F040E250E068E878E0CE0145960F94DB
:100DA00053764E2DB8018B2D0E94D62EE5960FB6A8
:100DB000F894DEBF0FBECDBFDF91CF911F910F9191
:100DC000FF90EF90DF90CF90BF9008951092F60EB5
:100DD0008FEFF60180831092470DD1CF8F929F92B3
:100DE000AF92BF92CF92DF92EF92FF920F931F9339
:100DF000CF93DF93CDB7DEB7C054D1090FB6F894C7
:100E0000DEBF0FBECDBF882309F409C2E7EEF7E0CD
:100E1000E12CF12C90819813F9C1182F87E18E9D58
:100E2000F0018F9DF00D1124E951F84F818181303F
:100E300031F461EA70E286E30E946C37F0C1809180
:100E40007208811709F4F1C06FEF610F8AE39DE02A
:100E50000F94776210927B0D6EE270E087E49DE064
:100E60000F942A76009711F0FC0110828091F60E03
:100E7000882379F01092F60E87E18E9DF0018F9D08
:100E8000F00D1124E951F84F8FEF80831092470D38
:100E9000C6C11093720810927308109274081092D1
:100EA00075081092760810927708109278081092C0
:100EB000790810927A088DEC9CECACECBEE3809340
:100EC0007B0890937C08A0937D08B0937E081092D5
:100ED0007F0810928808E7E4FDE001900020E9F720
:100EE000CF0188549D40459740F040E250E06BE5CB
:100EF0007DE088E898E00F94537641E06AE37DE076
:100F0000CB010F94595D80911F0F81110BC080910F
:100F1000F60E882309F489C01092F60E8FEF8093A5
:100F2000720883C080E1F82E8E010F5F1F4F20E012
:100F300030E040E450E0B8018CE19FE00F94BF2323
:100F400021961FAE2197F80101900020E9F7329712
:100F5000E017F10730F08081803218F41082319769
:100F6000F7CF46E050E06AE970E2C8010F94CA7515
:100F7000892B89F440E050E060E070E0CE010796F4
:100F80000F942E746093730870937408809375089F
:100F90009093760846C04AE050E06FE870E2C801DE
:100FA0000F94CA75892B89F44AE050E060E070E044
:100FB000CE010B960F942E74609377087093780887
:100FC0008093790890937A082CC041E150E06DE756
:100FD00070E2C8010F94CA75892B79F460E070E063
:100FE000CE0142960F94C87260937B0870937C0880
:100FF00080937D0890937E0814C047E050E065E739
:1010000070E2C8010F94CA75892B59F448E050E08A
:10101000BE01685F7F4F8FE798E00F945376109280
:101020008608FA94F11083CF72CF80917308909163
:101030007408A0917508B0917608892B8A2B8B2BA8
:1010400009F4DDC08091900381111AC08091770866
:1010500090917808A0917908B0917A08892B8A2B11
:101060008B2B09F0AEC080917B0890917C08A091F9
:101070007D08B0917E08892B8A2B8B2B09F0A1C0AB
:10108000809191038F33C0F0809177089091780818
:10109000A0917908B0917A08892B8A2B8B2BA1F526
:1010A00080917B0890917C08A0917D08B0917E088A
:1010B000892B8A2B8B2B41F56FE670E2CE010196CE
:1010C0000F94A275609173087091740880917508EF
:1010D00090917608AE014A5F5F4F0E9400A940914F
:1010E00073085091740860917508709176084C33BC
:1010F00051056105710518F46BE670E202C069E6FE
:1011000070E20F94837573C06FE570E2CE010196B3
:101110000F94A27520E030E040E05FE36091D107DA
:101120007091D2078091D3079091D4070F942470C7
:101130006B017C0160917708709178088091790843
:1011400090917A080F94EF6D4B015C012BED3FE01D
:1011500049E450E4C701B6010F942470A701960139
:101160000F9424709B01AC01C501B4010F94566D1E
:101170006B017C0120E030E44CE156E40F944F6DAC
:1011800020E030E04AE754E487FF0BC0C701B60116
:101190000F94566D00E02DE530E2AE01465F5F4FE3
:1011A00024C0C701B6010F94566D0F94BE6DDC01CB
:1011B000CB014BE550E2BE01665F7F4F0E942A3DA6
:1011C00016C063E570E2CE0101960F94A27560919E
:1011D0007B0870917C0880917D0890917E0800E0EA
:1011E00020E030E0AE01485F5F4F0E945D3EAE01FF
:1011F0004F5F5F4F66E383E00E94623310C041E4BB
:1012000050E266E383E00E947C3509C09FEFE91A53
:10121000F90A779696E0E916F10409F0FBCDC05C77
:10122000DF4F0FB6F894DEBF0FBECDBFDF91CF9179
:101230001F910F91FF90EF90DF90CF90BF90AF90F4
:101240009F908F900895E7EEF7E08FEF8083878B74
:1012500086A780932C088093430880935A08809334
:101260007208809371080895CF92DF92EF92FF92F7
:101270000F931F93CF93DF93CDB7DEB7CA56D10933
:101280000FB6F894DEBF0FBECDBF80917C0D85FDFB
:1012900029C04091910388E0840F405E682F0E942E
:1012A0005B330E94733284E090E090938C038093D0
:1012B0008B0340E050E066E57FE380E090E00E9431
:1012C000552C65E370E28FE00E946C3762E270E2B9
:1012D00089E10E946C370E9479328AE39DE00F9485
:1012E000485D9EC280FF04C08091F60E8823A9F05D
:1012F00040E050E066E57FE380E090E00E94552CFE
:1013000062E170E280E10E946C370E9479329BDFDB
:101310008AE39DE00F94575C83C2809171088F3FF0
:1013200031F48AE39DE00F949D628093710880916F
:10133000F60E882321F08FEF8093710871C280919F
:10134000710881111CC08091F30E811107C04FE01C
:1013500050E266E57FE38FE898EC06C04CE050E28F
:101360006DE97AE784E399E80E94552C6CEF7FE100
:1013700089E10E946C370E94793265DF51C2809109
:101380008A03882309F44FC060918B0370918C030A
:1013900077FF02C06D5F7F4F75956795759567956F
:1013A00061157105A1F48091F30E811108C00E94AE
:1013B0008FC861E088ED98E00E94D2A134C043DF7D
:1013C0000E94CB3B8AE39DE00F9466632CC0615082
:1013D0008AE39DE00F94776280917C0D86FD14C0B6
:1013E00010924B091092110D41E06AE37DE0CB01B0
:1013F0000F94595D80911F0F882309F411C20E9438
:10140000ECF58823F1F00CC20E94CB3B1CDF6AE3B1
:101410007DE0CB010F94CF6282E090E090938C034B
:1014200080938B03FDC1609171086F5F2EEE36E8EB
:101430004BE456E88EEB9FE10E94452F0E947932E3
:10144000EFC1809170038250823068F48091220253
:101450002FEF829FC001112464E670E00F941D718C
:1014600088E00E946B258091470D811108C044E3FC
:1014700050E06AE37DE087E49DE00F94537610929C
:101480005B0D6EE270E087E49DE00F942A76009792
:1014900011F0FC01108220E030E040E450E0BE0199
:1014A0006F5F7F4F8CE19FE00F94BF2321961FAEAB
:1014B000219741E150E06AEE7FE1CE0101960F9461
:1014C000CA75892B71F020E030E040E450E0BE01A5
:1014D0006F5F7F4F8CE19FE00F94BF2321961FAE7B
:1014E000219710923F0F1092400F1092410F1092CF
:1014F000420F40E050E0BA018CE19FE00F94E924F4
:101500000E946D2B61E088ED98E00E941BA2109272
:10151000CE0C10920F0D84E690E0909359028093C8
:10152000580210922D0910922E0910922F09109234
:10153000300924E62093490240E050E060E87FE370
:1015400040930F1750931017609311177093121751
:1015500090935702809356021092310910923209EB
:10156000109233091092340941E150E068ED7FE1B7
:10157000CE0101960F94CA758E010F5B1F4F892B08
:1015800009F028C11092EA171092E9171092490247
:101590008091770890917808A0917908B0917A08A5
:1015A000892B8A2B8B2B09F442C01092F2171092D0
:1015B000F1178091CC079091CD079093EA17809313
:1015C000E9178091CE078093490220E030E040E0A7
:1015D0005FE36091D1077091D2078091D30790911A
:1015E000D4070F9424706B017C012BED3FE049E49C
:1015F00050E40F942470A70196010F9424709B016E
:10160000AC0160E070E080E89FE30F94566D60935A
:101610000F177093101780931117909312178091E2
:10162000CF079091D00790935702809356028091F4
:10163000F30C8630B1F48EE79BEEE82EF80191832F
:1016400080831382128285E89BEE282F9583848302
:101650008CE1482F8683178210861186CC24C39490
:10166000CCC0109247091092480910924909109273
:101670004A091092110D80E2F80111928A95E9F75A
:101680000E94A7576091160D7091170D8091180D4B
:101690009091190D0F94BE6D77FF02C060E070E06D
:1016A0006B5F7F4F7F936F936091120D7091130D5D
:1016B0008091140D9091150D0F94BE6D77FF02C0AF
:1016C00060E070E06B5F7F4F7F936F9386EC9FE1EC
:1016D0009F938F931F930F930F947576C8010F9468
:1016E000C51B1092F30C809133020FB6F894DEBF45
:1016F0000FBECDBFA3961FAE1EAEA397A5961FAE7D
:101700001EAEA59780FF03C080E59CEC02C087EE6B
:101710009FE8282FA7969FAF8EAFA79788E8482FFE
:10172000A8968FAFA8978FEFA9968FAFA997CC24D3
:10173000C394E12CA396FFACA39700E0A5961FAD40
:10174000A597A7963FADA7975FEF60E070E088EDA3
:1017500098E00E947FA16FE778E085ED97E00F9415
:101760001776892B09F45CC08091D507882309F48A
:1017700057C080917F08882309F452C0A3961FAEFA
:101780001EAEA397A5961FAE1EAEA59785E99EE750
:10179000282FA7969FAF8EAFA79788E8482FA896C7
:1017A0008FAFA8978FEFA9968FAFA997C12CE12C87
:1017B000A396FFACA39700E0A5961FADA597A796AB
:1017C0003FADA7975FEF60E070E088ED98E00E9482
:1017D000F1A026C0F801118210821382128287E6DE
:1017E0009EE7282F9583848384E0482F8683178281
:1017F00010861186CC24C394E12C2396FFAC23974A
:1018000000E025961FAD259727963FAD279729968F
:101810005FAD299760E070E088ED98E00E947FA1BD
:10182000C659DF4F0FB6F894DEBF0FBECDBFDF91B4
:10183000CF911F910F91FF90EF90DF90CF9008957F
:10184000CF92EF92FF920F931F93CF93DF9300D02D
:101850001F921F92CDB7DEB78D830E94DFF51092E5
:1018600087031092860390917C0D8D8193FF02C0B7
:1018700094FFF3C0977E90937C0D882319F00F940A
:10188000084A0EC0EE24E3940091110D26E33DE0DA
:1018900042E35DE06EE27DE08AE29DE00F94CE409F
:1018A00084E690E0909359028093580290935702F7
:1018B000809356028091E207882309F45AC0109160
:1018C000110D84E0189FF0011124E15FF84E208192
:1018D00031814281538160912D0270912E0280915D
:1018E0002F02909130020F94566D2091F80C222314
:1018F00049F02091450230914602409147025091B3
:10190000480203C020E030E0A9010F94756C6983A0
:101910007A838B839C8341E0612FCE0101960F94E3
:101920008D411092360D1092370D1092380D109295
:10193000390D20E030E040E752E4609141027091BF
:10194000420280914302909144020F94566DC090E0
:10195000110D7B018C0126E33DE042E35DE06EE288
:101960007DE08AE29DE00F946F361092F80C1092A1
:10197000E2070E94492B0F94964920E030E040EFA7
:1019800051E46091520270915302809154029091FF
:1019900055020F94756C9B01AC016091320D7091F2
:1019A000330D8091340D9091350D0F94526F1816B0
:1019B0002CF40E946C4B0E94A35702C00E94A757B0
:1019C0000F94EB1B0F94024A1092360D1092370DB4
:1019D0001092380D1092390D41E06091110D86E39F
:1019E0009DE00F948D410E9493246093550970935C
:1019F000560980935709909358090E9482958091C7
:101A00007C0D877E80937C0D1092F30C8091700387
:101A1000823029F460E070E088E00E946B2584E663
:101A20008093490280E090E0A0E8BFE380930F1725
:101A300090931017A0931117B09312171092CE0C19
:101A40000F900F900F900F900F90DF91CF911F91FB
:101A50000F91FF90EF90CF9008954091320D5091EB
:101A6000330D6091340D7091350D409347095093BB
:101A700048096093490970934A09FCCECF92EF92CE
:101A8000FF920F931F93CF93DF93CDB7DEB72A97C3
:101A90000FB6F894DEBF0FBECDBF8091F30C9AEF66
:101AA000980F9230E0F18F3FD1F180917C0D83FD52
:101AB00036C00E94ECF5811132C09091DE11809108
:101AC000DD1198132CC0109247091092480910920A
:101AD000490910924A0980914B09886080934B090B
:101AE00060E088ED98E00E941BA21A8219821C8295
:101AF0001B8288E59FE7282F9E838D8384E0482FF3
:101B0000C12CE12CFA8000E01C813E8150E060E0B5
:101B100070E088ED98E00E947FA180E033C0809162
:101B2000FA0C882361F080914B098D7F80934B09DB
:101B30001A8219821C821B828AE799E70FC0809162
:101B4000F60E882369F180914B098D7F80934B09B4
:101B50001A8219821C821B8283E599E7282F9E83B3
:101B60008D8384E0482FCC24C394E12CFA8000E0DC
:101B70001C813E8150E060E070E088ED98E00E94BA
:101B8000F1A081E02A960FB6F894DEBF0FBECDBF5C
:101B9000DF91CF911F910F91FF90EF90CF9050CE9A
:101BA0002A960FB6F894DEBF0FBECDBFDF91CF915E
:101BB0001F910F91FF90EF90CF9008959F92AF9259
:101BC000BF92CF92DF92EF92FF920F931F93CF932A
:101BD000DF9300D01F92CDB7DEB78091F30C863033
:101BE00009F46CC120E030E040EF51E46091470916
:101BF000709148098091490990914A090F94766C37
:101C00007B018C0120E030E040EF51E46091520212
